:100000000C94A30A0C94D40A0C94D40A0C94D40A29
:100010000C94D40A0C94D40A0C94D40A0C94D40AE8
:100020000C94D40A0C94D40A0C94D40A0C94D40AD8
:100030000C94D40A0C94338C0C94D40A0C94D40AE7
:100040000C94D40A0C94D40A0C94D40A0C94D40AB8
:100050000C94D40A0C94D40A0C94D40A0C94A7518E
:100060000C94D40A0C94005D0C94D75C0C94D40AC4
:100070000C94D40A0C94D40A0C94D40A0C94D40A88
:100080000C94D40A0C94D40A0C94D40A0C94D40A78
:100090000C94AE5C0C94855C0C94D40A0C94598D31
:1000A0000C94D40A0C94D40A0C94D40A0C94D40A58
:1000B0000C94D40A0C94D40A0C94D40A0C94D40A48
:1000C0000C94D40A0C94D40A0C94D40A0C945C5C5E
:1000D0000C94335C0C94D40A0C940A5C0C94E15B91
:1000E0000C94D40A671D4E1EB61DAF1D7F1D6F1DDB
:1000F0004E1E6B1D4E1E4E1E4E1E4E1E4E1E610B84
:10010000CA0B3C0C950D0010C211CA11F812FE1258
:1001100006133D13521356134E1E98139C13A0132F
:100120005E15E2161B188A185219D219241C281DB4
:10013000753521363E36523666367A369736AB36C8
:10014000BF36DC36F03604371837F6370A381E3833
:100150006D5070505F5063506950A7507450785084
:100160007E50825086508C5090509450A7509A5098
:100170009E50A250084AD73B3BCE016E84BCBFFDC7
:10018000C12F3D6C74319ABD56833DDA3D00C77F67
:1001900011BED9E4BB4C3E916BAAAABE0000008000
:1001A0003F07634236B79BD8A71A39685618AEBACC
:1001B000AB558C1D3CB7CC5763BD6DEDFD753EF660
:1001C000177231BF000000803F08000000BE92247B
:1001D00049123EABAAAA2ABECDCCCC4C3E000000B0
:1001E00080BEABAAAAAA3E00000000BF00000080AB
:1001F0003F0000000000084178D3BB4387D1133D86
:10020000190E3CC3BD4282AD2B3E68EC8276BED94E
:100210008FE1A93E4C80EFFFBE01C4FF7F3F00008D
:10022000000000004E414E494E495459494E46CDBA
:10023000CCCC3D0AD7233C17B7D13877CC2B32959D
:1002400095E6241FB14F0A000020410000C842007B
:10025000401C4620BCBE4CCA1B0E5AAEC59D740045
:10026000407A10F35A00A0724E18090010A5D4E885
:100270000000E87648170000E40B54020000CA9A18
:100280003B000000E1F5050000809698000000406A
:10029000420F000000A086010000001027000000AF
:1002A00000E803000000006400000000000A0000F5
:1002B0000000000100000000002C76D888DC674FA9
:1002C0000823DFC1DFAE59E1B1B796E5E3E453C6D9
:1002D0003AE651997696E8E6C28426EB898C9B62D1
:1002E000ED407C6FFCEFBC9C9F40F2BAA56FA5F47B
:1002F00090055A2AF75C936B6CF9676DC11BFCE0A3
:10030000E40D47FEF520E6B500D0ED902E030094F5
:100310003577050080841E080000204E0A0000008A
:10032000C80C333333330F986E12831141EF8D2194
:1003300014893BE65516CFFEE6DB18D1844B381BFB
:10034000F77C1D901DA4BBE424203284725E2281C0
:1003500000C9F124ECA1E53D274D6F74696F6E0073
:100360004E6F2053656E736F7221004E6F204453A1
:1003700020546865726D6F6D657465722100445319
:1003800020546865726D2E00555620496E742E00FB
:10039000555620496E74656E7369747900434F3207
:1003A00020436F6E630053656E736F7220657272C7
:1003B0006F722100234E6F2073656E736F72210080
:1003C000434F3220436F6E63004D656173757269F0
:1003D0006E6700234E6F2073656E736F7220666FB9
:1003E000722074656D7020262068756D696469746B
:1003F0007921004E6F2053656E736F722100206665
:100400006F722074656D7020262068756D6964694F
:10041000747921002353656E736F72204572726F79
:1004200072200053656E736F72204572726F722175
:10043000002357726F6E672073656E736F7220664C
:100440006F722074656D7020262068756D6964690F
:100450007479210057726F6E672053656E736F72E7
:10046000210054656D702048756D69646974790068
:100470004C6967687420496E74656E73697479009D
:10048000466C616D6520495200482D6669656C6453
:100490000053656172636820446972656374696FB3
:1004A0006E004E6F2073656E736F7221004952208B
:1004B00054656D7065726174757265004D65617328
:1004C0007572696E672E2E004E6F2073656E736FA6
:1004D000723F0049522054656D7065726174757287
:1004E00065004D6561737572696E672E2E00234E2F
:1004F0006F2070482073656E736F72210070482002
:1005000076616C75650023496E76616C6964206B59
:1005100065792100204D756C746973656E736F7217
:1005200073004D756C746973656E736F72730044FC
:10053000697361626C6500456E61626C650052654D
:10054000626F6F74696E672E2E2E002344413A2D20
:10055000323300237265706C6965733D0023546902
:100560006D65206475726174696F6E3D0023546916
:100570006D6520696E74657276616C3D00576946E1
:10058000692049503A00234D5320456E61626C65E5
:100590006400234D532044697361626C65640023D9
:1005A0005265737420706172616D65746572732039
:1005B000746F2064656661756C742076616C756516
:1005C00073004C6F67676572204E616D653A20005D
:1005D000232D2D2D2D2D2D2D2D2D2D2D2D2D2D2D55
:1005E0002D2D2D2D2D2D2D2D2D2D2D2D2D2D2D2D3B
:1005F0002D2D2D2D2D00235265736F6C7574696F31
:100600006E3A20202000234D696E2056616C75657E
:100610003A2020202000234D61782056616C7565BA
:100620003A202020200023556E69717565204944C9
:100630003A20202020002344726976657220566596
:10064000723A202020002353656E736F723A202087
:10065000202020202000232D2D2D2D204D61676E80
:10066000657469632053656E736F72202D2D2D2D77
:100670002D2D2D2D2D2D2D2D2D2D2D2D2D2D2D2DAA
:1006800000482D6669656C643A20280020202020EF
:10069000202020202020202020202020002020207A
:1006A000202020202020202020202020200020206A
:1006B000202020202020202020202020202000205A
:1006C000202020202020202020202020202020004A
:1006D000202020202020202020202020202020003A
:1006E000202020202020202020202020202020002A
:1006F000233A53686F772F48696465204C43440060
:100700002A3A546869732048656C700044233A4360
:10071000616C6962726174696F6E00442A3A536554
:100720007474696E67730044433A436C6561722068
:100730004C43440044423A5265736574204C6F67E1
:100740006765720044303A566F6C746167650044A7
:10075000393A43757272656E7400566F6C746167D6
:10076000652B43757272656E740044383A456C654A
:1007700063747269630044373A4D6F74696F6E0039
:1007800044363A44532054656D700044353A55560A
:1007900020496E74656E736974790044343A4F323F
:1007A00020636F6E632E0044333A434F3220636FF1
:1007B0006E632E0044323A504D28313A322E353A8B
:1007C0003130290044323A504D28313A322E353AF0
:1007D0003130292A0044313A54757262696469746F
:1007E000790044303A566F6C7461676500393A6F2E
:1007F0007220334420616363656C2E00393A496E80
:10080000636C2E20616E672E00383A704820766146
:100810006C756500373A49522054656D7000373A5F
:1008200049522054656D702A00363A4D61676E65F5
:10083000746963206669656C6400353A47617320AA
:100840004C6576656C00343A495220466C616D65A2
:1008500000333A4C6967687420496E742E00323A4E
:10086000616E642048656967687400323A54656D4A
:100870007020507265737375726500313A54656DFE
:10088000702048756D696469747900303A536F75EA
:100890006E64204C6576656C00303A536F756E64FB
:1008A000204C6576656C2A0054696D65206C61701A
:1008B00073653A00576946692049503A00696E707D
:1008C00075742044535463616C6962726174653A53
:1008D0000020766F6C746167653D00235475726209
:1008E0006964697479205570706572204C696D690E
:1008F000743A200020766F6C746167653D00235464
:100900007572626964697479204C6F776572204CE6
:10091000696D69743A200023547572626964697460
:1009200079204C6F776572204C696D697420566927
:100930006E663A20004D61782072616E67653D00F9
:1009400023566F6C746167652073656E736F723ABE
:1009500000342D32306D4100414353373132204D48
:1009600061783D00414353373132204D61783D3548
:1009700041002343757272656E742073656E736FE8
:10098000723A0023445320546865726D6F6D65742C
:1009900065722063616C6962726174656420666F60
:1009A00072202300234E6F206E65656420746F20D3
:1009B00063616C6962726174652063757272656EE1
:1009C000742073656E736F72210023414353373176
:1009D000322063757272656E742073656E736F7208
:1009E000206F666673657420563D00235556207A45
:1009F00065726F20766F6C74616765203D00234FD0
:100A00003220766F6C253D00234F322063616C6984
:100A100062726174696F6E3A200023566F6C746164
:100A200067652870483D3130293A0023566F6C7451
:100A30006167652870483D34293A006765745365DD
:100A40006C665465737442697428293A200069738E
:100A5000496E74657272757074456E61626C65641E
:100A60002831293A2000676574496E746572727581
:100A700070744D617070696E672831293A20006783
:100A80006574496E74657272757074536F757263B4
:100A9000652831293A2000676574496E7465727261
:100AA000757074536F7572636528293A2000676505
:100AB000745261746528293A20332E313431353926
:100AC0003F00616363656C2E69734C6F77506F777D
:100AD000657228293A2000616363656C2E69734151
:100AE000736C65657028293A2000616363656C2E1C
:100AF0006973546170536F757263654F6E5A28291C
:100B00003A2000616363656C2E6973546170536FA2
:100B1000757263654F6E5928293A200061636365D9
:100B20006C2E6973546170536F757263654F6E58A4
:100B300028293A2000616363656C2E6973416374F0
:100B40006976697479536F757263654F6E5A282997
:100B50003A2000616363656C2E6973416374697642
:100B6000697479536F757263654F6E5928293A20FD
:100B70000069734163746976697479536F75726340
:100B8000654F6E5828293A20006973546170446596
:100B900074656374696F6E4F6E5A28293B206661D5
:100BA0006C73653F200069735461704465746563BC
:100BB00074696F6E4F6E5A28293B20747275653FB9
:100BC00020006973546170446574656374696F6E65
:100BD0004F6E5928293B2066616C73653F20006980
:100BE00073546170446574656374696F6E4F6E59B8
:100BF00028293B20747275653F2000697354617029
:100C0000446574656374696F6E4F6E5828293B2084
:100C100066616C73653F200069735461704465744C
:100C2000656374696F6E4F6E5828293B2074727526
:100C3000653F200067657453757070726573734209
:100C4000697428293B2066616C73653F20006765E5
:100C500074537570707265737342697428293B20F0
:100C6000747275653F2000697341637469766974B5
:100C700079416328293A20006973496E6163746978
:100C8000766974795A456E61626C656428293A20E8
:100C9000006973496E616374697669747959456E48
:100CA00061626C656428293A20006973496E61634A
:100CB00074697669747958456E61626C6564282937
:100CC0003A2000697341637469766974795A456E94
:100CD00061626C656428293A200069734163746914
:100CE0007669747959456E61626C656428293A2089
:100CF000006973416374697669747958456E6162FD
:100D00006C656428293A20006765744672656546FB
:100D1000616C6C4475726174696F6E28293A2000A9
:100D20006765744672656546616C6C54687265737C
:100D3000686F6C6428293A200067657454696D6592
:100D4000496E616374697669747928293A2000676D
:100D50006574496E61637469766974795468726503
:100D600073686F6C64282920006765744163746937
:100D7000766974795468726573686F6C6428292089
:100D800000676574446F75626C6554617057696E75
:100D9000646F7728292000676574446F75626C65FD
:100DA0005461704C6174656E637928293A2000673C
:100DB00065745461704475726174696F6E28293A64
:100DC0002000676574417869734F6666736574289F
:100DD00026782C2026792C20267A293A200067654F
:100DE000745461705468726573686F6C6428293A32
:100DF000200058595A2047733A200058595A204326
:100E00004F554E54533A2000736574206761696EE4
:100E1000735B5D3A006761696E735F6F7269675BF0
:100E20005D3A002353657474696E6773206F6620A2
:100E3000616C6C2073656E736F72733A0023536933
:100E40007A65206F6620686561646572202B206179
:100E50006C6C2073656E736F72733A200023536954
:100E60007A65206F66206865616465723A20004388
:100E7000616C6962726174696F6E20507265737320
:100E80007572653D00536561206C6576656C205018
:100E90002863616C63293D00234572726F723A705A
:100EA0007265737375726520424D503038352C2051
:100EB000636865636B20776972696E6721004952C8
:100EC0002054656D702073656E736F7220666F7548
:100ED0006E6400504D322E352073656E736F722034
:100EE0006C696B656C7920666F756E6400206D6F40
:100EF00062696C65206C6F676765722073746172DC
:100F000074656420616E64207265616479210057A4
:100F10006946692049503A0023576946692049507B
:100F200020616464726573733A2000456455484BD0
:100F3000205345534C6F676765720053656E736F3E
:100F40007220736C6F7420616E6420747970653ADE
:100F50000057656C636F6D6520746F20456455485C
:100F60004B00005EBCE2613FDD83C29C7E20A3FD9E
:100F70001F41009D23BE46DB65F88C11AF32CA5776
:100F8000E97400002100240027002A002D00300011
:100F9000330001010000040107010A0100002200E2
:100FA000250028002B002E00310034000201000033
:100FB000050108010B010000200023002600290084
:100FC0002C002F003200000100000301060109017E
:100FD00005050505070508080808020202020A0AB5
:100FE00008080404040401010101010101010303D3
:100FF000030303030303040707070C0C0C0C0C0C7E
:101000000C0C0202020206060606060606060B0B7A
:101010000B0B0B0B0B0B01021020200808102040BB
:1010200010204080020102010804020101020408AC
:10103000102040808040201008040201800402013A
:101040008040201008040201080402010102040883
:1010500010204080010204081020408000000A0B8C
:1010600002090C0D0E080703040100000000000037
:101070000000000000000000000000000000000070
:10108000000000000000000012111000000000002D
:101090000000000000000000000000000000000050
:1010A000000046696E64696E672057694669204989
:1010B0005000697465726174696F6E3D0073656E8E
:1010C000736F72233D0043757272656E7420737482
:1010D000617475733A206379636C653D006E637962
:1010E000636C653D006E73656E736F72733D006D6A
:1010F00061786E73656E736F72733D00656E6162C9
:101100006C65643D00234D756C746973656E736F17
:101110007273206D6561737572656D656E74207391
:10112000657474696E67733A007365703D00697623
:10113000616C3D006E697465723D00230043616C13
:101140002E204661696C65640043616C2E20446FFB
:101150006E65004E6F206E6565642100496E766194
:101160006C6964205028506129005365614C657694
:10117000656C2050285061293A0043616C696272A5
:101180006174652050004453542054656D70207381
:10119000656E736F720043757272656E742073654D
:1011A0006E736F72004F322073656E736F720055ED
:1011B000562073656E736F720043616C6962726171
:1011C0007465004661696C65640054422063616C1B
:1011D0002E20646F6E65005570706572204C696DCD
:1011E00069743A3E004C6F776572204C696D697482
:1011F0003A3E0054757262696469747900466169A7
:101200006C65640070482063616C2E20646F6E65AD
:10121000007048313020507265737320420070486E
:101220003420507265737320410043616C696272AF
:10123000617465004E45543D426C7565746F6F7402
:1012400068204C45004E45543D426C7565746F6F87
:101250007468004E45543D5769466900556E6B6E83
:101260006F776E00496E647573747269616C2034B7
:101270002D32306D4100414353373132204D61787A
:101280003D3541002343757272656E742073656E3F
:10129000736F723A0053657474696E6720466169B2
:1012A0006C65640053657474696E6720446F6E6585
:1012B000004368616E6765204E6574776F726B3EA0
:1012C00000547970653A0042542F57694669204EA0
:1012D0006574776F726B004368616E676520536554
:1012E0006E736F723E0043757272656E7420536543
:1012F0006E736F72004F7468657200496E642E20C1
:10130000342D32306D4100414353373132203C336C
:10131000304100414353373132203C3230410041AB
:101320004353373132203C3541003E4D61782056E1
:101330006F6C743A3E004368616E676520766F6C2F
:10134000746167653E00547970652000566F6C7457
:101350006167652053656E736F72004368616E67E5
:1013600065207479706520746F0053656E736F72B9
:101370003D4448540054656D702048756D6964693A
:1013800074790023456E64206F66204D756C746916
:1013900073656E736F72204379636C6523004572C9
:1013A000726F72206E756D62657220666F72207446
:1013B000686520617272617920746F206176726154
:1013C00067696E67212F6E004F3220436F6E630096
:1013D000234E6F2073656E736F7220666F7220509C
:1013E0004D21004E6F2073656E736F722100206E69
:1013F000672F4C00504D313A322E353A3130004D86
:101400006561737572696E672E2E00234E6F2073AF
:10141000656E736F722100536F756E64204C657634
:10142000656C004D6561737572696E672E2E0023C1
:101430004E6F2073656E736F722100536F756E640B
:10144000204C6576656C00234E6F205442207365F6
:101450006E736F723F004D6F74696F6E004F6666FA
:10146000206169722D636F6E6421004974277320B7
:10147000746F6F20636F6F6C210054656D7020690D
:10148000732066696E6521004973206169722D635E
:101490006F6E64206F6E3F00497427732071756909
:1014A000746520686F742100497427732076657213
:1014B0007920686F742120004F6666206169722D63
:1014C000636F6E6421004974277320746F6F20630B
:1014D0006F6F6C210054656D702069732066696EB2
:1014E0006521004973206169722D636F6E64206FFE
:1014F0006E3F004974277320717569746520686FA9
:1015000074210049742773207665727920686F749E
:10151000210054656D702048756D696469747900A7
:10152000416E676C65732F003E6128782C792C7AA8
:10153000292F673A00496E76616C6964206B657982
:101540002100FCAA5EAD11241FBECFEFD1E2DEBFA9
:10155000CDBF00E00CBF1CE0A0E0B2E0ECEDF4E792
:1015600001E00BBF02C007900D92AC37B107D9F76D
:1015700024E1ACE7BCE001C01D92A933B207E1F75A
:101580001AE0C2EADAE000E006C021970109802FE4
:10159000FE010E94A0B7C13AD10780E00807A9F771
:1015A0000E94CDA10C945DBA0C9400002F923F9242
:1015B0004F925F926F927F928F929F92AF92BF9263
:1015C000CF92DF92EF92FF920F931F93CF93DF930F
:1015D000CDB7DEB7C554D1090FB6F894DEBF0FBE44
:1015E000CDBF8C01E090BD0CF090BE0C8091C50C7D
:1015F000882349F063E575E08EE89FE00E94EF5A8A
:10160000C8010E94497C680125E0C20ED11C85E01A
:10161000C816D10428F18091BD0C9091BE0C8017A2
:10162000910731F10E9448320E94AA910C3E9FEF2F
:10163000190724F01093BE0C0093BD0C4AE0B801CA
:10164000CE0101960E94275ABE016F5F7F4F8BEA41
:1016500092E10E945F59CE0101960E94985908C0FC
:101660000E3FAFEF1A0721F40E94BA910C94841F29
:1016700062EC79E08FE992E10E943559B5E0CB1632
:10168000D10490F065EC7BE0CE0101960E94825A75
:101690004AE050E06FEF7FEFCE0101960E941733D2
:1016A000CE0101960E949859F8017C96E632F10528
:1016B00010F00C944E1E8827EE58FF4F8F4F0C945D
:1016C000A0B70E94483289E390E00E945A9A20E035
:1016D00030E04AE754E40E9427B3AB01BC0121E0AB
:1016E000CE0101960E94CC5965EC75E0CE0145967D
:1016F0000E94825ABE016F5F7F4FCE0145960E94C5
:10170000A85868EC75E00E949158BC018FE992E1FD
:101710000E944A59CE0145960E949859CE010196E1
:101720000E9498596CEC75E089E992E10E94355964
:1017300069E972E1CE0101960E947A5A4AE050E0CE
:1017400068E070E0CE0101960E94D133CE0101968F
:101750000E9498596FE972E1CE0101960E947A5A6F
:101760004AE050E06FEF7FEFCE0101960E94983281
:10177000CE0101960E94985969E972E18FE992E1E0
:101780000E9409598091B013882311F40C94801E93
:101790000C94F114E0903105F09032050E9448322B
:1017A00089E390E00E945A9A0E94B1B528EE33E096
:1017B000269FF001279FF00D369FF00D11244AE07F
:1017C000BF01CE0101960E94275A65EC75E0CE015B
:1017D00045960E94825ABE016F5F7F4FCE014596AB
:1017E0000E94A85868EC75E00E949158BC018FE9EE
:1017F00092E10E944A59CE0145960E949859CE0125
:1018000001960E9498598091A3129091A412099771
:1018100010F022E001C023E0C70124962FAF2497E7
:101820000E94E79AAB01BC0124962FAD2497CE010C
:1018300001960E94CC5960E376E0CE0145960E9465
:10184000825ABE016F5F7F4FCE0145960E94A85815
:1018500064ED75E00E949158BC018FE992E10E940D
:101860000959CE0145960E949859CE0101960E94D1
:10187000985967ED75E058CF8091B013882309F42B
:1018800048C184E59EE00E94295D61E080911E02CE
:101890000E94DA5060E080911C020E94DA500E949F
:1018A000BB836093BF0C7093C00C8093C10C90936A
:1018B000C20C0E94448F0E94618FAB01BC0123E0E7
:1018C000CE0145960E94CC59BE016B5E7F4FCE0182
:1018D00001960E947A5A6DE276E0CE0101960E944E
:1018E0009158BC0189E992E10E944A59CE010196C2
:1018F0000E949859CE0145960E94985963E47CE075
:10190000CE0101960E94825A69E972E1CE010196E8
:101910000E94A858BC018FE992E10E944A59CE0169
:1019200001960E9498590E94618F9B01AC012496F8
:101930006FAF249723963FAF239725964FAF2597F8
:1019400026965FAF26970E943E512B013C016EE127
:1019500070E080E090E00E9463510E94618F6B0113
:101960007C010E943E514B015C0184189508A60839
:10197000B70824962FAD249723963FAD239725963D
:101980004FAD259726965FAD2697E1ED8E16E7E0E1
:101990009E06A104B1040CF43FC0C701B6010E9429
:1019A00051B46B017C0120E030E0A9010E9407B630
:1019B00018165CF426EA3BE944EC5BE3C701B60188
:1019C0000E94C2B287FF0BC027C026EA3BE944EC65
:1019D0005BEBC701B6010E9407B61816ECF0C50113
:1019E000B40128EE33E040E050E00E94F4B3CA01B5
:1019F000B9010E94C8B24B015C0120E030E04AE727
:101A000054E4C701B6010E9427B3A50194010E94C6
:101A100018B5AB01BC0103C040E050E0BA0122E0C0
:101A2000CE0145960E94CC59BE016B5E7F4FCE0120
:101A300001960E947A5A60EE75E0CE0101960E94EE
:101A40009158BC0183E992E10E944A59CE01019666
:101A50000E949859CE0145960E94985964EE75E00F
:101A6000CE0101960E94825A63E972E1CE0101968D
:101A70000E94A858BC018FE992E10E940959CE0149
:101A800001960E94985965EC7BE0CE0101960E9478
:101A9000825A63E972E1CE0101960E94A858BC0106
:101AA00089E992E10E940959CE0101960E94985954
:101AB00069E573E0CE0101960E94725A4AE050E057
:101AC00060E070E0CE0101960E94D133CE01019614
:101AD0000E94985969E972E1CE0101960E947A5AF2
:101AE00045E050E06FEF7FEFCE0101960E94983203
:101AF000CE0101960E94985968EE75E08FE992E157
:101B00000E94FB5860E080911E020E94DA500C9403
:101B1000801E6091000270910102809102029091FA
:101B200003020E94A38F0C94801ED0900C0262ECE2
:101B300079E0CE01C5960E94825A7E01F5E1EF0E52
:101B4000F11C6D2DC7010E943455F886EF821D826D
:101B50001E82198289E08A8381E08B838C831C8AB0
:101B60001B8ACE0101960E949054CE0101960E94DC
:101B70002353CE0101960E94FC7EEE80F12C23E0DF
:101B8000E216F10409F46EC16EE773E0CE01C5966A
:101B90000E940F5962EC79E08FE992E10E94355979
:101BA000BE016B5C7F4FCE0183960E947A5A4AE059
:101BB00050E060E070E0CE0183960E94D133CE0108
:101BC00083960E94985961E080E00E94B1656AE0C6
:101BD00076E0CE01C5960E94355946EC842E4CE045
:101BE000942EAA24A394B12CC12CD12CCE14DF04A2
:101BF0000CF0EFC06C2DCE0101960E942254D4014E
:101C00002D913D914D915D914D010E9452B42B015A
:101C10003C0120E030E04CEF52EC0E94C2B287FF62
:101C200021C04AE0B501CE0183960E94275A65E69D
:101C300077E0CE0189960E94825ABE016D5D7F4F8A
:101C4000CE0189960E94A8586BEF75E00E949158CA
:101C5000BC018FE992E10E940959CE0189960E9448
:101C6000985945C022E0B301A201CE0183960E949B
:101C7000CC594AE0B501CE0189960E94275A65E603
:101C800077E0CE018F960E94825ABE01675D7F4F3A
:101C9000CE018F960E94A85862ED7AE00E9491587A
:101CA000BE016D5D7F4F0E94A858BC0183E992E19F
:101CB0000E944A59CE018F960E949859CE0189966A
:101CC0000E949859CE0183960E94985963E972E167
:101CD000CE0183960E947A5A65EC7BE0CE01839612
:101CE0000E949158BC018FE992E10E940959CE01EE
:101CF00083960E949859B1E0EB16F10459F4C1148F
:101D0000D10409F05FC06FE972E1CE01C5960E946F
:101D10004A5958C0E2E0EE16F10411F522E0B30191
:101D2000A201CE0189960E94CC59BE01675D7F4F0A
:101D3000CE0183960E947A5A65EC7BE0CE018396B1
:101D40000E949158BC01CE01C5960E940959CE014E
:101D500083960E949859CE0189960E94985932C064
:101D6000F3E0EF16F10471F163E972E1CE018396BD
:101D70000E947A5A44E150E06FEF7FEFCE018396E4
:101D80000E949832CE0183960E9498596CE976E0C1
:101D9000CE0183960E94825ACE0183960E946C32B5
:101DA000CE0183960E94985980910802882351F0B1
:101DB00080910C05882331F060ED77E080E090E0C1
:101DC0000E9463512FEFC21AD20A8FEFA81AB80AE5
:101DD0000DCFCE01C5960E949C578FE992E10E94DB
:101DE0009C57E114F104A9F46BE673E08FE992E1EA
:101DF0000E940F5960E673E0CE0183960E94725AEA
:101E00004AE050E06FEF7FEFCE0183960E94983258
:101E1000EFC094E0E916F10414F00C94A01EBE018A
:101E20006B5C7F4FCE0183960E947A5A4AE050E065
:101E30006FEF7FEFCE0183960E949832CE0183969A
:101E40000E9498596CE976E0CE0183960E94825AEE
:101E5000CE0183960E946C32CE0183960E949859DF
:101E60000C94A01E67E076E0CE01C5960E9435591D
:101E7000BE016B5C7F4FCE0183960E947A5A4AE086
:101E800050E060E070E0CE0183960E94D133CE0135
:101E900083960E94985962EC79E08FE992E10E9462
:101EA00035596FE972E1CE01C5960E944A59E12C7D
:101EB000F12C6E2DCE0101960E9422544B015C0143
:101EC00022E0AB01BC01CE01E114F10469F4839678
:101ED0000E94CC59BE016D5D7F4F8AE993E10E945B
:101EE000E15ACE0183961BC089960E94CC59BE014F
:101EF000675D7F4FCE0183960E947A5A65EC7BE046
:101F0000CE0183960E949158BC01CE01C5960E94D5
:101F10000959CE0183960E949859CE0189960E9454
:101F2000985922E0B501A401CE0189960E94CC59AE
:101F3000BE01675D7F4FCE0183960E947A5A65ECA1
:101F40007BE0CE0183960E949158BC018FE992E11B
:101F50000E940959CE0183960E949859CE01899614
:101F60000E949859AFEFEA1AFA0AB3E0EB16F104AF
:101F700009F09FCFCE01C5960E949C57BE016B5CB5
:101F80007F4FCE0183960E947A5A4AE050E06FEF6D
:101F90007FEFCE0183960E949832CE0183960E94F5
:101FA00098596CE976E0CE0183960E94825ACE0160
:101FB00083960E946C32CE0183960E9498598FE9D5
:101FC00092E10E949C576DE076E0CE0183960E94DC
:101FD000825A6FE972E1CE0183960E94A85867E1A8
:101FE00076E00E949158BC018FE992E10E944A5923
:101FF000CE0183960E949859CE01C5960C947E1E00
:10200000E0910E022296EFAF229760E08E2F0E94A1
:10201000DA508091B01381110AC08091941181111E
:1020200006C03FE0C32ED12CE12CF12C05C023E0EB
:10203000C22ED12CE12CF12C60E973E08FE992E102
:102040000E940F596FE972E1CE0101960E947A5AFF
:102050004AE050E06FEF7FEFCE0101960E94D1334E
:10206000CE0101960E9498591BAE1CAE1DAE1EAE4D
:102070001FAE21961FAE2197212C312C92E3692EA1
:10208000712C812C912C540122968FAD22970E94A5
:102090001951092E000CAA0BBB0B880E991EAA1E03
:1020A000BB1E65E070E080E090E00E946351F1E0CB
:1020B0006F1A710849F740901F05509020056090F5
:1020C000210570902205C501B4010E94C8B220E02C
:1020D00030E040EA50E40E9427B320E030E040E8DE
:1020E0005AE30E9427B320E030E048E452E40E9423
:1020F00018B5A30192010E9451B420E030E040E7FE
:1021000051E40E9427B34B015C01A30192016AE9EB
:1021100079E989E390E40E9451B49B01AC01C501C7
:10212000B4010E9418B520E030E0A9010E9452B429
:1021300020E030E040E251E40E9427B34B015C0113
:102140002FAD21963FAD2197A1010E9407B6181629
:102150002CF48FAE21969FAE2197150120E030E040
:10216000A901B401C5010E94C2B287FF04C0812C3D
:10217000912CA12CB12C22E0A401B501CE014596F1
:102180000E94CC59BE016B5E7F4FCE0101960E942A
:102190007A5A6AE276E0CE0101960E949158BC011B
:1021A00089E992E10E944A59CE0101960E9498590C
:1021B000CE0145960E94985969E972E1CE010196D7
:1021C0000E947A5A4AE050E060E070E0CE01019649
:1021D0000E949832CE0101960E9498590E949B510C
:1021E00040907C0C50907D0C60907E0C70907F0C29
:1021F0005301420124E6820E911CA11CB11C8616DB
:102200009706A806B90610F40C94A81E0E949B51CC
:102210000E94C6B24B015C01C301B2010E94C8B268
:1022200020E030E048EC51E40E9452B49B01AC0144
:10223000C501B4010E94C2B287FF02C00C94A81E5F
:102240006CE370E080E090E00E9463518BAD9CAD48
:10225000ADADBEAD0196A11DB11D8BAF9CAFADAFB5
:10226000BEAFC816D906EA06FB060CF007CF64E637
:1022700070E080E090E00E9463510E94483264E682
:1022800070E080E090E00E94635168E873E089E9C3
:1022900092E10E940F5969E972E1CE0101960E9414
:1022A0007A5A44E150E060E070E0CE0101960E946D
:1022B000D133CE0101960E94985922E04FAD21966C
:1022C0005FAD2197B101CE0145960E94CC59BE0168
:1022D0006B5E7F4FCE0101960E947A5A6AE276E0E9
:1022E000CE0101960E949158BC0189E992E10E94B9
:1022F0004A59CE0101960E949859CE0145960E94F6
:10230000985969E972E1CE0101960E947A5A42E336
:1023100050E06FEF7FEFCE0101960E949832CE0120
:1023200001960E94985964E170E080E090E00E947C
:1023300063510E948A326EE170E080E090E00E947A
:1023400063516EE170E080E090E00E9463516FE2C3
:1023500076E0CE0101960E94825A69E972E1CE01CF
:1023600001960E94A85863E376E00E9491586FE9B5
:1023700072E10E94A858BC018FE992E10E944A597B
:102380000C947C1E80911002909111020E94877A19
:102390000C94801E0E94483269EC73E08FE992E150
:1023A0000E940F596FE972E1CE0101960E947A5A9C
:1023B0004AE050E060E070E0CE0101960E94D13327
:1023C000CE0101960E94985960EC73E089E992E190
:1023D0000E940F5969E972E1CE0101960E947A5A72
:1023E00044E150E06FEF7FEFCE0101960E949832FA
:1023F000CE0101960E9498598091AE139091AF132F
:102400008230910549F40E9459A081111AC010929E
:10241000AF131092AE1315C0892B99F40E9459A0E6
:10242000882339F082E090E09093AF138093AE134D
:1024300008C00E9459A08111F5CF0E9459A08111B6
:10244000F1CF8091AE139091AF13029739F164EB05
:1024500073E08FE992E10E940F596FE972E1CE01BA
:1024600001960E947A5A4AE050E060E070E0CE01A6
:1024700001960E94D133CE0101960E9498596FE9CE
:1024800072E1CE0101960E947A5A65EC7BE0CE01A2
:1024900001960E94915869E972E134C68AE090E0A1
:1024A0000E94E6916B017C0120E030E0A9010E94CE
:1024B000C2B2181634F08AE090E00E94E6916B01F7
:1024C0007C018BE0A82EB12C20E030E042ED53E4FB
:1024D000C701B6010E94C2B2181684F420E030E0B1
:1024E000A901C701B6010E94C2B21816C4F066EA7B
:1024F00073E08FE992E10E940F5942C091E0A91A5E
:10250000B10861F368EC70E080E090E00E946351F4
:1025100083E090E00E94E6916B017C01D5CF20E042
:1025200030E048EC52E4C701B6010E94C2B287FF16
:1025300002C021E001C020E0B701A601CE01019652
:102540000E94CC5967E376E0CE0145960E94825AFC
:10255000BE016F5F7F4FCE0145960E94A8586CE385
:1025600076E00E949158BC018FE992E10E944A599D
:10257000CE0145960E949859CE0101960E94985925
:102580006FE972E1CE0101960E947A5A42E350E06F
:102590006FEF7FEFCE0101960E949832CE01019637
:1025A0000E9498596DE973E089E992E10E940F5900
:1025B00069E972E1CE0101960E947A5A42E350E045
:1025C00060E070E0CE0101960E94D133CE01019609
:1025D0000E9498598091B013882311F40C94801EA6
:1025E00060E273E080E090E00E9463510C94801EF2
:1025F0000E949B510E946F780C94801E80910A0269
:1026000090910B020E94447D0C94801EE090310555
:10261000F09032050E94483265E070E080E090E082
:102620000E946351C7010E94E79AAB01BC0123E0FD
:10263000CE0101960E94CC5960E376E0CE0145962A
:102640000E94825ABE016F5F7F4FCE0145960E9465
:10265000A85864ED75E00E949158BC018FE992E1A1
:102660000E944A59CE0145960E949859CE01019682
:102670000E94985960E476E057C89091A80C81E0D8
:1026800089278093A80C8091B013882331F06FE9DB
:1026900072E187EB9DE00E94D05B68EC70E080E027
:1026A00090E0A2CF1092B0130C94801E81E0809332
:1026B000B0138093A21180919911882349F161EBA5
:1026C00077E08BEA92E10E94355986EE9FEF909376
:1026D000BE0C8093BD0C20919C1130919D11809176
:1026E0009E1190919F118217930724F010929F11D1
:1026F00010929E11109290111092911110929211BD
:10270000109293116CE271E080E090E00E946351BE
:102710006BEA72E181EB92E10E944A598091BD0C13
:102720009091BE0C9093AD138093AC130C94801ECB
:102730000E9477340C94801E0E9484760C94801E34
:1027400062E674E0CE0101960E94725A4AE050E0BF
:102750006FEF7FEFCE0101960E949832CE01019675
:102760000E94985960912F057091300580911D0548
:1027700090911E050E943995B4E18B2E912CA12CCD
:10278000B12CC12CD12CBFEFCB1ADB0AC501B4018F
:102790000E94635160912F057091300580911D0555
:1027A00090911E050E9439957C01E3E0CE16D1047C
:1027B00034F4A4E18A0E911CA11CB11CE4CFFEE10B
:1027C000CF16D1041CF4892BA1F703C0009709F0A0
:1027D0000DC180911D0590911E058B309105C9F4A6
:1027E0008091F7129091F812A091F912B091FA121B
:1027F00080932F1490933014A0933114B09332141B
:102800008091F3129091F412A091F512B091F6120A
:102810001DC08631910521F30C9701F5809122149A
:1028200090912314A0912414B091251480932F1417
:1028300090933014A0933114B093321480911E14ED
:1028400090911F14A0912014B091211480932B1407
:1028500090932C14A0932D14B0932E1440912F1408
:1028600050913014609131147091321421E0CE01F6
:1028700001960E94CC596AE076E0CE0145960E940E
:10288000825ABE016F5F7F4FCE0145960E94A858C5
:10289000BC018FE992E10E944A59CE0145960E94FF
:1028A0009859CE0101960E94985940912B1450914D
:1028B0002C1460912D1470912E1421E0CE010196FC
:1028C0000E94CC5968E476E0CE0145960E94825A77
:1028D000BE016F5F7F4FCE0145960E94A858BC0194
:1028E0008FE992E10E940959CE0145960E949859BC
:1028F000CE0101960E94985963EF7BE08FE992E147
:102900000E94FB5862EC79E0CE0101960E94825A47
:1029100044E150E060E070E0CE0101960E94D133C6
:10292000CE0101960E949859C0902F14D090301477
:10293000E0903114F090321420E030E0A901C7019A
:10294000B6010E9407B620E030E040E05FE387FD7B
:1029500005C0C701B6010E9452B404C0C701B60148
:102960000E9451B40E94B1B52AE0AB01BC01CE0176
:1029700001960E94FB59BE016F5F7F4F89E992E18A
:102980000E945F59CE0101960E94985960E087E04D
:102990000E94B16569E972E18AE993E10E94E15A16
:1029A0006FED8AE993E10E94DA5A6EE476E08AE9F3
:1029B00093E10E94E05B60912B1470912C14809144
:1029C0002D1490912E140E94B1B54AE050E08AE98E
:1029D00093E10E94B75B63EF7BE08AE993E10E9499
:1029E000E05B64E670E080E090E0FECD8F3F9F4FBB
:1029F000ACF064E574E0CE0101960E94725A4AE0A0
:102A000050E060E070E0CE0101960E94D133CE012B
:102A100001960E94985961E374E04AC08EEFE8166F
:102A20008FEFF80689F163E274E0CE0101960E940F
:102A3000725A4AE050E060E070E0CE0101960E94D8
:102A4000D133CE0101960E94985964E174E08FE978
:102A500092E10E940F594AE0B701CE0101960E940F
:102A6000275ABE016F5F7F4F8FE992E10E9409599B
:102A7000CE0101960E9498596EEF73E08FE992E1C2
:102A80000E94B9580C94801E63EF73E0CE0101964A
:102A90000E94725A4AE050E060E070E0CE01019678
:102AA0000E94D133CE0101960E94985963ED73E0E4
:102AB0008FE992E10E940F590C94801E80912002B0
:102AC000882311F40C94801E62EC79E0CE0101960B
:102AD0000E94825A4AE050E061E070E0CE01019627
:102AE0000E94D133CE0101960E9498590E9448322B
:102AF0000E94E1812B013C010E94BB834B015C01E0
:102B000060913D0270913E0280913F02909140029F
:102B10000E94C8B29B01AC0124966FAF2497239604
:102B20003FAF239725964FAF259726965FAF269701
:102B30000E94E1810E94C8B224962FAD249723966B
:102B40003FAD239725964FAD259726965FAD2697E7
:102B50000E9418B521E03EED42E45EE30E94C0B65B
:102B60009B01AC0160E070E080E89FE30E9451B4FB
:102B700020E03AE24DE257E40E9427B36B017C016A
:102B8000C301B2010E94C8B220E030E048EC52E438
:102B90000E9418B5AB01BC0122E0CE0101960E9453
:102BA000CC59BE016F5F7F4F83E992E10E945F596C
:102BB000CE0101960E94985969E778E083E992E195
:102BC0000E94FB5863E972E189E992E10E944A5947
:102BD00065E778E0CE0101960E94825A63E972E1CE
:102BE000CE0101960E94A858BC0183E992E10E949F
:102BF0004A59CE0101960E9498596AE076E08FE921
:102C000092E10E94355921E0B501A401CE0101965F
:102C10000E94CC59BE016F5F7F4F8FE992E10E9405
:102C20000959CE0101960E94985961E576E08FE935
:102C300092E10E94FB5821E0B701A601CE01459622
:102C40000E94CC59BE016B5E7F4FCE0101960E945F
:102C50007A5A6DE276E0CE0101960E949158BC014D
:102C60008FE992E10E940959CE0101960E9498597C
:102C7000CE0145960E94985963E972E1CE01019612
:102C80000E947A5A65EC7BE0CE0101960E94915831
:102C90006FE972E10E94A858BC018FE992E10E949D
:102CA0004A59CE0101960E94985921E0B501A4012C
:102CB000CE0101960E94CC59BE016F5F7F4F85EA1D
:102CC00092E10E945F59CE0101960E94985965EAEF
:102CD00072E1CE0101960E947A5A4AE050E060E02B
:102CE00070E0CE0101960E94D133CE0101960E9480
:102CF000985965E070E080E090E00E9463516CE9D3
:102D000076E0CE0101960E94825ACE0101960E9481
:102D10006C32CE0101960E94985969E972E1CE01A8
:102D200001960E947A5A4AE050E06FEF7FEFCE01A1
:102D300001960E949832CE0101960E94985920E097
:102D4000B701A601CE0145960E94CC59BE016B5E2B
:102D50007F4FCE0101960E947A5A6DE276E0CE0155
:102D600001960E949158BC0185EA92E10E944A595D
:102D7000CE0101960E949859CE0145960E9498591D
:102D800065EA72E1CE0101960E947A5A4AE050E06B
:102D900064EF7FEFCE0101960E949832CE0101963A
:102DA0000E94985965E070E080E090E00E946351D5
:102DB0008091B013882309F4A3C768E572E080E02E
:102DC00090E012CC8091B01381110AC080919411CF
:102DD000811106C0AEE18A2E912CA12CB12C05C028
:102DE000F3E08F2E912CA12CB12C60E774E08FE9D9
:102DF00092E10E940F596FE972E1CE0101960E94A3
:102E00007A5A4AE050E06FEF7FEFCE0101960E94C0
:102E10009832CE0101960E949859412C512C3201D2
:102E2000C12CD12C760183E20E94966587E090E068
:102E30000E9491650E948F6566E970E080E090E0F5
:102E40000E94635183E20E94966580E290E00E94B6
:102E500091650E948F6566E970E080E090E00E94D5
:102E6000635162E070E083E290E00E94688140E09C
:102E700050E0BA0180916B0D90E020916C0D821BA7
:102E80009109181619062CF58BE290E125964FAFA3
:102E9000259726965FAF269723966FAF23972496A4
:102EA0007FAF24970E94B48B25964FAD2597269629
:102EB0005FAD269723966FAD239724967FAD249719
:102EC000762F652F542F4427480F511D611D711D0A
:102ED000D1CFCB01BA010E94C8B22AE939E949E948
:102EE0005FE30E9418B50E94B1B5AB01BC01C416E6
:102EF000D506E606F70614F46A017B012AE0CE0146
:102F000045960E94FB59BE016B5E7F4FCE01019634
:102F10000E947A5A67E576E0CE0101960E949158A8
:102F2000BC0189E992E10E944A59CE0101960E94B2
:102F30009859CE0145960E94985969E972E1CE01EF
:102F400001960E947A5A4EE150E060E070E0CE01B6
:102F500001960E941733CE0101960E9498599FEF67
:102F6000491A590A690A790A84149504A604B7040F
:102F70000CF059CF2AE0B701A601CE0145960E9478
:102F8000FB59BE016B5E7F4FCE0101960E947A5ABB
:102F900067E576E0CE0101960E949158BC0189E96F
:102FA00092E10E944A59CE0101960E949859CE01A1
:102FB00045960E94985969E972E1CE0101960E94F6
:102FC0007A5A4AE050E060E070E0CE0101960E943B
:102FD000D133CE0101960E9498592AE0B701A6018B
:102FE000CE0101960E94FB5965ED79E0CE01459630
:102FF0000E94825ABE016F5F7F4FCE0145960E94AC
:10300000A8586BE576E00E9491586FE972E10E9442
:10301000A858BC018FE992E10E944A59CE01459619
:103020000E949859CE0101960E94985962E370E07F
:1030300080E090E0D9CAE0902D05F0902E0581E067
:103040008093520264E670E080E090E00E94635159
:103050000E944832C7010E94409460E074E0681BFF
:10306000790B4AE0CE0101960E94275A60E676E08D
:10307000CE0145960E94825ABE016F5F7F4FCE01FE
:1030800045960E94A858BC018FE992E10E944A59D6
:10309000CE0145960E949859CE0101960E949859FA
:1030A00060E087E00E94B16560E874E0CE010196BF
:1030B0000E94725A42E350E068E070E0CE0101964F
:1030C0000E94D133CE0101960E9498596FE972E1B6
:1030D000CE0101960E947A5A42E350E06FEF7FEFF3
:1030E000CE0101960E949832CE0101960E94985915
:1030F00067E676E0CE0101960E94825A6FE972E19E
:10310000CE0101960E94A858BC018FE992E10E946D
:103110004A595CCA80912B0590912C050E944094DD
:103120007C019093850C8093840C62E370E080E0D6
:1031300090E00E9463514AE0B701CE0101960E94DF
:10314000275ABE016F5F7F4F8FE992E10E945F595E
:10315000CE0101960E9498598091F1129091F2123D
:10316000892B09F45DC06DEE72E1CE0145960E9497
:103170007A5ABE016B5E7F4FCE0101960E947A5A49
:1031800044E150E060E070E0CE0101960E94D1334E
:10319000CE0101960E94985961E776E0CE01019632
:1031A0000E94825A6FE972E1CE0101960E94A858EE
:1031B000BC0189E992E10E944A59CE0101960E9420
:1031C000985969E972E1CE0101960E947A5A44E168
:1031D00050E06FEF7FEFCE0101960E949832CE0152
:1031E00001960E949859BE016B5E7F4FCE010196F9
:1031F0000E947A5A65EC7BE0CE0101960E949158BC
:1032000069E972E10E94A858BC018FE992E10E942D
:103210004A59CE0101960E949859CE014596D8C9C7
:103220006CE776E089E992E10E94355969E972E13B
:10323000CE0101960E947A5A44E150E060E070E0CD
:10324000CE0101960E94D133CE0101960E94985979
:1032500060E676E0CE0101960E94825A6FE972E143
:10326000CE0101960E94A858BC0189E992E10E9412
:103270004A59CE0101960E94985969E972E1CE013E
:1032800001960E947A5A44E150E06FEF7FEFCE0141
:1032900001960E949832CE0101960E94985961E7EA
:1032A00076E028CF80912002882309F429C58091F7
:1032B000B013811104C080919411882329F082E019
:1032C00090E00E949E381CC5C0900002D090010280
:1032D000E0900202F090030220E030E040E450E48D
:1032E000C701B6010E9407B618166CF420E030E062
:1032F0004AEF54E4C701B6010E9427B30E94B1B55A
:103300006B017C0106C050E3C52E55E7D52EE12C9C
:10331000F12C0E94483260E080E00E94B16561E9D2
:1033200074E08AE993E10E94EF5A61E080E00E9434
:10333000B16569E874E08AE993E10E94EF5A64E6B6
:1033400070E080E090E00E9463510E949B51609386
:10335000800C7093810C8093820C9093830C0E945C
:103360009B518090800C9090810CA090820CB0902A
:10337000830CDC01CB0188199909AA09BB098C15BA
:103380009D05AE05BF050CF0BBC483E090E00E9434
:103390009E380E949B5164E170E080E090E00E94C2
:1033A0006351DDCF8091B013811102C00E94483279
:1033B0008091210290912202029751F08091C30CDA
:1033C0009091C40C009709F4A1C1039709F49EC120
:1033D0006CEB74E089E992E10E940F5969E972E1AE
:1033E000CE0101960E947A5A44E150E060E070E01C
:1033F000CE0101960E94D133CE0101960E949859C8
:103400006DEA74E089E992E10E940F5969E972E17D
:10341000CE0101960E947A5A44E150E06FEF7FEFAF
:10342000CE0101960E949832CE0101960E949859D1
:1034300087E00E942581BC0180E090E00E94C6B236
:103440002AE037ED43EA5CE30E9427B323E333E944
:1034500048E853E40E9451B42B013C010E9454817E
:103460006B017C0144E0A42EB12C20E030E048EC5C
:1034700052E4C701B6010E9407B6181684F4A1E011
:10348000AA1AB10809F4D1C064E670E080E090E0C7
:103490000E9463510E9454816B017C01E6CF21E0C0
:1034A000B301A201CE0101960E94CC5962E976E0F7
:1034B000CE0145960E94825ABE016F5F7F4FCE01BA
:1034C00045960E94A858BC018FE992E10E944A5992
:1034D000CE0145960E949859CE0101960E949859B6
:1034E0006FE972E1CE0101960E947A5A42E350E000
:1034F0006FEF7FEFCE0101960E949832CE010196C8
:103500000E9498596CE976E0CE0101960E94825A99
:10351000CE0101960E946C32CE0101960E9498590C
:103520006BE976E08FE992E10E94FB5821E0B70158
:10353000A601CE0101960E94CC596AE076E0CE0148
:1035400045960E94825ABE016F5F7F4FCE0145961D
:103550000E94A858BC0185EA92E10E944A59CE0116
:1035600045960E949859CE0101960E94985965ECA3
:103570007BE0CE0101960E94825A65EA72E1CE019B
:1035800001960E94A858BC0189E992E10E944A591B
:10359000CE0101960E94985969E972E1CE01019627
:1035A0000E947A5A4AE050E060E070E0CE01019655
:1035B0000E941733CE0101960E9498596CE976E07B
:1035C000CE0101960E94825ACE0101960E946C3271
:1035D000CE0101960E9498596BE976E085EA92E166
:1035E0000E94FB5865EA72E1CE0101960E947A5A68
:1035F00065EC7BE0CE0101960E9491586FE972E183
:103600000E94A858BC018FE992E10E944A59CE015C
:1036100001960E9498598091C30C9091C40C039715
:1036200009F062C084E090E05BC062EA74E089E97E
:1036300092E10E940F5969E972E1CE0101960E9460
:103640007A5A4AE050E060E070E0CE0101960E94B4
:10365000D133CE0101960E94985960E876E0CE0100
:1036600001960E94825A69E972E1CE0101960E9498
:10367000A858BC018FE992E10E944A59CE010196F7
:103680000E9498598091C30C9091C40C049721F426
:103690001092C40C1092C30C81E090E0CBC062EC9D
:1036A00079E085EA92E10E94355965EA72E1CE013E
:1036B00001960E947A5A65EC7BE0CE0101960E9449
:1036C00091586FE972E10E94A858BC018FE992E11C
:1036D0000E944A59CE0101960E94985983E090E0D9
:1036E0009093C40C8093C30C64E670E080E090E09B
:1036F0000E9463518091B013882309F4A0C060E256
:1037000073E080E090E00E94635199C084E59EE000
:103710000E94295D64E670E080E090E00E946351C1
:1037200062EE74E089E992E10E940F5969E972E161
:10373000CE0101960E947A5A44E150E060E070E0C8
:10374000CE0101960E94D133CE0101960E94985974
:1037500063ED74E089E992E10E940F5969E972E131
:10376000CE0101960E947A5A44E150E06FEF7FEF5C
:10377000CE0101960E949832CE0101960E9498597E
:103780008CE40E9475696B017C0134E0A32EB12C9E
:10379000A7019601C701B6010E9451B7882309F419
:1037A000EEC2B1E0AB1AB10861F068EC70E080E005
:1037B00090E00E9463518CE40E9475696B017C016A
:1037C000E7CF68EC74E089E992E10E940F5969E95A
:1037D00072E1CE0101960E947A5A4AE050E060E020
:1037E00070E0CE0101960E94D133CE0101960E9475
:1037F000985960E876E0CE0101960E94825A69E904
:1038000072E1CE0101960E94A858BC018FE992E1B5
:103810000E944A59CE0101960E9498598091C30C8A
:103820009091C40C039721F41092C40C1092C30C15
:1038300082E090E0909322028093210255CF87EBA3
:103840009DE00E94B5565CC26DEF74E089E992E19B
:103850000E940F5969E972E1CE0101960E947A5ADD
:103860004AE050E060E070E0CE0101960E94D13362
:10387000CE0101960E949859F0911A02FBAF8091F7
:10388000A00C81110DC00E949B5160939C0C709301
:103890009D0C80939E0C90939F0C81E08093A00CD4
:1038A0008091940C81110DC00E949B516093900CEB
:1038B0007093910C8093920C9093930C81E0809381
:1038C000940C10928F0C10928E0C20908E0C3090D5
:1038D0008F0C88E2281631040CF084C08BAD0E9456
:1038E0001951F101EE0FFF1FE55EF24F91838083C6
:1038F0000E94E06620E030E040EA50E40E9427B3F6
:1039000020E030E040E85AE30E9427B36B017C01DD
:1039100060938A0C70938B0C80938C0C90938D0C1D
:103920004090160250901702609018027090190291
:10393000A30192016091120270911302809114020E
:10394000909115020E9451B49B01AC0160E070E0BF
:1039500080EC90E40E9451B44B015C0120E030E027
:10396000A9010E94C2B220E030E040E650E481119B
:1039700005C0C701B6010E9427B31EC0C701B6012A
:103980000E9427B3A30192010E9452B420E030E0CC
:1039900040E850E40E9451B4A50194010E9418B57A
:1039A00020E030E040EC50E40E9427B320E030E01B
:1039B00040E850E40E9452B46093860C7093870CE8
:1039C0008093880C9093890C64E170E080E090E033
:1039D0000E9463512FEF221A320A30928F0C2092EC
:1039E0008E0C73CFC090860CD090870CE090880C22
:1039F000F090890C20E030E0A901C701B6010E94D7
:103A000007B687FD1EC022E0B701A601CE010196D0
:103A10000E94CC596EE976E0CE0145960E94825A0A
:103A2000BE016F5F7F4FCE0145960E94A858BC0132
:103A30008FE992E10E944A59CE0145960E94985919
:103A400049C16EEE74E08FE992E10E940F5946C1C0
:103A500080912002882309F453C18091B013811111
:103A60002BC080919411811127C0C0900002D0908A
:103A70000102E0900202F090030220E030E04AE709
:103A800054E4C701B6010E9427B30E94B1B54B01AF
:103A90005C0120E030E040EA50E4C701B6010E943A
:103AA00027B320E030E040EA50E40E9452B40E9484
:103AB000B1B5A501940108C021E030E040E050E03C
:103AC0006AE070E080E090E00E941E9B19C1C7018F
:103AD0000E940E7315C1C7010E944F5E11C18091F3
:103AE000C50C882309F40CC16BE475E0CE01019686
:103AF0000E94725ACE0101960E94439AFDC08091A5
:103B0000190D90911A0D892BA1F481E090E090930A
:103B10001A0D8093190D8EED93E09093EF0C809326
:103B2000EE0C0E94D16868EC70E080E090E00E94AA
:103B300063516EE375E0CE0101960E94725A44E62D
:103B400050E06FEF7FEFCE0101960E949832CE01D8
:103B500001960E949859E0E0F0E01995D1C00E94CA
:103B60001EA10E9448320E94AA91CAC09091991148
:103B700081E0892780939911882369F167E375E0D3
:103B80008FE992E10E940F590E949B51609390111E
:103B900070939111809392119093931180919C1145
:103BA00090919D11181619065CF420919E11309188
:103BB0009F112817390724F010929F1110929E111F
:103BC0009091A01180919B1198175CF01092A01118
:103BD0001092A11106C06FE275E08FE992E10E9498
:103BE0000F5980919911809394116FE972E1CE0180
:103BF00001960E947A5A4AE050E068E070E0CE01F7
:103C000001960E94D133CE0101960E94985962E23A
:103C100075E0CE0101960E94725A4AE050E06FEFC3
:103C20007FEFCE0101960E949832CE0101960E944C
:103C3000985964E175E08FE992E10E94B9586CEE01
:103C400079E0CE0101960E94825A6FE972E1CE01BD
:103C500001960E94A858BC018FE992E10E944A593E
:103C6000CE0101960E9498598091B0138093A211C1
:103C70008CE291E00E94F7688091B013882309F4E8
:103C80003FC061EB77E08BEA92E10E94355986EE06
:103C90009FEF9093BE0C8093BD0C32C0F092BE0C8F
:103CA000E092BD0C87EB9DE00E94B55666E075E0A2
:103CB0008FE992E10E940F5962EC79E0CE01019602
:103CC0000E94825A4AE050E060E070E0CE01019626
:103CD0000E94D133CE0101960E9498596FE972E19A
:103CE000CE0101960E947A5A4AE050E06FEF7FEFD2
:103CF000CE0101960E949832CE0101960E949859F9
:103D00008091A3129091A412009799F0419718F412
:103D1000023011050CF56FE972E1CE0101960E94A7
:103D20007A5ACE0101960E94439ACE0101960E94D2
:103D3000985964E670E080E090E00E946351E4C02E
:103D400067E176E08FE992E10E94FB580C94FC0F4A
:103D50000E948A320C9420116FE972E1CE01019623
:103D60000E947A5A4AE050E06FEF7FEFCE01019651
:103D70000E949832CE0101960E949859CCCF21E042
:103D8000B701A601CE0145960E94CC5962E976E0C2
:103D9000CE0101960E94825ABE016B5E7F4FCE011A
:103DA00001960E94A858BC018FE992E10E944A59ED
:103DB000CE0101960E949859CE0145960E949859CD
:103DC0006FE972E1CE0101960E947A5A42E350E017
:103DD0006FEF7FEFCE0101960E949832CE010196DF
:103DE0000E9498596CE976E0CE0101960E94825AB1
:103DF000CE0101960E946C32CE0101960E94985924
:103E00006BE976E08FE992E10E94FB5886E60E941A
:103E100075696B017C0184E0A82EB12CA701960185
:103E2000C701B6010E9451B7882389F0E1E0AE1ABC
:103E3000B10809F434CC68EC70E080E090E00E94B6
:103E4000635186E60E9475696B017C01E7CF21E032
:103E5000B701A601CE0145960E94CC596AE076E0F2
:103E6000CE0101960E94825ABE016B5E7F4FCE0149
:103E700001960E94A858BC0185EA92E10E944A5925
:103E8000CE0101960E949859CE0145960E949859FC
:103E900065EC7BE0CE0101960E94825A65EA72E1F0
:103EA000CE0101960E94A858BC0189E992E10E94C6
:103EB0004A59CE0101960E94985969E972E1CE01F2
:103EC00001960E947A5A4AE050E06FEF7FEFCE01F0
:103ED00001960E941733CE0101960E9498596CE911
:103EE00076E0CE0101960E94825ACE0101960E9490
:103EF0006C32CE0101960E9498596BE976E085EA12
:103F000092E10E94FB58D1CBCB5BDF4F0FB6F89408
:103F1000DEBF0FBECDBFDF91CF911F910F91FF90FC
:103F2000EF90DF90CF90BF90AF909F908F907F9059
:103F30006F905F904F903F902F9008952F923F92F7
:103F40004F925F926F927F928F929F92AF92BF92A9
:103F5000CF92DF92EF92FF920F931F93CF93DF9355
:103F6000CDB7DEB728970FB6F894DEBF0FBECDBF32
:103F7000FC018EE390E19387828780913B1090E073
:103F8000958784878091081190E097878687809134
:103F90003710853009F0B7C38091401090914110DF
:103FA000885891098D35910588F480913B108430B3
:103FB00041F480914210909143108097479708F404
:103FC00007C280913B10843408F0E8C180913B1017
:103FD0008A3108F448C080913E1090913F10843F90
:103FE000914050F4118610868FEF9FEFDC0184839F
:103FF0009583A683B78351C0809140109091411062
:1040000085974B9780F514E4E12E10E1F12E82E0C4
:1040100090E040E050E0BA018C010F5F1F4F20910B
:104020003B1030E0021713076CF49701225031095E
:10403000D9012D913C91275031092730310508F4E1
:104040000AC2C801019795958795918780870C973B
:104050001CF41186108607C04483558366837783DA
:1040600084E090E01CC180913B108A3108F448C084
:1040700080913E1090913F108032934008F4B2CF6F
:104080008091401090914110C697869708F403C222
:1040900037C044835583668377838BE090E0FFC00D
:1040A000D7012D913C91255231092B31310508F072
:1040B00004C2440F551F661F771F41600296B4E08B
:1040C000EB0EF11C8C010F5F1F4F20913B1030E075
:1040D0000217130764F4970122503109D9012D9179
:1040E0003C912C5031092B303105D0F2C801019799
:1040F00095958795918780870C975CF61186108639
:1041000080913B10823208F44CC080914010909115
:1041100041100697079708F044C044E4C42E40E1DC
:10412000D42E82E090E040E050E0BA018C010F5FB5
:104130001F4F20913B1030E0021713070CF5D601FA
:104140001297ED90FC9011979D01BEE1EB1AF108DA
:10415000A7E1EA16F10408F0BEC1440F551F661F1F
:10416000771F4160D6012D913C91B4E0CB0ED11C5C
:10417000235031092530310510F40296D7CFC801FC
:104180000197959587959187808740971CF41186B4
:10419000108607C044835583668377838CE090E064
:1041A0007EC07F011C821B8281E090E09A8389831C
:1041B00080913B108D3008F475C029E733E0AE01E3
:1041C0004D5F5F4FBE016F5F7F4FCF010E946385E0
:1041D000892B09F067C029E733E0AE014D5F5F4FDF
:1041E000BE016F5F7F4FC7010E946385019709F091
:1041F00059C029E733E0AE014D5F5F4FBE016F5FED
:104200007F4FC7010E946385892B09F04BC0812C29
:10421000912C540100E010E080913B1090E0298146
:104220003A81281739077CF529E733E0AE014D5F65
:104230005F4FBE016F5F7F4FC7010E9463856C01B6
:1042400029E733E0AE014D5F5F4FBE016F5F7F4FE7
:10425000C7010E946385E1E0CE16D10449F4892BA1
:1042600009F5880C991CAA1CBB1C689480F808C02E
:10427000CD28C1F40197B1F4880C991CAA1CBB1C71
:104280000F5F1F4FC9CFD70119961C930E93189734
:10429000F70184829582A682B78281E090E09183C3
:1042A000808329C21C821B8281E090E09A838983EB
:1042B000D7011C968D919C911D97181619060CF02C
:1042C00061C01A96ED91FC911B9782E090E09A8371
:1042D00089838281938189974E9708F053C083E048
:1042E00090E09A838983848195810B970A9708F0DF
:1042F00049C02CEB31E0AE014D5F5F4FBE016F5FF7
:104300007F4FC7010E946385892BE1F52CEB31E0DB
:10431000AE014D5F5F4FBE016F5F7F4FC7010E94CF
:104320006385019779F5412C512C320100E010E0B2
:1043300029813A81D7011C968D919C911D97281750
:1043400039070CF010C12CEB31E0AE014D5F5F4F2F
:10435000BE016F5F7F4FC7010E9463855C01033020
:10436000110509F0C6C02CEB31E0AE014D5F5F4F87
:10437000BE016F5F7F4FC7010E946385A816B90613
:1043800009F4B7C0D7011A96ED91FC911B97828171
:104390009381C697869708F4F2C03EC1809142107F
:1043A00090914310825491098E9708F00FCE20E02F
:1043B00030E0C12CD12C7601A9014C5B5F4EDA01B3
:1043C0004D915C91495051094930510598F0FECD0D
:1043D00080914410909145100997099708F0F1CD0C
:1043E000118610868FEF9FEFDC0184839583A6836F
:1043F000B7838CC1B9016A5B7F4EDB014D915C9143
:104400004751510942315105C0F4D701C601880F07
:10441000991FAA1FBB1F6C017D016894C0F82C5F17
:104420003F4F2038310541F620E230E031872087C8
:10443000C482D582E682F78269C1DB014D915C912D
:10444000465051094730510508F0C0CDCC0CDD1C59
:10445000EE1CFF1CE4CFD7012D913C912351310973
:104460002F30310550F4440F551F661F771F4160F0
:104470000296B4E0EB0EF11CCFCDD7012D913C910B
:104480002A5031092930310508F0EDCD440F551F70
:10449000661F771FEDCF8091421090914310C69711
:1044A000869708F02DCE86E4E82E80E1F82E83E092
:1044B00090E040E050E0BA0105CED7012D913C914B
:1044C0002C5031092A30310508F01ACE440F551FFF
:1044D000661F771FF3CDD9012D913C912C503109E6
:1044E0002B30310508F05DCE440F551F661F771F36
:1044F00039CE2CEB31E0AE014D5F5F4FBE016F5FF7
:104500007F4FC7010E9463856C010330110579F468
:104510002CEB31E0AE014D5F5F4FBE016F5F7F4F0F
:10452000C7010E946385C816D90609F02BCFA114D4
:10453000B10459F4CA94CD2809F024CF440C551C79
:10454000661C771C689440F80BC0AA94AB2809F04D
:1045500019CFCD2809F016CF440C551C661C771CCA
:104560000F5F1F4FE5CE19961C930E931897F70116
:10457000448255826682778282E090E090CE848188
:1045800095814B97459708F047C0DF0116966F015C
:1045900026ECC20ED11C20E030E040E050E060E0AC
:1045A00070E080E090E00D911C9111970950110985
:1045B0000830110588F512960D911C911397015141
:1045C00011090D301105D8F401E00E94A8B721604F
:1045D0001496AC15BD0539F7F7012483358346835E
:1045E000578300E20E94C3B72283338385E090E0C3
:1045F0009183808380E390E0918780877CC01296CE
:104600000D911C911397045011090530110520F4E8
:1046100001E00E94A8B7DCCF80913B10893340F0C5
:1046200082819381895791098335910508F47CC172
:1046300080913B10823209F46CC08281938189574A
:1046400091098335910508F4E6C1828193818C54E8
:104650009109C59708F064C080913B10843031F413
:10466000848195818097479708F434C280913B10EC
:10467000843408F455C08481958189549109C39785
:1046800008F04EC09F012A5F3F4FAF014A575F4F6E
:10469000812C912C5401D9016D917C916950710943
:1046A00069307105E8F5D90112966D917C911397E7
:1046B000665171096131710508F022C2D501C4014A
:1046C000880F991FAA1FBB1F4C015D01689480F8D9
:1046D0002C5F3F4F24173507F1F620E230E0F70159
:1046E00031872087D70184829582A682B78287E0AE
:1046F00090E08D939C9381E090E0BFC282E0809334
:10470000371010923B1080E090E0B7C283E090E059
:10471000C6CD828193810A97099708F460C18DCF35
:1047200080913B10863460F1828193810C970B97C6
:1047300008F4F6C125C0D90112966D917C911397AA
:104740006E5171096731710508F01EC2D501C401AF
:10475000880F991FAA1FBB1F4C015D01689480F848
:104760004E5F5F4F2C5F3F4F4534510509F4F3C155
:10477000D9016D917C916C5071096B307105D8F243
:1047800080913B10883578F1828193818558910919
:104790008B35910508F408C226C0BC016F5F7F4FBE
:1047A000D8012D913C91275031092730310508F06F
:1047B0000AC2440F551F416002960C5F1F4F2091A3
:1047C0003B1030E024503109821793070CF004C2EB
:1047D000980122503109D9012D913C91295031097C
:1047E00028303105D0F280913B108032E1F4828193
:1047F000938106970697B8F4848195810997099764
:1048000090F49F012A5F3F4FAF01425C5F4F812CC4
:10481000912C5401D9016D917C91665071096630DB
:10482000710508F4F3C1D7011C962D903C901D979B
:10483000B6E02B1631040CF461CF8F010A5F1F4FD5
:1048400073E0C72ED12CE5EC8E2EEDE99E2EECE127
:10485000AE2EE1E8BE2EF801608171813497608050
:10486000718080E090E00E94C6B26D837E838F836A
:104870009887B30180E090E00E94C6B22B013C0112
:104880002DEC3CEC4CE45FE30E9427B39B01AC01B0
:104890006D817E818F8198850E94C2B287FD19C08B
:1048A0002DEC3CEC4CE45FE36D817E818F8198853B
:1048B0000E9427B39B01AC01C301B2010E94C2B2A6
:1048C000E82F880FFF0BEE27FF0FEE1FFF27319613
:1048D00002C0E0E0F0E0A501940163E971E080E04E
:1048E00091E00E946AB74F01FF0FAA08BB08862615
:1048F0009726A826B926FFEFCF1ADF0A0E5F1F4FB3
:10490000C214D30409F0A7CFD70114968D929D92BB
:10491000AD92BC92179780E290E019969C938E938B
:1049200018978FEF9FEFE5CE84819581CA9789977D
:1049300008F07ECE9F012A5F3F4F812C912C5401BD
:1049400043E050E0D9016D917C916A507109693062
:10495000710508F06DCED90112966D917C91139777
:10496000665171096131710550F5D501C401880F97
:10497000991FAA1FBB1F4C015D01689480F84E5F10
:104980005F4F2C5F3F4F4B335105E1F69F012A5893
:104990003F4FD9012D913C912A50310929303105E1
:1049A00008F046CE2CE130E0F70131872087D701AF
:1049B00084829582A682B7828AE090E09ACED9015D
:1049C00012966D917C91139766507109673071054D
:1049D00008F02ECE880C991CAA1CBB1CD0CF2091AD
:1049E0003B10CF01820F911D820F911DDC011297A8
:1049F0008D919C910A97099708F01FCEF7011186B7
:104A000010868FEF9FEFDC0184839583A683B783A5
:104A100086E090E044CC80913B10813208F415CEC2
:104A200084819581CA97899708F00FCE9F012A5FEC
:104A30003F4F812C912C540143E050E0D9016D91FE
:104A40007C916A5071096930710508F0FECDD90179
:104A500012966D917C9113976651710961317105C0
:104A600070F112966D917C911397665071096730C1
:104A7000710508F0EACD880C991CAA1CBB1C4E5F7E
:104A80005F4F2C5F3F4F43325105C1F69F012A5BB8
:104A90003F4FD9012D913C912A50310929303105E0
:104AA00008F0D3CD20E130E0F70131872087D7012E
:104AB00084829582A682B78286E090E01ACED501E4
:104AC000C401880F991FAA1FBB1F4C015D01689488
:104AD00080F8D5CF868197810997099708F0C6CDD0
:104AE000D70119961C921E9218978FEF9FEFDC0149
:104AF000F70184839583A683B78387E090E0CFCBCB
:104B0000D90112966D917C911397665071096730A7
:104B1000710508F005CE880C991CAA1CBB1CD8CDC9
:104B2000848195810997099708F02ACE868197811B
:104B30008C974F9708F024CE8085918589974D9763
:104B400008F01ECE9F01265F3F4F812C912C54010F
:104B500045E050E00DCE9F0126573F4FD9012D91E2
:104B60003C912C5031092B30310508F009CE20E260
:104B700030E0F70131872087D70184829582A682B1
:104B8000B78288E090E0B5CDD90112966D917C9105
:104B90001397695071096930710508F0F1CD880CDF
:104BA000991CAA1CBB1CDCCD84819581825491097F
:104BB0008E9708F018CE8F01045C1F4F8DE190E0B6
:104BC00040E050E0FCCDD8012D913C9128513109B5
:104BD00022313105C0F0CB01019795958795D7011A
:104BE00019969C938E9318978A970CF4FCCD052EFA
:104BF000000C660B770BF70144835583668377833C
:104C000089E090E04CCB440F551FD6CDD9011296C8
:104C10006D917C9113976951710963317105E8F4C5
:104C2000D501C401880F991FAA1FBB1F4C015D014C
:104C3000689480F82C5F3F4F2417350709F0EACDC0
:104C40002EE030E0F70131872087D70184829582FA
:104C5000A682B7828FE090E04CCDD90112966D917B
:104C60007C911397695071096930710508F0DBCDAB
:104C7000880C991CAA1CBB1CDDCF28960FB6F89493
:104C8000DEBF0FBECDBFDF91CF911F910F91FF907F
:104C9000EF90DF90CF90BF90AF909F908F907F90DC
:104CA0006F905F904F903F902F9008955F926F921A
:104CB0007F928F929F92AF92BF92CF92DF92EF92AC
:104CC000FF920F931F93CF93DF93CDB7DEB7E49797
:104CD0000FB6F894DEBF0FBECDBF62EA76E0CE011C
:104CE0000B960E94825ABE01655F7F4F87EB92E16F
:104CF0000E947658811116C068EA76E0CE010196CE
:104D00000E94825ABE016F5F7F4F87EB92E10E9443
:104D1000765811E0811101C010E0CE0101960E9489
:104D2000985901C011E0CE010B960E9498591123A9
:104D300009F476C026E030E045E050E067EB72E130
:104D4000CE0101960E94965ABE016F5F7F4F89E99E
:104D500092E10E945F59CE0101960E94985989E91B
:104D600092E10E9491576B017C0162ED7AE0CE01E5
:104D700001960E94825ABE016F5F7F4F87EB92E1DE
:104D80000E94FB57AC014F5F5F4F67EB72E1CE01B2
:104D90000B960E943B3EBE01655F7F4F89E992E121
:104DA0000E945F59CE010B960E949859CE01019640
:104DB0000E94985989E992E10E949157DB01E3E250
:104DC000F2E041E050E020912302309124022417C8
:104DD00035075CF0228133812A173B0711F41382D7
:104DE00012824F5F5F4F3296EECF9601220F331F34
:104DF000F901ED5DFD4F7183608382E090E00E94D8
:104E0000039367EB72E1CE0101960E947A5ACE01BC
:104E100001960E947238CE0101960E94985949C0AD
:104E20006EEA76E0CE010B960E94825ABE01655F63
:104E30007F4F87EB92E10E947658811116C064EB98
:104E400076E0CE0101960E94825ABE016F5F7F4FCD
:104E500087EB92E10E94765811E0811101C010E0C9
:104E6000CE0101960E94985901C011E0CE010B9627
:104E70000E949859112349F1E3E2F2E081E090E0C9
:104E800020912302309124022817390774F08630CC
:104E900091051CF49383828305C09C012E5F3F4FD4
:104EA0003383228301963296EBCF82E090E00E941A
:104EB00003931092EF0C1092EE0C80E090E00E94B1
:104EC0002169109209020C941D326AEB76E0CE0142
:104ED0000B960E94825ABE01655F7F4F87EB92E17D
:104EE0000E947658811116C061EC76E0CE010196E1
:104EF0000E94825ABE016F5F7F4F87EB92E10E9452
:104F0000765811E0811101C010E0CE0101960E9497
:104F1000985901C011E0CE010B960E9498591123B7
:104F2000F9F08091190D90911A0D892BA1F481E06F
:104F300090E090931A0D8093190D8EED93E090936D
:104F4000EF0C8093EE0C0E94D16868EC70E080E07A
:104F500090E00E946351E0E0F0E019950C941D325E
:104F600068EC76E0CE010B960E94825ABE01655F26
:104F70007F4F87EB92E10E947658811116C060ED59
:104F800076E0CE0101960E94825ABE016F5F7F4F8C
:104F900087EB92E10E94765811E0811101C010E088
:104FA000CE0101960E94985901C011E0CE010B96E6
:104FB0000E9498591123B1F068ED76E0CE01019678
:104FC0000E94825A68E873E1CE0101960E94A858B7
:104FD000BC018FE992E10E944A59CE0101960E94DC
:104FE000985938C062EE76E0CE010B960E94825A44
:104FF000BE01655F7F4F87EB92E10E947658811179
:1050000016C069EE76E0CE0101960E94825ABE017A
:105010006F5F7F4F87EB92E10E94765811E081111C
:1050200001C010E0CE0101960E94985901C011E024
:10503000CE010B960E9498591123A9F062EC75E0FD
:105040008FE992E10E940F596EE873E18FE992E1D6
:105050000E9409596CEE79E0CE0101960E94825AB5
:105060006FE972E19EC760EF76E0CE010B960E9479
:10507000825ABE01655F7F4F87EB92E10E947658AE
:10508000811116C066EF76E0CE0101960E94825A29
:10509000BE016F5F7F4F87EB92E10E94765811E06F
:1050A000811101C010E0CE0101960E94985901C003
:1050B00011E0CE010B960E949859112311F16FE96E
:1050C00075E08FE992E10E940F596FE972E1CE011C
:1050D00001960E947A5ACE0101960E94439ACE010F
:1050E00001960E9498590E948B8E1092090262EFDD
:1050F00076E087EB92E10E9435590E94826A0C9417
:105100001D326CEF76E0CE010B960E94825ABE01F2
:10511000655F7F4F87EB92E10E947658811116C040
:1051200063E077E0CE0101960E94825ABE016F5F74
:105130007F4F87EB92E10E94765811E0811101C008
:1051400010E0CE0101960E94985901C011E0CE01F5
:105150000B960E949859112309F48CC062ED7AE0F5
:10516000CE0101960E94825ABE016F5F7F4F87EB8E
:1051700092E10E94FB57AC014F5F5F4F67EB72E11A
:10518000CE010B960E943B3EBE01655F7F4F89E9D1
:1051900092E10E945F59CE010B960E949859CE0170
:1051A00001960E94985989E992E10E9491578B01DA
:1051B00062E975E08FE992E10E940F59809199119F
:1051C000882331F066E875E08FE992E10E940F597B
:1051D0000115110511F40C940832CE0101960E94BC
:1051E0007762CE0101960E94439ACE0101960E94F9
:1051F0009859023011050CF464CE63E27EE0CE01D2
:105200000B960E94725ABE01655F7F4FCE010196D8
:105210000E947A5ACE0101960E94439ACE010196CD
:105220000E949859E12CF12C80919B11082E000CC2
:10523000990BE816F9068CF4B701CE0101960E948D
:105240006261CE0101960E94439ACE0101960E94AE
:105250009859FFEFEF1AFF0AE7CFCE010B960E9495
:1052600098590230110509F42CCE8CE291E00E948D
:105270004B6927CE6AE077E0CE010B960E94825AF6
:10528000BE01655F7F4F87EB92E10E9476588111E6
:1052900016C061E177E0CE0101960E94825ABE01FC
:1052A0006F5F7F4F87EB92E10E94765811E081118A
:1052B00001C010E0CE0101960E94985901C011E092
:1052C000CE010B960E949859112309F48CC367EB09
:1052D00072E1CE018F960E947A5A62ED7AE0CE0199
:1052E00001960E94825ABE016F5F7F4FCE018F965A
:1052F0000E94FB57AC014F5F5F4FBE01615D7F4F66
:10530000CE0189960E943B3ECE0101960E9498599B
:10531000BE01615D7F4FCE0101960E947A5ACE0197
:1053200001960E947238CE0101960E9498596EE053
:1053300077E0CE0101960E94825ABE016F5F7F4FD7
:10534000CE0189960E944B588C01CE0101960E9495
:10535000985962EC79E0CE0183960E94825A62EC01
:1053600079E0CE014D960E94825A1016110684F5FE
:10537000A8014F5F5F4F8DA59EA54817590790F470
:10538000BE01675D7F4FCE0101960E943B3EBE018C
:105390006F5F7F4FCE0183960E945F59CE010196C9
:1053A0000E949859980140E050E0BE01675D7F4F30
:1053B000CE0101960E94965ABE016F5F7F4FCE01CB
:1053C0004D960E945F59CE0101960E9498590DC0DA
:1053D00062EC79E0CE0183960E943559BE01675D8B
:1053E0007F4FCE014D960E944A5989A19AA1892BDF
:1053F00009F4EAC2CE014D960E9491577B0121E04B
:10540000E21AF10848E1E416F1041CF027E1E22E6B
:10541000F12CF7FE03C0EE24EA94FE2C4AE0B7011B
:10542000CE010B960E94275A60E177E0CE014196AB
:105430000E94825ABE01655F7F4FCE0141960E9455
:10544000A858BC01CE0101960E947A5ACE0101965D
:105450000E947238CE0101960E949859CE01419661
:105460000E949859CE010B960E949859BE016D5D1D
:105470007F4FCE0189960E944A596EE077E0CE01B7
:1054800001960E94825ABE016F5F7F4FCE018996BE
:105490000E944B588C01CE0101960E94985962ECF3
:1054A00079E0CE0183960E94355962EC79E0CE0115
:1054B0004D960E943559101611060CF04DC0A801EA
:1054C0004F5F5F4F8DA59EA54817590790F4BE0109
:1054D000675D7F4FCE0101960E943B3EBE016F5F2C
:1054E0007F4FCE0183960E945F59CE0101960E94A4
:1054F0009859980140E050E0BE01675D7F4FCE01B2
:1055000001960E94965ABE016F5F7F4FCE014D9665
:105510000E945F59CE0101960E9498598E010F5F3B
:105520001F4FC12CD12CA7014F5F5F4F8AE0849F92
:105530009001859F300D1124F901E756FE4E5F0161
:105540008E9D90018F9D300D1124A90149555E4E0D
:105550004A018AE2582EC0C062EC79E0CE018396FF
:105560000E943559BE01675D7F4FCE014D960E9466
:105570004A59D4CFCE014D96C114D10409F0B9C017
:105580005FEFE516F50609F4B4C00E949C57A1141C
:10559000B10439F044E050E0B501CE014D960E94CF
:1055A00036A0B501CE0141960E94825A65E177E0AE
:1055B000CE0147960E94825ABE016F5E7F4FCE0198
:1055C00047960E94A858BC01CE010B960E947A5AB9
:1055D000CE010B960E947238CE010B960E9498590C
:1055E000CE0147960E949859CE0141960E94985943
:1055F00089A19AA1029708F475C061E070E0CE011C
:105600004D960E946558082E000C990B8033910529
:105610000CF44C96E52DE81B8E2FF4018083FFEFF0
:10562000CF1ADF0ABE016D5D7F4FCE0189960E94C1
:105630004A596EE077E0CE010B960E94825ABE0175
:10564000655F7F4FCE0189960E944B583C01CE0189
:105650000B960E94985962EC79E0CE0183960E94E5
:10566000355962EC79E0CE014D960E9435591614F9
:1056700017040CF044C0A3014F5F5F4F8DA59EA59A
:105680004817590790F4BE01675D7F4FCE010B9616
:105690000E943B3EBE01655F7F4FCE0183960E9414
:1056A0005F59CE010B960E949859930140E050E05B
:1056B000BE01675D7F4FCE010B960E94965ABE01D8
:1056C000655F7F4FCE014D960E945F59CE010B96CC
:1056D0000E9498590E5F1F4F89A19AA1892B09F04A
:1056E00049CF1BC0CE014D960E949157F4016083B3
:1056F00096CF0E949157F8017183608390CF62EC3E
:1057000079E0CE0183960E943559BE01675D7F4FD7
:10571000CE014D960E944A59DDCF2FEFE216F206D8
:1057200009F07EC06EE077E0CE010B960E94825AAF
:10573000BE01655F7F4FCE0183960E944B588C015E
:10574000CE010B960E94985917FF3EC109811A811C
:105750001016110634F4093111052CF008E110E09F
:1057600002C001E010E000939B114AE0B801CE01B5
:1057700041960E94275A63E277E0CE0147960E9445
:10578000825ABE016F5E7F4FCE0147960E94A85895
:10579000BC01CE010B960E947A5ACE010B960E9454
:1057A0007238CE010B960E949859CE0147960E94FE
:1057B0009859CE0141960E949859C114D10459F1CB
:1057C0008B819C8197FF02C080E090E090939D11B7
:1057D00080939C1141E0C416D104E9F08D819E8133
:1057E000181619062CF48017910724F48C0102C0B6
:1057F00001E010E001500093A01152E0C516D10461
:1058000051F08F8198851816190614F081E090E008
:1058100081508093A1118CE291E00E94F768D4C07E
:1058200080919A11082E000C990BE816F9060CF0DD
:1058300084C04AE0B601CE0141960E94275A6DE22B
:1058400077E0CE0147960E94825ABE016F5E7F4F7D
:10585000CE0147960E94A858BC01CE010B960E942B
:105860007A5ACE010B960E947238CE010B960E9496
:105870009859CE0147960E949859CE0141960E94B0
:1058800098598AE08E9DF0018F9DF00D1124E75606
:10589000FE4E81E0878783E090E0918B808B938B35
:1058A000828BC114D10409F48FC08B819C81803814
:1058B000910514F08FE790E080382FEF920714F4F1
:1058C00080E89FEF878741E0C416D10409F47CC0CB
:1058D0008AE08E9DF0018F9DF00D1124E756FE4E5B
:1058E0008D819E8197FF02C080E090E0918B808B3C
:1058F00052E0C516D10409F467C08AE08E9DF0011C
:105900008F9DF00D1124E756FE4E8F81988597FFED
:1059100002C080E090E0938B828B80919B11082ED7
:10592000000C990BE816F9061CF0E394E0929B1129
:105930008CE291E00E944B6947C0BE016D5D7F4FD4
:10594000CE0147960E947A5A60919A11062E000C59
:10595000770B4AE0CE010B960E94275A65E377E069
:10596000CE0141960E94825ABE01695E7F4FCE01F0
:1059700041960E94A85866E477E00E949158BE01C3
:10598000655F7F4F0E94A858BC01CE0147960E94D8
:105990004A59CE0141960E949859CE010B960E9419
:1059A0009859BE01695E7F4FCE010B960E947A5ACC
:1059B000CE010B960E94439ACE010B960E949859F5
:1059C000CE0147960E949859CE014D960E94985953
:1059D000CE0183960E949859CE0189960E949859CB
:1059E000CE018F964CC26AE477E0CE010B960E94FE
:1059F000825ABE01655F7F4F87EB92E10E94765825
:105A0000811116C06FE477E0CE0101960E94825AA0
:105A1000BE016F5F7F4F87EB92E10E94765811E0E5
:105A2000811101C010E0CE0101960E94985901C079
:105A300011E0CE010B960E9498591123C9F162ED35
:105A40007AE0CE0101960E94825ABE016F5F7F4FBD
:105A500087EB92E10E94FB57AC014F5F5F4F67EB12
:105A600072E1CE010B960E943B3EBE01655F7F4F07
:105A700089E992E10E945F59CE010B960E949859E4
:105A8000CE0101960E94985989E992E10E949157AE
:105A90006115710521F481E08093080206C0613030
:105AA000710509F00ECA109208020E94BA9109CA43
:105AB00064E577E0CE010B960E94825ABE01655FD5
:105AC0007F4F87EB92E10E947658811116C068E5FE
:105AD00077E0CE0101960E94825ABE016F5F7F4F30
:105AE00087EB92E10E94765811E0811101C010E02D
:105AF000CE0101960E94985901C011E0CE010B968B
:105B00000E949859112309F424C143E050E067EB47
:105B100072E1CE0101960E943B3EBE016F5F7F4F56
:105B200089E992E10E945F59CE0101960E9498593D
:105B300069E972E1CE0101960E947A5ACE0101967E
:105B40000E947238CE0101960E9498591092EF0C73
:105B50001092EE0C69E972E184E993E10E944A59DE
:105B600069E972E18EE893E10E944A5986E291E187
:105B7000009739F048E050E0BC0184E993E10E94CD
:105B800036A084E891E1009739F04CE050E0BC0188
:105B90008EE893E10E9436A08091EE0C9091EF0C7C
:105BA0000E9421696CE577E0CE0101960E94825A3D
:105BB0006EE873E1CE0101960E94A858BC01CE01A7
:105BC00041960E947A5ACE0101960E94985980917E
:105BD000801190918111892B39F4BE016F5E7F4F46
:105BE00087EB9DE00E94E15A809180119091811194
:105BF000029709F09BC06EE873E1CE0147960E94C0
:105C00007A5A64E677E0CE0101960E94825ACE016C
:105C100001960E948AADCE0101960E94985964EFC8
:105C200071E080E090E00E94635167E677E0CE018A
:105C300001960E94825ACE0101960E948AADCE0141
:105C400001960E94985964EF71E080E090E00E9414
:105C5000635160E777E0CE0101960E94825ACE013F
:105C600001960E948AADCE0101960E94985964EF78
:105C700071E080E090E00E94635169E777E0CE0137
:105C800001960E94825ACE0101960E948AADCE01F1
:105C900001960E94985964EF71E080E090E00E94C4
:105CA000635167E877E0CE0101960E94825ACE01E7
:105CB00001960E948AADCE0101960E94985964EF28
:105CC00071E080E090E00E9463516CE577E0CE01E6
:105CD00001960E94825ABE01695E7F4FCE010196F5
:105CE0000E94A858BC01CE010B960E947A5ACE01A0
:105CF00001960E949859CE010B960E949C57BE01B6
:105D0000655F7F4FCE0101960E947A5ACE010196BF
:105D10000E948AADCE0101960E949859CE010B9641
:105D20000E949859CE0147960E94985966E271E107
:105D3000CE0101960E94825ACE0101960E947238CD
:105D4000CE0101960E94985910920902CE01419607
:105D500096C065E977E0CE010B960E94825ABE019B
:105D6000655F7F4F87EB92E10E947658811116C0E4
:105D70006AE977E0CE0101960E94825ABE016F5F08
:105D80007F4F87EB92E10E94765811E0811101C0AC
:105D900010E0CE0101960E94985901C011E0CE0199
:105DA0000B960E949859112309F46CC044E050E00E
:105DB00067EB72E1CE0101960E943B3EBE016F5F30
:105DC0007F4F89E992E10E945F59CE0101960E94BE
:105DD00098596FE977E0CE010B960E94825A69E9E3
:105DE00072E1CE010B960E94A858BC01CE0101962B
:105DF0000E947A5ACE010B960E9498598091801188
:105E000090918111892B39F4BE016F5F7F4F87EB31
:105E10009DE00E94E15A68EB7BE080E090E00E9408
:105E200063518091801190918111029779F4BE01A4
:105E30006F5F7F4FCE010B960E947A5ACE010B9670
:105E40000E948AADCE010B960E94985968EB7BE0C8
:105E500080E090E00E946351BE016F5F7F4FCE01F2
:105E60000B960E947A5ACE010B960E947238CE0190
:105E70000B960E94985910920902CE0101960E9439
:105E80009859DBC266EA77E0CE010B960E94825AEF
:105E9000BE01655F7F4F87EB92E10E9476588111CA
:105EA00016C06AEA77E0CE0101960E94825ABE01CE
:105EB0006F5F7F4F87EB92E10E94765811E081116E
:105EC00001C010E0CE0101960E94985901C011E076
:105ED000CE010B960E949859112309F474C067EB08
:105EE00072E189E992E10E944A5981E080930902B6
:105EF00067EB72E1CE0101960E947A5ACE010196BB
:105F00000E947238CE0101960E94985980918011AA
:105F100090918111029709F169E972E187EB9DE0A7
:105F20000E94E15A68EB7BE080E090E00E946351C0
:105F3000CE0101960E94B088BE016F5F7F4F87EB54
:105F400092E10E945F59CE0101960E94985960ED3E
:105F500077E080E090E00E94635180918011909101
:105F60008111029771F469E972E1CE0101960E94F4
:105F70007A5ACE0101960E948AADCE0101960E9406
:105F800098598091BB129091BC12892B11F40C94FA
:105F900061276CEE79E0CE0101960E94825A67EB90
:105FA00072E1CE0101960E94A858BC01CE010B9669
:105FB0000E947A5ACE010B960E94439ACE010B960C
:105FC0000E9498592FC26EEA77E0CE010B960E948C
:105FD000825ABE01655F7F4F87EB92E10E9476583F
:105FE000811116C064EB77E0CE0101960E94825ABF
:105FF000BE016F5F7F4F87EB92E10E94765811E000
:10600000811101C010E0CE0101960E94985901C093
:1060100011E0CE010B960E949859112309F457C044
:106020008091801190918111019711F00C9461275A
:10603000CE0101960E94C2638D819E81009709F472
:10604000F1C1E981FA812081222309F4EBC107978C
:1060500008F4E8C16DE775E0CE010B960E94725A14
:1060600048EC50E06FEF7FEFCE010B96E0D2CE010F
:106070000B960E949859BE016F5F7F4FCE010B9621
:106080000E947A5A40ED57E06FEF7FEFCE010B96FA
:106090004FD2CE010B960E9498596AEB77E0CE0161
:1060A0000B960E94825A67EB72E1CE010B960E941A
:1060B000A858BC01CE0141960E947A5ACE01419661
:1060C0000E94439ACE0141960E94985977CF68EC7E
:1060D00077E0CE010B960E94825ABE01655F7F4F2A
:1060E00087EB92E10E947658811116C06DEC77E043
:1060F000CE0101960E94825ABE016F5F7F4F87EBEF
:1061000092E10E94765811E0811101C010E0CE01A9
:1061100001960E94985901C011E0CE010B960E9491
:106120009859112359F125E030E044E050E067EB45
:1061300072E1CE0101960E94965ABE016F5F7F4FB9
:1061400089E992E10E945F59CE0101960E94985917
:1061500067EB72E1CE0101960E947A5ACE01019658
:10616000C1D7CE0101960E94985989E992E10E9417
:106170009157CB010E94745D0C94612762ED77E02A
:10618000CE010B960E94825ABE01655F7F4F87EB5E
:1061900092E10E947658811116C069ED77E0CE0138
:1061A00001960E94825ABE016F5F7F4F87EB92E19A
:1061B0000E94765811E0811101C010E0CE010196D5
:1061C0000E94985901C011E0CE010B960E94985987
:1061D000112359F127E030E046E050E067EB72E12F
:1061E000CE0101960E94965ABE016F5F7F4F89E9EA
:1061F00092E10E945F59CE0101960E94985989E967
:1062000092E10E949157672B19F41092C50C03C0BC
:1062100081E08093C50C67EB72E1CE0101960E948C
:106220007A5ACE0101965ED7FDC060EE77E0CE01CE
:1062300001960E94825ABE016F5F7F4F87EB92E109
:106240000E947658182FCE0101960E94985911236A
:1062500009F476C08091BB129091BC12079708F4A4
:10626000ECC046E050E067EB72E1CE0101960E947F
:106270003B3EBE016F5F7F4F89E992E10E945F590B
:10628000CE0101960E94985989E992E10E948657B1
:1062900060930402709305028093060290930702B4
:1062A0006DE675E08FE992E10E940F59409104027A
:1062B00050910502609106027091070221E0CE0123
:1062C00001960E94CC59BE016F5F7F4FCE010B96A5
:1062D0000E947A5A62EE75E0CE010B960E949158A8
:1062E000BC018FE992E10E940959CE010B960E94F0
:1062F0009859CE0101960E9498596FE972E1CE013A
:1063000001960E947A5ACE0101960E94439ACE01CC
:1063100001960E9498590E949B5128EE33E040E07C
:1063200050E00E9420B4CA01B9010E94C6B2609335
:10633000A90C7093AA0C8093AB0C9093AC0C7DC00D
:1063400067EE77E0CE0101960E94825ABE016F5F30
:106350007F4F87EB92E10E947658182FCE0101966D
:106360000E949859112309F463C08091BB12909147
:10637000BC12079708F461C046E050E067EB72E199
:10638000CE0101960E943B3EBE016F5F7F4F89E9BF
:1063900092E10E945F59CE0101960E94985989E9C5
:1063A00092E10E94865760930002709301028093ED
:1063B0000202909303026DE575E08FE992E10E947D
:1063C0000F594091000250910102609102027091B8
:1063D000030221E0CE0101960E94CC59BE016F5FFD
:1063E0007F4FCE010B960E947A5A62EE75E0CE0185
:1063F0000B960E949158BC018FE992E10E940959C5
:10640000CE010B960E949859CE0101960E94985990
:106410006FE972E1CE0101960E947A5ACE0101968F
:106420000E94439ACE0101960E9498590C946127CC
:106430000E94473E182F882399F0109109021123DA
:1064400071F067EB72E1CE0101960E947A5ACE019B
:10645000019648D6CE0101960E94985901C011E0DC
:10646000812FE4960FB6F894DEBF0FBECDBFDF914B
:10647000CF911F910F91FF90EF90DF90CF90BF9041
:10648000AF909F908F907F906F905F900895089548
:10649000809108028823F9F080910C058823D9F0B7
:1064A00081E00E94A0658BE39FE10197F1F760E036
:1064B00080E00E94B16560EE76E08AE993E10E9497
:1064C000EF5A61E080E00E94B16560ED76E08AE914
:1064D00093E10C94EF5A0895CF93DF932091080233
:1064E0002223A9F020910C05222389F0EC016FED05
:1064F0008AE993E10E94DA5A8C819D81892B39F0D7
:10650000BE018AE993E1DF91CF910C94E15ADF91CA
:10651000CF91089580910802882349F080910C055D
:10652000882329F060E08AE993E10C94935508955B
:106530008F929F92AF92BF92EF92FF920F931F9311
:10654000CF93DF937C01EB018A01809108028823BD
:1065500009F462C080910C05882309F45DC077FFBF
:1065600018C0C095D09561E08C2F0E94B165B7012D
:106570008AE993E10E94E15A6FEB76E08AE993E1C0
:106580000E94EF5AF701848161E08C0F0E94B1658F
:1065900033C00E949B5180907C0C90907D0CA09009
:1065A0007E0CB0907F0C24E6820E911CA11CB11CC5
:1065B00086169706A806B90678F561E08C2F0E942A
:1065C000B165B7018AE993E10E94E15A6EEA76E08B
:1065D0008AE993E10E94EF5AF701848161E08C0F10
:1065E0000E94B1650E949B5160937C0C70937D0C5E
:1065F00080937E0C90937F0CB801110F880B990B40
:10660000DF91CF911F910F91FF90EF90BF90AF90CE
:106610009F908F900C946351DF91CF911F910F91B8
:10662000FF90EF90BF90AF909F908F900895AF92A2
:10663000BF92CF92DF92EF92FF920F931F93CF936F
:10664000DF93CDB7DEB762970FB6F894DEBF0FBE0B
:10665000CDBF20910802222309F492C020910C059D
:10666000222309F48DC06A017B015C010E949B51C9
:106670000091B90C1091BA0C2091BB0C3091BC0C5C
:106680000C591F4F2F4F3F4F061717072807390781
:1066900008F076C0F7FE08C087010095109560E00D
:1066A000802F0E94B1654BC060E080E00E94B16520
:1066B0000E949B5128EE33E040E050E00E94F4B38A
:1066C000CA01B90120E831E541E050E00E94F4B38D
:1066D000AB01BC012AE0CE0101960E94FB59BE012C
:1066E0006F5F7F4FCE0107960E947A5A6CEF7AE077
:1066F000CE0107960E949158BC01CE010D960E94D2
:106700007A5ACE0107960E949859CE0101960E94AE
:106710009859BE01635F7F4F8AE993E10E94E15A75
:1067200009891A89E114F10431F00E0D1F1D60E092
:10673000802F0E94B165CE010D960E949859B50137
:106740008AE993E10E94E15A6DE976E08AE993E1F2
:106750000E94EF5AF501848160E0800F0E94B165CC
:106760000E949B516093B90C7093BA0C8093BB0C40
:106770009093BC0CB601DD0C880B990B0E94635101
:1067800062960FB6F894DEBF0FBECDBFDF91CF91FA
:106790001F910F91FF90EF90DF90CF90BF90AF903F
:1067A0000895BF92CF92DF92EF92FF920F931F93C3
:1067B000CF93DF93CDB7DEB762970FB6F894DEBF05
:1067C0000FBECDBF6C018B017A0180910802882336
:1067D00009F47DC080910C05882309F478C077FF07
:1067E00007C00095109560E0802F0E94B1654EC0F3
:1067F00060E080E00E94B1650E949B5128EE33E08A
:1068000040E050E00E94F4B3CA01B90120E831E54C
:1068100041E050E00E94F4B3AB01BC012AE0CE019C
:1068200001960E94FB59BE016F5F7F4FCE01079614
:106830000E947A5A6CEF7AE0CE0107960E94915836
:10684000BC01CE010D960E947A5ACE0107960E9495
:106850009859CE0101960E949859BE01635F7F4FFF
:106860008AE993E10E94E15AB98860E08B2D0E9489
:10687000B1650115110511F40B2D04C060E0802FE6
:106880000E94B165CE010D960E949859B6018AE921
:1068900093E10E94E15A6CE876E08AE993E10E9474
:1068A000EF5AF601848160E0800F0E94B1650E947A
:1068B0009B516093B90C7093BA0C8093BB0C90936E
:1068C000BC0CB701FF0C880B990B0E9463516296B8
:1068D0000FB6F894DEBF0FBECDBFDF91CF911F91F1
:1068E0000F91FF90EF90DF90CF90BF9008952F927F
:1068F0003F924F925F926F927F928F929F92AF9250
:10690000BF92CF92DF92EF92FF920F931F93CF939C
:10691000DF93CDB7DEB7E4970FB6F894DEBF0FBEB6
:10692000CDBF8091AB13882319F01092AB13C1C374
:1069300081E08093AB137E018FE1E80EF11C62ECE5
:1069400079E0C7010E94825A212C312C82E08BA76A
:106950001E2D0F2D88EE882E83E0982EA12CB12CB1
:1069600090E8492E91E5592E66246394712CF1012B
:106970003197E031F10530F48827E856FF4F8F4F0B
:106980000C94A0B762EC79E0812F902F0E943559CA
:106990008091801190918111892B31F46EEE77E016
:1069A000812F902F0E9435598091801190918111F3
:1069B000019731F462EF77E0812F902F0E943559D3
:1069C0008091801190918111029731F468EF77E006
:1069D000812F902F0E9435598BA19CA1892BB9F052
:1069E0006EE873E1812F902F0E940959612F702F5B
:1069F000CE0101960E947A5A48EC50E06FEF7FEF8B
:106A0000CE010196CEDECE0101960E9498596DEF1F
:106A100077E0CE0101960E94825A68E873E1CE01C8
:106A200001960E94A858BC01CE0107960E947A5A8E
:106A300040ED57E06FEF7FEFCE01079679DDCE0195
:106A400007960E949859CE0101960E94985980910C
:106A50008011909181110197E1F5CE0101960E947C
:106A6000C2638D819E81009781F1E981FA81208145
:106A7000222359F1079748F164EB78E0CE0107969D
:106A80000E94725A48EC50E06FEF7FEFCE010796FC
:106A9000CEDDCE0107960E949859BE016F5F7F4FF1
:106AA000CE0107960E947A5A48EC50E06FEF7FEFD4
:106AB000CE0107963DDDCE0107960E94985960ED04
:106AC00077E080E090E00E946351CE0101960E9441
:106AD000985964E670E080E090E00E94635182E0A3
:106AE0008093371010923B10CBC268EA78E0CE0159
:106AF00001960E94725A48EC50E06FEF7FEFCE0192
:106B0000019695DDCE0101960E9498590E949B51F5
:106B10006B017C010E949B51A50194010E9420B44D
:106B2000CA01B901A30192010E9420B420E13EE014
:106B300040E050E00E94F4B32CA73DA74EA75FA70A
:106B40002CE330E040E050E00E94F4B328AB39ABD6
:106B50004AAB5BABAB01BC012AE0CE0101960E94BF
:106B6000FB592AE048A959A96AA97BA9CE01079631
:106B70000E94FB592AE04CA55DA56EA57FA5CE011C
:106B80000D960E94FB59C701B601A50194010E9410
:106B900020B4CA01B901A30192010E9420B4BA0134
:106BA000A9012AE0CE0149960E94FB59BE01675E09
:106BB0007F4FCE0143960E947A5A62E078E0CE0180
:106BC00043960E949158BE01635F7F4F0E94A85870
:106BD00065E078E00E949158BE01695F7F4F0E9496
:106BE000A85868E078E00E949158BE016F5F7F4F1F
:106BF0000E94A85862EE75E00E949158BC01CE0137
:106C000085960E947A5ACE0143960E949859CE01E9
:106C100049960E949859CE010D960E949859CE012E
:106C200007960E949859CE0101960E94985940ED0E
:106C300057E06FEF7FEFCE0185967ADCCE01859627
:106C40001DC28091C30C9091C40C019719F469E99D
:106C500078E002C06BE878E0CE0101960E94725A9B
:106C600048EC50E06FEF7FEFCE010196E0DCCE0103
:106C700001960E9498596BE778E0F3C16BE678E0E3
:106C8000CE0101960E94725A48EC50E06FEF7FEF00
:106C9000CE010196CCDCCE0101960E9498596EE59A
:106CA00078E0DFC161E578E0CE0101960E94725A7A
:106CB00048EC50E06FEF7FEFCE010196B8DCCE01DB
:106CC00001960E94985966E478E0CBC16AE378E0C7
:106CD000CE0101960E94725A48EC50E06FEF7FEFB0
:106CE000CE010196A4DCCE0101960E94985969E27A
:106CF00078E0B7C18091C30C9091C40C039719F44C
:106D00006EE178E002C064E178E0CE0101960E9475
:106D1000725A48EC50E06FEF7FEFCE01019687DCAE
:106D2000CE0101960E94985969E078E09AC16CEF13
:106D300077E0CE0101960E94725A48EC50E06FEF66
:106D40007FEFCE01019673DCCE0101960E94985927
:106D50006DEE77E086C162EE77E0CE0101960E948B
:106D6000725A48EC50E06FEF7FEFCE0101965FDC86
:106D7000CE0101960E94985965ED77E072C180912D
:106D8000C30C9091C40C029719F464EC77E002C034
:106D900064EB77E0CE0101960E94725A48EC50E015
:106DA0006FEF7FEFCE01019642DCCE0101960E948B
:106DB000985967EA77E055C16BE977E0CE01019613
:106DC0000E94725A48EC50E06FEF7FEFCE010196BF
:106DD0002EDCCE0101960E9498596BE877E041C104
:106DE00060E877E0CE0101960E94725A48EC50E0CC
:106DF0006FEF7FEFCE0101961ADCCE0101960E9463
:106E0000985966E777E02DC16AE677E0CE010196F2
:106E10000E94725A48EC50E06FEF7FEFCE0101966E
:106E200006DCCE0101960E9498596AE577E019C107
:106E3000209139116FE477E0812F902F2CAB0E94C5
:106E40000F592CA924306CF422300CF045C02223B9
:106E500081F0213009F061C06BE078E0812F902F44
:106E600059C0243009F059C06FE078E08FE992E111
:106E700051C0C0903A11D0903B11E0903C11F0907D
:106E80003D1120E030E048E452E4C701B6010E9421
:106E9000C2B287FF02C081E08BA7A701960160E024
:106EA00070E080EA90E40E9418B5AB01BC012BA50C
:106EB000CE0107960E949D5969E378E0CE010196C4
:106EC0000E94825ABE01695F7F4FCE0101960E94E7
:106ED000A85864E178E018C08AE02802B0011124C3
:106EE0004AE0CE0107960E94275A6EEC7BE0CE0165
:106EF00001960E94825ABE01695F7F4FCE010196C2
:106F00000E94A8586DE078E00E949158BC01812F42
:106F1000902F1DC00E94FB5824C060913911062E8D
:106F2000000C770B4AE0CE0107960E94275A65E9CC
:106F30007AE0CE0101960E94825ABE01695F7F4FBE
:106F4000CE0101960E94A858BC018FE992E10E94EF
:106F50000959CE0101960E949859CE0107960E94C8
:106F60009859612F702FCE0101960E947A5A48ECF1
:106F700050E06FEF7FEFCE01019659DBCE01019615
:106F80000E94985964E477E0812F902F0E940F5956
:106F900060913711709138114AE0CE0107960E9436
:106FA000275A6EEC7BE0CE0101960E94825ABE0108
:106FB000695F7F4FCE0101960E94A85866EA7BE088
:106FC0000E949158BC01812F902F0E940959CE0137
:106FD00001960E949859CE0107960E949859612FF8
:106FE000702FCE0101960E947A5A3FC064E377E089
:106FF000CE0101960E94725A48EC50E06FEF7FEF8D
:10700000CE01019614DBCE0101960E94985967E2E9
:1070100077E027C06BE177E0CE0101960E94725ABB
:1070200048EC50E06FEF7FEFCE01019600DBCE0120
:1070300001960E9498596CE077E013C060E077E019
:10704000CE0101960E94725A48EC50E06FEF7FEF3C
:10705000CE010196ECDACE0101960E94985960EFBC
:1070600076E0CE0101960E94725A40ED57E06FEF34
:107070007FEFCE0101965CDACE0101960E9498590D
:107080000E941A84882319F01092AB130EC00E943C
:1070900041708091AB13882341F08FEF281A380A92
:1070A00081E12816310409F062CCCE014F960E948E
:1070B0009859E4960FB6F894DEBF0FBECDBFDF91AE
:1070C000CF911F910F91FF90EF90DF90CF90BF90E5
:1070D000AF909F908F907F906F905F904F903F9078
:1070E0002F9008950F931F93CF93DF9300D000D07C
:1070F000CDB7DEB72091C50C2223A9F08C016CEE30
:1071000079E0CE0101960E94825AB801CE01019623
:107110000E94A858BC018EE89FE00E94D05BCE017F
:1071200001960E94985926960FB6F894DEBF0FBEBE
:10713000CDBFDF91CF911F910F9108954F925F9234
:107140006F927F928F929F92AF92BF92CF92DF9277
:10715000EF92FF920F931F93CF93DF93CDB7DEB7DC
:10716000CA54D1090FB6F894DEBF0FBECDBF8C0153
:1071700062EC79E0CE018B960E94825A62EC79E053
:10718000CE0185960E94825ABE016F5F7F4F84EDCB
:1071900092E10E945E4F8D889E88AF88B88C498CA2
:1071A0005A8C6B8C7C8C8D8D9E8DAF8DB8A1279663
:1071B0008CAF9DAFAEAFBFAF2797C80101970397C4
:1071C00008F0D4C1A3019201C501B40190580E94F6
:1071D000C5B42BED3FE049EC5FE30E9452B420912F
:1071E000390230913A0240913B0250913C020E9498
:1071F00052B46B017C0120E030E0A9010E94C2B2D0
:1072000087FD09C0C092B50CD092B60CE092B70CC5
:10721000F092B80C10C02BED3FE049EC50E4C701F0
:10722000B6010E9452B46093B50C7093B60C809373
:10723000B70C9093B80CC090B50CD090B60CE09001
:10724000B70CF090B80C2BED3FE049EC50E4C701CF
:10725000B6010E9407B6181684F42BED3FE049EC06
:1072600050E4C701B6010E9451B46093B50C70930D
:10727000B60C8093B70C9093B80C20E030E044E358
:1072800053E46091B50C7091B60C8091B70C90915D
:10729000B80C0E9427B32BED3FE049E450E40E9474
:1072A00018B56093B10C7093B20C8093B30C9093AB
:1072B000B40C0E94B1B54AE0CE01C7960E94275A8D
:1072C00067E178E0CE01C1960E94825ABE01695CF6
:1072D0007F4FCE01C1960E94A85861E278E00E94DB
:1072E0009158BC0185EA92E10E944A59CE01C196AB
:1072F0000E949859CE01C7960E949859C090B10C2F
:10730000D090B20CE090B30CF090B40C20E030E0E0
:1073100044EB52E4C701B6010E94C2B2181694F0C1
:1073200020E030E040E05FE3C701B6010E9452B4C4
:107330000E94B1B54AE0CE01C7960E94275A68E282
:1073400078E023C020E030E044E353E4C701B60115
:107350000E94C2B21816A4F1A701960160E070E87D
:1073600084E393E40E9451B46093B10C7093B20C27
:107370008093B30C9093B40C0E94B1B54AE0CE0157
:10738000C7960E94275A6BE278E0CE01C1960E9410
:10739000825ABE01695C7F4FCE01C1960E94A858F7
:1073A000BC01CE018B960E944A59CE01C1960E9423
:1073B0009859CE01C7960E94985968E27BE063C055
:1073C00020E030E047E853E4C701B6010E94C2B2B2
:1073D000181604F120E030E044E353E4C701B6019D
:1073E0000E9451B420E030E040E05FE30E9452B4DC
:1073F0006093B10C7093B20C8093B30C9093B40C67
:107400000E94B1B54AE0CE01C7960E94275A6BE2AE
:1074100078E01FC0A701960160E070E084EB93E480
:107420000E9451B420E030E040E05FE30E9452B49B
:107430006093B10C7093B20C8093B30C9093B40C26
:107440000E94B1B54AE0CE01C7960E94275A68E271
:1074500078E0CE01C1960E94825ABE01695C7F4FDE
:10746000CE01C1960E94A858BC01CE018B960E9405
:107470004A59CE01C1960E949859CE01C7960E94E2
:1074800098596EE278E0CE0185960E943559BE018A
:10749000655D7F4FCE01C1960E947A5A4AE050E066
:1074A00060E070E0CE01C1967CD9CE01C1960E9409
:1074B00098590E949B512091B90C3091BA0C40917F
:1074C000BB0C5091BC0C69017A01A4E6CA0ED11C18
:1074D000E11CF11CC616D706E806F90608F436C208
:1074E00028962FAF289729963FAF29972A964FAF16
:1074F0002A972B965FAF2B970E949B510E94C6B292
:107500006B017C0128962FAD289729963FAD2997CE
:107510002A964FAD2A972B965FAD2B97CA01B901DA
:107520000E94C8B220E030E048EC51E40E9452B41E
:107530009B01AC01C701B6010E94C2B287FD06C221
:1075400065EC7BE0CE01C1960E94825ABE016B5D64
:107550007F4FCE01C1960E94A858BC01CE018B96E8
:107560000E940959CE01C1960E949859C8010297FC
:10757000029708F0C5C120E030E040E251E4C501C7
:10758000B4010E9427B36B017C0120E030E040E2AF
:1075900051E4C301B2010E9427B34B015C0120E01A
:1075A00030E040E251E427966CAD7DAD8EAD9FADED
:1075B00027970E9427B32B013C010E949B512091E9
:1075C000800C3091810C4091820C5091830C621B95
:1075D000730B840B950B0E94C6B220E030E04AE7A3
:1075E00054E40E9418B5AB01BC0123E0CE01C7965C
:1075F0000E94CC5969E378E0CE01C1960E94825A7C
:10760000BE01695C7F4FCE01C1960E94A8586CEF05
:107610007AE00E949158BC0183E992E10E944A59A4
:10762000CE01C1960E949859CE01C7960E949859E2
:1076300063E972E1CE01C1960E947A5A65EA72E16D
:10764000CE01C1960E94A858BE01655D7F4F0E9481
:10765000A858BC01CE018B960E944A59CE01C19612
:107660000E94985961E876E08FE992E10E940F59F3
:1076700021E0B701A601CE01C1960E94CC59BE01FE
:107680006F5C7F4F8FE992E10E940959CE01C1964C
:107690000E94985921E0B301A201CE01CD960E942B
:1076A000CC5921E0B501A401CE01C7960E94CC5966
:1076B00065EC7BE0CE01C1960E94825ABE01695CF6
:1076C0007F4FCE01C1960E94A85865EC7BE00E94D6
:1076D0009158BE01635C7F4F0E94A85860E378E038
:1076E0000E949158BC018FE992E10E940959CE0194
:1076F000C1960E949859CE01C7960E949859CE0112
:10770000CD960E949859A7019601C701B6010E9423
:1077100027B36B017C01A5019401C501B4010E944E
:1077200027B39B01AC01C701B6010E9452B46B01A3
:107730007C01A3019201C301B2010E9427B39B0106
:10774000AC01C701B6010E9452B40E9410B76B0190
:107750007C016093AD0C7093AE0C8093AF0C909352
:10776000B00C64E378E08FE992E10E94FB5821E0DD
:10777000B701A601CE01C1960E94CC59BE016F5C33
:107780007F4FCE01C7960E947A5A65E478E0CE0119
:10779000C7960E949158BC0185EA92E10E944A591D
:1077A000CE01C7960E949859CE01C1960E94985961
:1077B00065EA72E18FE992E10E940959C090AD0C2F
:1077C000D090AE0CE090AF0CF090B00C20E030E028
:1077D0004AE754E4C701B6010E9407B687FD29C0F5
:1077E00020E030E04AE754E4C701B6010E9418B532
:1077F000AB01BC0123E0CE01C1960E949D59BE01A0
:107800006F5C7F4FCE01C7960E947A5A66E478E09B
:10781000CE01C7960E949158BC0185EA92E10E9470
:107820004A59CE01C7960E949859CE01C1960E942E
:10783000985920E030E64AE656E46091AD0C70912C
:10784000AE0C8091AF0C9091B00C0E94C2B2BE0100
:10785000655D7F4F87FF50C0CE01C1960E947A5A66
:1078600068E378E0CE01C1960E9491586FE972E119
:107870000E94A858BC018FE992E10E944A59CE01AA
:10788000C1960E94985903301105A1F46FE972E185
:10789000CE01C1960E947A5ACE01C1960E94439AA7
:1078A000CE01C1960E94985962EC79E08FE992E18D
:1078B0000E9435596BE378E0CE01C1960E94825A4E
:1078C00065EA72E1CE01C1960E94A858BC01CE01C2
:1078D000C7960E947A5A4AE050E06FEF7FEFCE01E0
:1078E000C7960E949832CE01C7960E949859CE0141
:1078F000C1960E94985904C08FE992E10E944A59AA
:107900006AE070E080E090E00E946351CE018596CD
:107910000E949859CE018B960E949859C65BDF4F02
:107920000FB6F894DEBF0FBECDBFDF91CF911F9190
:107930000F91FF90EF90DF90CF90BF90AF909F900E
:107940008F907F906F905F904F90089562EC79E0F8
:10795000CE01C1960E94825ACE01C1960E946C321D
:10796000CE01C1960E949859BE016B5D7F4F8AE996
:1079700093E10E94E15AE4CD1F93CF93DF93CDB7FB
:10798000DEB7A8970FB6F894DEBF0FBECDBF182F95
:107990000E94BA668EE10E94966562E08BE290E1F9
:1079A0000E94FF8B60E08BE290E10E94FF8B0E94BF
:1079B0008F658EE10E94966561E08BE290E10E9406
:1079C000FF8B60E28BE290E10E94FF8B0E948F654B
:1079D00080E290E09093D8128093D71280E090E8F4
:1079E000A9E8B4E480934E0290934F02A093500212
:1079F000B093510280E090E0A5E7B4E480934A029E
:107A000090934B02A0934C02B0934D02BE016F5F66
:107A10007F4F84ED92E10E94114F112309F494C02D
:107A200066E576E08EE89FE00E94EF5A8EE89FE0E0
:107A30000E94BD5B66E476E08EE89FE00E94EF5A0C
:107A4000BE016F5F7F4F8EE89FE00E94C05B66E3E0
:107A500076E08EE89FE00E94EF5A4D855E856F8547
:107A600078892AE030E08EE89FE00E94705B8EE823
:107A70009FE00E94BD5B66E276E08EE89FE00E9498
:107A8000EF5A49895A896B897C892AE030E08EE86F
:107A90009FE00E94705B8EE89FE00E94BD5B66E104
:107AA00076E08EE89FE00E94EF5A20E030E040E26E
:107AB00051E4698D7A8D8B8D9C8D0E9427B342E0B5
:107AC0000E94DC6564E478E08EE89FE00E94C05B81
:107AD00066E076E08EE89FE00E94EF5A20E030E01A
:107AE00040E251E46D8D7E8D8F8D98A10E9427B369
:107AF00042E00E94DC6564E478E08EE89FE00E944A
:107B0000C05B66EF75E08EE89FE00E94EF5A20E0D0
:107B100030E040E251E469A17AA18BA19CA10E94CE
:107B200027B342E00E94DC6564E478E08EE89FE0E1
:107B30000E94C05B60ED75E08EE89FE00E94EF5A06
:107B40008EE89FE00E94BD5B64EF71E080E090E012
:107B50000E946351A8960FB6F894DEBF0FBECDBF4A
:107B6000DF91CF911F910895EF92FF920F931F9392
:107B7000CF93DF931F92CDB7DEB77C01FC0100816C
:107B80001181C80169830E94DEB36981681719F009
:107B9000C8010E94E6B3C7010F90DF91CF911F91FA
:107BA0000F91FF90EF900895CF92DF92EF92FF92A6
:107BB0000F931F93CF93DF93EC016A017B01E88958
:107BC000F98982E080834115514E61057105B1F05C
:107BD00060E079E08DE390E0A70196010E9420B477
:107BE00089019A010150110921093109369527951A
:107BF00017950795980101151041A8F0E889F989B2
:107C0000108260E874E88EE190E0A70196010E947E
:107C100020B4DA01C9010197A109B109B695A79568
:107C2000979587959C01EC85FD853083EE85FF85D2
:107C30002083188EEC89FD8986E08083EA89FB89A0
:107C4000808180618083EA89FB898081886080836C
:107C5000EA89FB89808180688083EA89FB89808149
:107C60008F7D8083DF91CF911F910F91FF90EF90D7
:107C7000DF90CF900895CF93DF93EC01FB01248137
:107C800035810E94965ACE01DF91CF9108952F92AF
:107C90003F924F925F926F927F928F929F92AF929C
:107CA000BF92DF92EF92FF920F931F93CF93DF93D8
:107CB000CDB7DEB7A8970FB6F894DEBF0FBECDBF25
:107CC0007E0145E1E40EF11C65E778E0C7010E9402
:107CD000825AB70187EB92E10E947658811117C052
:107CE00068E976E0CE0101960E94825ABE016F5F7C
:107CF0007F4F87EB92E10E947658DD24D394811167
:107D000001C0D12CCE0101960E94985902C0DD24F9
:107D1000D394C7010E949859DD2009F4D8C08091FE
:107D2000BB129091BC12409710F00C94B54742E002
:107D300050E067EB72E1CE0101969DDFBE016F5FFF
:107D40007F4F89E992E10E945F59CE0101960E941E
:107D5000985969E972E1CE0101960E947A5ACE01E2
:107D60000196C0D9CE0101960E94985989E992E105
:107D70000E94865720E030E048EC52E40E9427B38E
:107D80000E94B1B5AB01BC0140933D0250933E024D
:107D900060933F02709340022AE0CE0101960E9458
:107DA000FB59CE0101969ED9CE0101960E949859A9
:107DB00060913D0270913E0280913F02909140029D
:107DC0008B019C0100591F452140310901341C4998
:107DD00021053105D0F068E478E0CE0101960E94DB
:107DE000825A69E972E1CE0101960E94A8586BE5BA
:107DF00078E00E949158BC018FE992E10E944A59B3
:107E0000CE0101960E9498594AC019821A821B829B
:107E10001C821D821E821F8218860E94C8B220E02A
:107E200030E048EC52E40E9418B58E010F5F1F4FFE
:107E300022E047E00E94CFADBC018FE992E10E94B1
:107E400035596BE678E0C7010E94825A6FE972E10A
:107E5000C7010E94A85868E778E00E949158BC01C9
:107E60008FE992E10E944A59C7010E9498591092E5
:107E7000EF0C1092EE0C80913D0290913E02A09189
:107E80003F02B091400280930A1190930B11A0938E
:107E90000C11B0930D1180E090E00E9421696CEE0E
:107EA00079E0CE0101960E94825A6FE972E1CE011B
:107EB00001960E94A858BC01C7010E947A5AC701C6
:107EC0000E94439AC7010E9498590C94AD476DE7F0
:107ED00078E0C7010E94825AB70187EB92E10E94C5
:107EE0007658811117C062E878E0CE0101960E94B1
:107EF000825ABE016F5F7F4F87EB92E10E947658F6
:107F0000DD24D394811101C0D12CCE0101960E94B1
:107F1000985902C0DD24D394C7010E949859DD20EE
:107F2000B9F126E030E044E050E067EB72E1CE01C9
:107F300001960E94965ABE016F5F7F4F89E992E1D8
:107F40000E945F59CE0101960E94985989E992E1F9
:107F50000E949157709383116093821170931E0554
:107F600060931D0567EB72E1CE0101960E947A5A7B
:107F7000CE010196B7D8CE0101960E949859109271
:107F8000EF0C1092EE0C80E090E00E942169E9C7AE
:107F900067E878E0CE0183960E94825ABE016D5D4B
:107FA0007F4F87EB92E10E9476588111DFC76AE824
:107FB00078E0C7010E94825AB70187EB92E10E94E4
:107FC0007658811116C06DE878E0CE0101960E94C6
:107FD000825ABE016F5F7F4F87EB92E10E94765815
:107FE00011E0811101C010E0CE0101960E94985964
:107FF00001C011E0C7010E949859CE0183960E94EA
:1080000098591111B7C76BEA78E0C7010E94825AEC
:10801000B70187EB92E10E947658811117C061EB9E
:1080200078E0CE0101960E94825ABE016F5F7F4FB9
:1080300087EB92E10E947658DD24D394811101C030
:10804000D12CCE0101960E94985902C0DD24D39410
:10805000C7010E949859DD2009F4BEC08091BB126F
:108060009091BC120797F0F046E050E067EB72E1A8
:10807000CE01019600DEBE016F5F7F4F89E992E17C
:108080000E945F59CE0101960E94985989E992E1B8
:108090000E948657609323057093240580932505DD
:1080A00090932605809110029091110299270E94C9
:1080B0004094BC01990F880B990B0E94C8B22DE027
:1080C00038E643E55BE30E9427B32B013C01209196
:1080D0006B0230916C0240916D0250916E020E94D1
:1080E000C2B218164CF06091530270915402809104
:1080F0005502909156021BC020917F023091800260
:108100004091810250918202C301B2010E9407B6E0
:1081100087FF05C0C301B2010E94006808C06091DA
:108120006702709168028091690290916A0220E072
:1081300030E048EC52E40E9427B32B013C0120E0E0
:1081400030E0A9010E94C2B2181634F0412C512C23
:10815000E8EA6E2EE1E47E2E40922305509224053B
:10816000609225057092260540923E1150923F1173
:1081700060924011709241118091C50C882381F06A
:1081800068E07AE08EE89FE00E94EF5A6091230554
:108190007091240580912505909126050E94BE7C52
:1081A0001092EF0C1092EE0C80E090E00E9421699A
:1081B0006EEF79E08FE992E10E940F59409123051B
:1081C00050912405609125057091260522E0CE018D
:1081D00001960E94CC597DC267EB78E0C7010E94EE
:1081E000825AB70187EB92E10E947658811117C03D
:1081F0006BEB78E0CE0101960E94825ABE016F5F60
:108200007F4F87EB92E10E947658DD24D394811151
:1082100001C0D12CCE0101960E94985902C0DD24E4
:10822000D394C7010E949859DD2009F46DC0B09025
:108230000E0260E08B2D0E94DA5009E110E0412C23
:10824000512C32018B2D0E941951BC01990F880BC2
:10825000990B0E94C8B29B01AC01C301B2010E94FC
:1082600052B42B013C016AE070E080E090E00E9493
:1082700063510150110931F720E030E040EA50E449
:10828000C301B2010E9427B320E030EC4FE754E471
:108290000E9418B520E030E048EC51E40E9418B587
:1082A00060931F057093200580932105909322050C
:1082B00060935411709355118093561190935711F8
:1082C0001092EF0C1092EE0C80E090E00E94216979
:1082D0006BEE79E08FE992E10E940F5940911F0502
:1082E00050912005609121057091220522E0CE0178
:1082F00001960E94CC59BE016F5F7F4FC7010E945B
:108300007A5A64ED75E06FC06FEB78E0C7010E94A8
:10831000825AB70187EB92E10E947658811117C00B
:1083200065EC78E0CE0101960E94825ABE016F5F33
:108330007F4F87EB92E10E947658DD24D394811120
:1083400001C0D12CCE0101960E94985902C0DD24B3
:10835000D394C7010E949859DD2009F457C0809139
:108360003911082E000C990B0197039708F047C0AC
:1083700089E390E00E944094BC01990F880B990B0F
:108380000E94C8B22AE137E64CE950E40E9427B3C4
:1083900060933A1170933B1180933C1190933D117F
:1083A0001092EF0C1092EE0C80E090E00E94216998
:1083B0006AEC79E08FE992E10E940F5940913A11FD
:1083C00050913B1160913C1170913D1122E0CE0122
:1083D00001960E94CC59BE016F5F7F4FC7010E947A
:1083E0007A5A6BEC78E0C7010E949158BC018FE982
:1083F00092E10E940959C7010E94985971C164EA2B
:1084000079E08FE992E10E940F599DC56EEC78E00A
:10841000C7010E94825AB70187EB92E10E94765809
:10842000811117C062ED78E0CE0101960E94825A58
:10843000BE016F5F7F4F87EB92E10E947658DD248B
:10844000D394811101C0D12CCE0101960E9498597C
:1084500002C0DD24D394C7010E949859DD2009F49D
:1084600042C126E030E044E050E067EB72E1CE012B
:1084700001960E94965ABE016F5F7F4F89E992E193
:108480000E945F59CE0101960E94985989E992E1B4
:108490000E9491574B015C011B0162ED7AE0CE0115
:1084A00001960E94825ABE016F5F7F4F87EB92E177
:1084B0000E94FB57AC014F5F5F4F67EB72E1C70152
:1084C000DADBB70189E992E10E945F59C7010E9496
:1084D0009859CE0101960E94985910910C0289E991
:1084E00092E10E9486572B013C018091C50C8823A4
:1084F000B9F06DEB78E08EE89FE00E94EF5A4AE019
:1085000050E0B4018EE89FE00E94B75B65EC7BE031
:108510008EE89FE00E94E05BC301B2010E94BE7C36
:10852000612FC7010E943455F886EF821D821E829A
:10853000198289E08A8381E08B838C831C8A1B8A61
:10854000CE0101960E949054CE0101960E942353C1
:10855000CE0101960E94FC7E0E8110E00B301105C9
:1085600014F00AE010E0FBE58F16910408F44CC00B
:1085700076ECA72E7CE0B72E3501212C312C210181
:10858000E12CF12CE016F106B9F06E2DCE0101962A
:108590000E9422549B01AC01F3016193719381937A
:1085A00091933F01C201B1010E9452B41B012C0101
:1085B000FFEFEF1AFF0AE6CFB801012E000C880B7F
:1085C000990B0E94C8B29B01AC01C201B1010E948B
:1085D00018B52B013C01E12CF12CE016F10609F451
:1085E00053C0F5012081318142815381C301B20121
:1085F0000E9451B4F50161937193819391935F014E
:10860000FFEFEF1AFF0AE9CF12141304ECF402157E
:1086100013050CF0840101501109602FCE01019661
:108620000E9422549B01AC01000F111F000F111F6B
:108630000A53134FC301B2010E9451B4F801608381
:1086400071838283938320C02328F1F496ECA92EB2
:108650009CE0B92EE12CF12CE016F106A9F06E2D6C
:10866000CE0101960E9422549B01AC01C301B201CC
:108670000E9451B4F50161937193819391935F01CD
:10868000FFEFEF1AFF0AE8CFE6ECFCE0A8E5B1E166
:1086900041915191619171914D935D936D937D9352
:1086A0004CE0EE3EF407A1F71092EF0C1092EE0CA6
:1086B00080E090E00E94216963E879E08FE992E12F
:1086C0000E940F5944E050E067EB72E1CE01019641
:1086D000D2DABE016F5F7F4F8FE992E10E940959A4
:1086E000CE0101962EC466ED78E0C7010E94825A41
:1086F000B70187EB92E10E947658811117C06DEDAA
:1087000078E0CE0101960E94825ABE016F5F7F4FD2
:1087100087EB92E10E947658DD24D394811101C049
:10872000D12CCE0101960E94985902C0DD24D39429
:10873000C7010E949859DD2009F419C127E030E0F3
:1087400046E050E067EB72E1CE0101960E94965A36
:10875000BE016F5F7F4F89E992E10E945F59CE01B0
:1087600001960E94985989E992E10E9491578B01E4
:108770006093391187EB92E10E949C5765EC7BE096
:10878000CE0101960E94825ABE016F5F7F4F87EB38
:1087900092E10E94FB57AC014F5F5F4F67EB72E1C4
:1087A000C70169DAC7010E94865760933A11709336
:1087B0003B1180933C1190933D11C7010E94985941
:1087C000CE0101960E94985962E779E08FE992E123
:1087D0000E940F590430110594F4023011050CF079
:1087E00058C001151105B1F00130110509F096C00E
:1087F00064E679E08FE992E10E94B95872C00430D2
:10880000110509F08BC061E579E08FE992E10E94E2
:10881000B958A4C020E030E0A90160913A117091EC
:108820003B1180913C1190913D110E94C2B21816EB
:1088300064F080E090E0A0E8BFE380933A11909369
:108840003B11A0933C11B0933D1120913A1130910E
:108850003B1140913C1150913D1160E070E080EA85
:1088600090E40E9418B5AB01BC0122E0C7010E9450
:108870009D5964EE78E0CE0101960E94825AB701BC
:10888000CE0101960E94A85864E178E00E949158B8
:1088900059C068E579E08FE992E10E94B9588AE011
:1088A000809FB001819F700D11244AE0CE01019696
:1088B0000E94275ABE016F5F7F4FC7010E947A5AFC
:1088C0006DE078E0C7010E949158BC018FE992E108
:1088D0000E940959C7010E949859CE0101960E9431
:1088E000985920E030E048E453E460913A117091E7
:1088F0003B1180913C1190913D110E94C2B218161B
:108900006CF180E090E4ACE1B5E480933A1190938F
:108910003B11A0933C11B0933D1120C060913911DF
:10892000062E000C770B4AE0C7010E94275A6FEE13
:1089300078E0CE0101960E94825AB701CE010196DD
:108940000E94A858BC018FE992E10E940959CE010A
:1089500001960E949859C7010E9498591092EF0CF5
:108960001092EE0C80E090E00E942169ECC266EF6C
:1089700078E0C7010E94825AB70187EB92E10E941A
:108980007658811117C06DEF78E0CE0101960E94F4
:10899000825ABE016F5F7F4F87EB92E10E9476584B
:1089A000DD24D394811101C0D12CCE0101960E9407
:1089B000985902C0DD24D394C7010E949859DD2044
:1089C00009F4C7C027E030E046E050E067EB72E111
:1089D000CE0101960E94965ABE016F5F7F4F89E9D2
:1089E00092E10E945F59CE0101960E94985989E94F
:1089F00092E10E9491576093361187EB92E10E94B9
:108A00009C5789E992E10E94915761157105810592
:108A1000910519F485E090E007C06130710581058A
:108A2000910539F489E190E09093381180933711E2
:108A300022C065EC7BE0CE0101960E94825ABE0105
:108A40006F5F7F4F87EB92E10E94FB57AC014F5F56
:108A50005F4F67EB72E1C7010ED9C7010E949157C2
:108A60007093381160933711C7010E949859CE0155
:108A700001960E9498591092EF0C1092EE0C80E033
:108A800090E00E94216960E479E08FE992E10E9420
:108A90000F5980913611833034F565E379E08FE921
:108AA00092E10E94B95860913711709138114AE0F3
:108AB000CE0101960E94275ABE016F5F7F4FC7010A
:108AC0000E947A5A66EA7BE0C7010E949158BC0175
:108AD0008FE992E10E940959C7010E949859CE017D
:108AE00001960E9498598091361183300CF42BC264
:108AF00060913711709138114AE0CE0183960E943F
:108B0000275A60913611062E000C770B4AE0C701F8
:108B10000E94275A6FEE78E0CE0101960E94825A99
:108B2000B701CE0101960E94A858BE016D5D7F4F2E
:108B30000E94A858BC018FE992E10E940959CE0118
:108B400001960E949859C7010E949859CE018396B8
:108B5000F8C164E079E0C7010E94825AB70187EB4F
:108B600092E10E947658811117C068E079E0CE0149
:108B700001960E94825ABE016F5F7F4F87EB92E1A0
:108B80000E947658DD24D394811101C0D12CCE01EE
:108B900001960E94985902C0DD24D394C7010E9417
:108BA0009859DD2009F455C080910A0290910B027A
:108BB0000E94547B6093190570931A0580931B05DE
:108BC00090931C05609322117093231180932411BC
:108BD0009093251180E090E5A3ECB7E480930D0518
:108BE00090930E05A0930F05B093100580931A1172
:108BF00090931B11A0931C11B0931D118091C50C73
:108C0000882381F067E179E08EE89FE00E94EF5AC7
:108C10006091190570911A0580911B0590911C05B2
:108C20000E94BE7C1092EF0C1092EE0C80E090E05F
:108C30000E9421694091190550911A0560911B0508
:108C400070911C0522E0C7010E94CC596CE079E0CC
:108C500065C167E179E0C7010E94825AB70187EBDD
:108C600092E10E947658811117C06BE179E0CE0144
:108C700001960E94825ABE016F5F7F4F87EB92E19F
:108C80000E947658DD24D394811101C0D12CCE01ED
:108C900001960E94985902C0DD24D394C7010E9416
:108CA0009859DD2009F485C08091BB129091BC12C7
:108CB0000497F8F044E050E067EB72E1CE010196D2
:108CC0000E943B3EBE016F5F7F4F89E992E10E94A7
:108CD0005F59CE0101960E94985989E992E10E945C
:108CE0008657609311057093120580931305909336
:108CF00014058091110590911205A0911305B09172
:108D000014058093161190931711A0931811B09326
:108D100019118091C50C882389F06EEF78E08EE8F8
:108D20009FE00E94EF5A60911105709112058091A9
:108D300013059091140542E00E94DC6580910A02BF
:108D400090910B020E94547B609315057093160559
:108D5000809317059093180560931E1170931F114F
:108D600080932011909321118091C50C882381F06C
:108D700064EF78E08EE89FE00E94EF5A609115055D
:108D80007091160580911705909118050E94BE7C80
:108D90001092EF0C1092EE0C80E090E00E9421699E
:108DA00040911505509116056091170570911805B1
:108DB000AFC067E279E0C7010E94825AB70187EB32
:108DC00092E10E947658811117C06BE279E0CE01E2
:108DD00001960E94825ABE016F5F7F4F87EB92E13E
:108DE0000E947658DD24D394811101C0D12CCE018C
:108DF00001960E94985902C0DD24D394C7010E94B5
:108E00009859DD2009F4AFC08091BB129091BC123B
:108E10000497F8F044E050E067EB72E1CE01019670
:108E20000E943B3EBE016F5F7F4F89E992E10E9445
:108E30005F59CE0101960E94985989E992E10E94FA
:108E4000865760930D0570930E0580930F059093E0
:108E5000100580910D0590910E05A0910F05B09120
:108E6000100580931A1190931B11A0931C11B093BD
:108E70001D118091C50C882389F06BED78E08EE898
:108E80009FE00E94EF5A60910D0570910E05809150
:108E90000F059091100542E00E94DC6580910A0266
:108EA00090910B020E94547B6093190570931A05F0
:108EB00080931B0590931C056093221170932311DE
:108EC00080932411909325118091C50C882381F003
:108ED00061ED78E08EE89FE00E94EF5A60911905FD
:108EE00070911A0580911B0590911C050E94BE7C13
:108EF0001092EF0C1092EE0C80E090E00E9421693D
:108F00004091190550911A0560911B0570911C053F
:108F100022E0C7010E94CC596FE179E0CE010196B1
:108F20000E94825AB701CE0101960E94A858BC0146
:108F30008FE992E10E944A59CE0101960E94985908
:108F4000C7010E9498596FE972E1CE0101960E9413
:108F50007A5ACE0101960E94439ACE0101960E9450
:108F60009859109209028D2D6DC16CC1CE01839666
:108F70000E9498590AE010E0412C512C3201AA2499
:108F8000AA9483E0B82E6EE170E080E090E00E9449
:108F9000635180911A020E941951B5010E948DB748
:108FA000072E000C880B990B0E94C8B220E030E01D
:108FB00040EA50E40E9427B39B01AC01C301B20117
:108FC0000E9452B42B013C0101501109E1F620E04E
:108FD00030E040E251E40E9418B52B013C0160E909
:108FE00078E0CE0183960E94825ABE016D5D7F4F6C
:108FF00087EB92E10E94765881111AC164E978E00A
:10900000C7010E94825AB70187EB92E10E9476580D
:10901000811116C068E978E0CE0101960E94825A5B
:10902000BE016F5F7F4F87EB92E10E94765811E09F
:10903000811101C010E0CE0101960E94985901C033
:1090400011E0C7010E949859CE0183960E94985959
:10905000112309F446C020E030E040E650E4C301AB
:10906000B2010E9427B39B01AC0160E070E080E890
:1090700090E40E9451B4609316027093170280939B
:109080001802909319026BE27AE08FE992E10E9454
:109090000F59409116025091170260911802709179
:1090A000190222E0CE0101960E94CC59BE016F5FE9
:1090B0007F4F8FE992E10E940959CE0101960E94EB
:1090C00098598091160290911702A0911802B091C0
:1090D000190280932E1190932F11A0933011B09309
:1090E00031116CE978E0CE0183960E94825ABE016C
:1090F0006D5D7F4F87EB92E10E94765881119DC094
:1091000061EA78E0C7010E94825AB70187EB92E1D9
:109110000E947658811116C066EA78E0CE01019669
:109120000E94825ABE016F5F7F4F87EB92E10E94DF
:10913000765811E0811101C010E0CE0101960E9425
:10914000985901C011E0C7010E949859CE01839639
:109150000E949859112309F44EC020E030E040E607
:1091600050E4C301B2010E9427B39B01AC0160E04F
:1091700070E080E291E40E9451B460931202709317
:10918000130280931402909315026AE17AE08FE94A
:1091900092E10E940F594091120250911302609186
:1091A00014027091150222E0CE0101960E94CC5962
:1091B000BE016F5F7F4F8FE992E10E940959CE0196
:1091C00001960E9498598091120290911302A091E9
:1091D0001402B09115028093321190933311A09331
:1091E0003411B09335111092EF0C1092EE0C80E018
:1091F00090E00E9421696CEE79E0CE0101960E9418
:10920000825A6FE972E1CE0101960E94A858BC0112
:10921000C7010E947A5AC7010E94439AC7010E945F
:109220009859CE0101960E949859DD24D3949BCE83
:10923000CE0183960E9498590ECFCE0183960E944C
:1092400098598BCFA8960FB6F894DEBF0FBECDBF4E
:10925000DF91CF911F910F91FF90EF90DF90BF9022
:10926000AF909F908F907F906F905F904F903F90C6
:109270002F9008954F925F926F927F928F929F925C
:10928000AF92BF92DF92EF92FF920F931F93CF9313
:10929000DF93CDB7DEB7A9970FB6F894DEBF0FBE48
:1092A000CDBFD82E882351F08091C50C882331F092
:1092B00062EC79E08EE89FE00E94C05B0E94BA6693
:1092C00060E08DE20E94797C60E18DE20E94797C11
:1092D00068E08DE20E94797C409003135090041363
:1092E000609005137090061349825A826B827C82CB
:1092F0008090071390900813A0900913B0900A1360
:109300008D829E82AF82B88680910B1390910C1350
:10931000A0910D13B0910E138EA39FA3A8A7B9A778
:1093200089879A87AB87BC87DD2099F18091C50C2E
:10933000882379F17E019DE0E90EF11C65E17EE074
:10934000C7010E94725AC7010E947238C7010E9469
:1093500098598E010F5F1F4FD8016D917D918D91AE
:109360009D918D0146E00E94DC6565EC7BE08EE816
:109370009FE00E94E05B0E151F0571F762EC79E03B
:10938000C8010E94825AC8010E947238C8010E9416
:10939000985923E938E144E85FE3C301B2010E9430
:1093A00027B32B013C016D877E878F87988B22E442
:1093B00030E645E85FE3C501B4010E9427B34B01E5
:1093C0005C01698B7A8B8B8B9C8B25E83BEE41E9AA
:1093D0005FE36EA17FA188A599A50E9427B36D8B3D
:1093E0007E8B8F8B988F4092031350920413609260
:1093F0000513709206138092071390920813A0929F
:109400000913B0920A1360930B1370930C1380939B
:109410000D1390930E13DD2009F4A5C08091C50CA7
:10942000882309F4A0C07E01B9E1EB0EF11C68E0CD
:109430007EE0C7010E94725AC7010E947238C701BC
:109440000E9498598E01035F1F4FF801619171913D
:10945000819191918F0142E00E94DC6565EC7BE097
:109460008EE89FE00E94E05B0E151F0571F762EC2D
:1094700079E0C8010E94825AC8010E947238C8016E
:109480000E9498594FE053E166E070E082E30E9449
:109490000F7C80901013912C982C882480910F13AE
:1094A000882AA0901213B12CBA2CAA2480911113EF
:1094B000A82AE0901413F12CFE2CEE2480911313B3
:1094C000E82A6BEF7DE08EE89FE00E94EF5A4AE0C9
:1094D00050E0B4018EE89FE00E94B75B65EC7BE052
:1094E0008EE89FE00E94E05B4AE050E0B5018EE824
:1094F0009FE00E94B75B65EC7BE08EE89FE00E94F6
:10950000E05B4AE050E0B7018EE89FE00E94B75B65
:1095100062EC79E08EE89FE00E94C05BC8010E9487
:10952000CD7C62EF7DE08EE89FE00E94EF5A7E01E5
:10953000F5E2EF0EF11CD8016D917D918D919D9119
:109540008D014AE00E94DC6565EC7BE08EE89FE0DF
:109550000E94E05B0E151F0571F762EC79E08EE862
:109560009FE00E94C05B61E08DE10E94797CDD207C
:10957000B1F08091C50C882391F06EED7DE08EE80E
:109580009FE00E94EF5AAE014B5D5F4F61E070E0DB
:109590008DE10E940F7C8DA190E00E94497C62E0E9
:1095A0008EE10E94797C63E08FE10E94797C64E027
:1095B00080E20E94797CDD2009F450C08091C50CC6
:1095C000882309F44BC062EC7DE08EE89FE00E94A6
:1095D000EF5AAE014B5D5F4F61E070E08EE10E949B
:1095E0000F7CADA0B12CAE014B5D5F4F61E070E030
:1095F0008FE10E940F7CEDA0F12CAE014B5D5F4F1F
:1096000061E070E080E20E940F7C0DA110E04AE072
:1096100050E0B5018EE89FE00E94B75B65EC7BE00F
:109620008EE89FE00E94E05B4AE050E0B7018EE8E0
:109630009FE00E94B75B65EC7BE08EE89FE00E94B4
:10964000E05B4AE050E0B8018EE89FE00E94B75B23
:1096500062EC79E08EE89FE00E94C05B65E081E209
:109660000E94797CDD20B1F08091C50C882391F0B7
:109670006FEA7DE08EE89FE00E94EF5AAE014B5DFD
:109680005F4F61E070E081E20E940F7C8DA190E06D
:109690000E94497C66E082E20E94797CDD20B1F084
:1096A0008091C50C882391F067E97DE08EE89FE00A
:1096B0000E94EF5AAE014B5D5F4F61E070E082E2C5
:1096C0000E940F7C8DA190E00E94497C67E083E2BC
:1096D0000E94797CDD20B1F08091C50C882391F047
:1096E00061E87DE08EE89FE00E94EF5AAE014B5D9D
:1096F0005F4F61E070E083E20E940F7C8DA190E0FB
:109700000E94497C68E084E20E94797CDD20B1F00F
:109710008091C50C882391F069E67DE08EE89FE09A
:109720000E94EF5AAE014B5D5F4F61E070E084E252
:109730000E940F7C8DA190E00E94497C69E085E247
:109740000E94797CDD20B1F08091C50C882391F0D6
:109750006FE47DE08EE89FE00E94EF5AAE014B5D22
:109760005F4F61E070E085E20E940F7C8DA190E088
:109770000E94497C6AE086E20E94797CDD20B1F09B
:109780008091C50C882391F069E37DE08EE89FE02D
:109790000E94EF5AAE014B5D5F4F61E070E086E2E0
:1097A0000E940F7C8DA190E00E94497C6BE088E2D2
:1097B0000E94797CDD20B1F08091C50C882391F066
:1097C00060E27DE08EE89FE00E94EF5AAE014B5DC3
:1097D0005F4F61E070E088E20E940F7C8DA190E015
:1097E0000E94497C6CE089E20E94797CDD2009F4CA
:1097F00079C08091C50C882309F474C068E07DE0CD
:109800008EE89FE00E94EF5AAE014B5D5F4F61E032
:1098100070E089E20E940F7C8DA190E00E94497C5B
:1098200061EF7CE08EE89FE00E94EF5A66E070E016
:1098300087E20E945F7C90E00E94497C6AED7CE0B8
:109840008EE89FE00E94EF5A65E070E087E20E9498
:109850005F7C90E00E94497C63EC7CE08EE89FE0B6
:109860000E94EF5A64E070E087E20E945F7C90E023
:109870000E94497C6AEA7CE08EE89FE00E94EF5AF1
:1098800062E070E087E20E945F7C90E00E94497C89
:1098900061E97CE08EE89FE00E94EF5A61E070E0B1
:1098A00087E20E945F7C90E00E94497C68E77CE050
:1098B0008EE89FE00E94EF5A60E070E087E20E942D
:1098C0005F7C90E00E94497C67E67CE08EE89FE048
:1098D0000E94EF5A63E070E087E20E945F7C90E0B4
:1098E0000E94497C41E067E070E087E20E948E7C44
:1098F00041E063E070E087E20E948E7C41E063E03B
:1099000070E08AE20E948E7CDD2091F08091C50C8F
:10991000882371F06EE47CE08EE89FE00E94EF5AAD
:1099200063E070E08AE20E945F7C90E00E94497CE4
:1099300040E063E070E08AE20E948E7CDD2091F0DE
:109940008091C50C882371F064E37CE08EE89FE091
:109950000E94EF5A63E070E08AE20E945F7C90E030
:109960000E94497C41E062E070E08AE20E948E7CC5
:10997000DD2091F08091C50C882371F068E17CE0D6
:109980008EE89FE00E94EF5A62E070E08AE20E9457
:109990005F7C90E00E94497C40E062E070E08AE2F7
:1099A0000E948E7CDD2091F08091C50C882371F09F
:1099B0006BEF7BE08EE89FE00E94EF5A62E070E080
:1099C0008AE20E945F7C90E00E94497C41E061E075
:1099D00070E08AE20E948E7CDD2091F08091C50CBF
:1099E000882371F06FED7BE08EE89FE00E94EF5AD4
:1099F00061E070E08AE20E945F7C90E00E94497C16
:109A000040E061E070E08AE20E948E7CDD2091F00F
:109A10008091C50C882371F062EC7BE08EE89FE0BA
:109A20000E94EF5A61E070E08AE20E945F7C90E061
:109A30000E94497C41E060E070E08AE20E948E7CF6
:109A4000DD2091F08091C50C882371F066EA7BE0FF
:109A50008EE89FE00E94EF5A60E070E08AE20E9488
:109A60005F7C90E00E94497C40E060E070E08AE228
:109A70000E948E7CDD2091F08091C50C882371F0CE
:109A800069E87BE08EE89FE00E94EF5A60E070E0BA
:109A90008AE20E945F7C90E00E94497C41E066E09F
:109AA00070E087E20E948E7C41E065E070E087E232
:109AB0000E948E7C41E064E070E087E20E948E7C30
:109AC00040E062E070E087E20E948E7C40E061E06E
:109AD00070E087E20E948E7C40E060E070E087E208
:109AE0000E948E7CDD2009F475C08091C50C88230E
:109AF00009F470C061E77BE08EE89FE00E94EF5AB6
:109B000066E070E08BE20E945F7C90E00E94497CFE
:109B100063E57BE08EE89FE00E94EF5A65E070E02D
:109B20008BE20E945F7C90E00E94497C65E37BE0D1
:109B30008EE89FE00E94EF5A64E070E08BE20E94A2
:109B40005F7C90E00E94497C6CE17BE08EE89FE0C6
:109B50000E94EF5A62E070E08BE20E945F7C90E02E
:109B60000E94497C63E07BE08EE89FE00E94EF5A10
:109B700061E070E08BE20E945F7C90E00E94497C93
:109B80006AEE7AE08EE89FE00E94EF5A60E070E0B3
:109B90008BE20E945F7C90E00E94497C67ED7AE056
:109BA0008EE89FE00E94EF5A63E070E08BE20E9433
:109BB0005F7C90E00E94497C62EC7AE08EE89FE056
:109BC0000E94EF5A64E070E08CE20E945F7C90E0BB
:109BD0000E94497C40E064E070E08CE20E948E7C50
:109BE000AE014B5D5F4F61E070E08CE20E940F7C44
:109BF0006DA1607F66608CE20E94797CDD2009F4B3
:109C000065C08091C50C882309F460C06EEA7AE0D3
:109C10008EE89FE00E94EF5AAE014B5D5F4F61E01E
:109C200070E08CE20E940F7C6DA16F7070E0665056
:109C30007109072E000C880B990B0E94C8B29B017A
:109C4000AC0160E070E080E090E40E94C0B620E0EB
:109C500030E048EC50E40E9427B30E94BE7C67E9E4
:109C60007AE08EE89FE00E94EF5AAE014B5D5F4FB5
:109C700061E070E080E30E940F7C4DA150E060E065
:109C800070E02AE08EE89FE00E94285B8EE89FE06B
:109C90000E94BD5B6FE77AE08EE89FE00E94EF5A7A
:109CA00061E070E080E30E945F7C90E00E94497C6C
:109CB00066E67AE08EE89FE00E94EF5A61E070E08D
:109CC0008FE20E945F7C90E00E94497C41E061E06D
:109CD00070E08FE20E948E7CDD2091F08091C50CB7
:109CE000882371F06EE47AE08EE89FE00E94EF5ADC
:109CF00061E070E08EE20E945F7C90E00E94497C0F
:109D000041E061E070E08EE20E948E7C40E067E01E
:109D100070E081E30E948E7CDD2009F455C08091C3
:109D2000C50C882309F450C06BE37AE08EE89FE00D
:109D30000E94EF5A67E070E081E30E945F7C90E050
:109D40000E94497C6FE279E08EE89FE00E94E05B30
:109D5000AE014B5D5F4F61E070E080E00E940F7CE0
:109D60008DA10E94358D62EC79E08EE89FE00E9423
:109D7000C05B0DE110E06BE579E08EE89FE00E94AA
:109D8000E05B40E150E0B8018EE89FE00E94B75BE5
:109D900063E379E08EE89FE00E94E05BAE014B5DFB
:109DA0005F4F61E070E0802F0E940F7C8DA10E94C8
:109DB000358D62EC79E08EE89FE00E94C05B0F5F1A
:109DC0001F4F0A331105B9F6A9960FB6F894DEBFF6
:109DD0000FBECDBFDF91CF911F910F91FF90EF90FC
:109DE000DF90BF90AF909F908F907F906F905F902B
:109DF0004F900895DC0180E0615090F09D9198278C
:109E0000E92FEF70F0E0EE59F04F249192959F709A
:109E1000E92FF0E0EE58F04FE4918E2F8227ECCF3F
:109E200008950F931F93CF93DF938C01EB0188E28A
:109E3000FB0111928A95E9F74BE050E068EB79E07D
:109E4000CE010E9434BA1B8681E090E0A0E0B0E031
:109E50008C879D87AE87BF87F80185899689A789FA
:109E6000B08D888B998BAA8BBB8B82E090E0A0E0B1
:109E7000B0E08C8B9D8BAE8BBF8B1CA21DA21EA253
:109E80001FA280E090E0A8E4B4E4888F998FAA8FA5
:109E9000BB8F80E090E0A8E4B4EC8C8F9D8FAE8FF8
:109EA000BF8F8DEC9CECACE4BEE388A399A3AAA37E
:109EB000BBA3DF91CF911F910F9108954F925F92B5
:109EC0006F927F928F929F92AF92BF92CF92DF92CA
:109ED000EF92FF920F931F93CF93DF938C01EB01CF
:109EE00084E2FB0111928A95E9F78EE10E94966562
:109EF00083E090E00E9491650E948F6566E08EE1AC
:109F00000E94796A80916B0D90E020916C0D821B0C
:109F1000910986309105ECF38BE290E10E94B48BBD
:109F2000882E8BE290E10E94B48B982E8BE290E118
:109F30000E94B48B682E8BE290E10E94B48B782E45
:109F40008BE290E10E94B48B482E8BE290E10E945C
:109F5000B48B582EB82CA12CB5016929072E000C02
:109F6000880B990B0E94C8B24B015C01F801658314
:109F7000768387839087D42CC12CB6016529072E60
:109F8000000C880B990B0E94C8B2F8016187728798
:109F900083879487F62CE12CB7016729072E000CE4
:109FA000880B990B0E94C8B2F8016587768787876E
:109FB000908B118A128A138A148A84E290E0A0E0BE
:109FC000B0E088839983AA83BB8385899689A78912
:109FD000B08D8C839D83AE83BF8382E090E0A0E050
:109FE000B0E088879987AA87BB87188A198A1A8A56
:109FF0001B8AC0904E02D0904F02E0905002F09029
:10A000005102A7019601C501B4010E9418B520E0D4
:10A0100030E048EC52E40E9427B36C8B7D8B8E8B32
:10A020009F8BA7019601F8016185728583859485D0
:10A030000E9418B520E030E048EC52E40E9427B3BB
:10A04000688F798F8A8F9B8F20914A0230914B02C3
:10A0500040914C0250914D02F801658576858785C7
:10A0600090890E9418B520E030E048EC52E40E944C
:10A0700027B36C8F7D8F8E8F9F8F81E0DF91CF9183
:10A080001F910F91FF90EF90DF90CF90BF90AF9016
:10A090009F908F907F906F905F904F900895862F44
:10A0A0000C944B5D90E0FC013197E231F10508F032
:10A0B0004EC08827E855FF4F8F4F0C94A0B7809172
:10A0C00080008F7703C0809180008F7D8093800017
:10A0D000089580918000877FF9CF84B58F7702C083
:10A0E00084B58F7D84BD08958091B0008F7703C0C3
:10A0F0008091B0008F7D8093B00008958091900092
:10A100008F7707C0809190008F7D03C08091900071
:10A11000877F8093900008958091A0008F7707C07B
:10A120008091A0008F7D03C08091A000877F8093E5
:10A13000A0000895809120018F7707C080912001B1
:10A140008F7D03C080912001877F80932001089537
:10A150001F93CF93DF93282F30E0F901E45AFF4E8D
:10A160008491F901EA5EFF4ED491F901E053F04F7A
:10A17000C491CC23C1F0162F811194DFEC2FF0E0B5
:10A18000EE0FFF1FE456F04FA591B4918FB7F894EE
:10A19000111105C09C91ED2FE095E92302C0EC91CF
:10A1A000ED2BEC938FBFDF91CF911F910895862FF8
:10A1B000642FCECFCF93DF9390E0FC01EA5EFF4E99
:10A1C0002491FC01E053F04F8491882361F190E0E9
:10A1D000880F991FFC01EE57F04FC591D491FC01F7
:10A1E000E456F04FA591B491611109C09FB7F8945E
:10A1F0008881209582238883EC912E230BC06230C6
:10A2000061F49FB7F8943881822F809583238883E7
:10A21000EC912E2B2C939FBF06C08FB7F894E8814A
:10A220002E2B28838FBFDF91CF910895862F642F27
:10A23000C1CF863308F0865390917B00282F287079
:10A24000977F922B90937B0087702091520290E42D
:10A25000299F90011124822B80937C0080917A00A9
:10A26000806480937A0080917A0086FDFCCF809193
:10A2700078002091790090E0922B08953FB7F894F0
:10A280008091F50C9091F60CA091F70CB091F80C20
:10A2900026B5A89B05C02F3F19F00196A11DB11D41
:10A2A0003FBFBA2FA92F982F8827820F911DA11D7C
:10A2B000B11DBC01CD0142E0660F771F881F991FB9
:10A2C0004A95D1F708958F929F92AF92BF92CF9205
:10A2D000DF92EF92FF926B017C01D0DF4B015C01BA
:10A2E000C114D104E104F104E9F0C8DFDC01CB01C1
:10A2F00088199909AA09BB09883E9340A105B105AF
:10A3000078F321E0C21AD108E108F10888EE880E3E
:10A3100083E0981EA11CB11CC114D104E104F10416
:10A3200021F7DECFFF90EF90DF90CF90BF90AF90FE
:10A330009F908F9008952FB7F8946091F10C7091D1
:10A34000F20C8091F30C9091F40C2FBF08951F92A2
:10A350000F920FB60F9211242F933F938F939F93D9
:10A36000AF93BF938091F10C9091F20CA091F30CFC
:10A37000B091F40C3091F00C23E0230F2D3720F432
:10A380000196A11DB11D05C026E8230F0296A11D4F
:10A39000B11D2093F00C8093F10C9093F20CA093DC
:10A3A000F30CB093F40C8091F50C9091F60CA09105
:10A3B000F70CB091F80C0196A11DB11D8093F50C1E
:10A3C0009093F60CA093F70CB093F80CBF91AF915B
:10A3D0009F918F913F912F910F900FBE0F901F90E3
:10A3E0001895DF92EF92FF920F931F93CF93DF9315
:10A3F0007C018B01D42EDC011696ED91FC91179710
:10A40000138615861486DF011B9633961E92AE17AF
:10A41000BF07E1F7C0E0B801D70116968D919C9176
:10A4200017970E946C7ED82F811102C0D0E00DC01A
:10A43000CD1107C067E0C801DDDCF80197818917FD
:10A4400021F0CF5FDC1690F3E6CF8D2FDF91CF9117
:10A450001F910F91FF90EF90DF900895FC01908184
:10A460000180F281E02DF8948181892B8183228102
:10A47000892F809528232283A7E0B0E01197F1F778
:10A48000218182238183A3E2B0E01197F1F78081DB
:10A490007894EFECF0E03197F1F7982381E009F43C
:10A4A00080E00895FC0190810180F281E02D892FE8
:10A4B000809560FF12C0F89422818223828381817B
:10A4C000892B8183A3E2B0E01197F1F78281982B69
:10A4D0009283789487ED90E011C0F89422818223D2
:10A4E00082838181892B8183AFEFB0E01197F1F7EF
:10A4F0008281982B928378948FE090E00197F1F716
:10A500000895CF92DF92EF92FF920F931F93CF9314
:10A51000DF931F92CDB7DEB76C01E62E08E010E0A6
:10A52000FF24F39461E08F2D8E2109F460E0C601D1
:10A530004983B8DFFF0C015011094981011511054C
:10A5400089F7411115C0F894D6011196ED91FC914F
:10A55000129791818C918095892381831196ED9139
:10A56000FC91129792818C918095892382837894B3
:10A570000F90DF91CF911F910F91FF90EF90DF909F
:10A58000CF900895CF92DF92EF92FF920F931F9397
:10A59000CF93DF931F92CDB7DEB78C01F62E40E04C
:10A5A00065E57983AEDFCF2C7981D72E760188E0FF
:10A5B000E80EF11CF60161916F0140E0C801A1DFD6
:10A5C000CE14DF04B9F70F90DF91CF911F910F9157
:10A5D000FF90EF90DF90CF900895FC019081018073
:10A5E000F281E02DF8948181292F209582238183A7
:10A5F00078948DE743E050E0815021F1DA01119722
:10A60000F1F730813923C1F3F89482818223828368
:10A610008181892B81837894ABE7B7E01197F1F7BB
:10A62000F894818128232183A3E1B1E01197F1F708
:10A630008081982381E009F080E07894E3E6F6E0F9
:10A640003197F1F708958F929F92AF92BF92CF9278
:10A65000DF92EF92FF920F931F93CF93DF93EC0162
:10A660008E819F81BADF40E06CEC8E819F8149DF53
:10A67000488164E48E819F8144DF8A81882309F4C4
:10A680003EC0E981E950E33040F4F0E0EE0FFF1FF7
:10A69000E75CFA4F0081118102C00EEE12E08B815F
:10A6A0008823E1F08881811119C045DE4B015C01EE
:10A6B0006801110FEE08FF088E819F81CFDE813087
:10A6C000F1F039DEDC01CB018C199D09AE09BF091F
:10A6D00088159905AA05BB0578F311C0B801110FBB
:10A6E000880B990BDF91CF911F910F91FF90EF9005
:10A6F000DF90CF90BF90AF909F908F90E4CDDF918F
:10A70000CF911F910F91FF90EF90DF90CF90BF906E
:10A71000AF909F908F9008954F925F926F927F922B
:10A720008F929F92AF92BF92CF92DF92EF92FF9261
:10A730000F931F93CF93DF931F921F92CDB7DEB776
:10A740002C018A01FC018681978169837A8345DF28
:10A7500069817A818823A1F1F2018681978112DFD4
:10A7600040E06EEBF20186819781CBDE78014801F3
:10A77000F9E08F0E911CF2016680778088E0A82EA8
:10A78000B12CCC24C394D12CC30168DE8111DC2808
:10A79000CC0CF1E0AF1AB108B9F7F701D1927F0103
:10A7A000E815F90541F7F2018681978116DF8130BE
:10A7B00039F468E0C8011EDB91E0F80120858213BE
:10A7C00090E0892F0F900F90DF91CF911F910F9103
:10A7D000FF90EF90DF90CF90BF90AF909F908F90C1
:10A7E0007F906F905F904F900895CF93DF93CDB798
:10A7F000DEB729970FB6F894DEBF0FBECDBFAE010E
:10A800004F5F5F4F89DF882389F08D818F3361F03F
:10A8100020F48F3159F489E00CC08F3519F08F374F
:10A8200039F004C08BE005C08AE003C080E001C0BD
:10A830008CE029960FB6F894DEBF0FBECDBFDF9136
:10A84000CF9108950F931F93CF93DF93CDB7DEB7CA
:10A8500061970FB6F894DEBF0FBECDBF8C01462FB7
:10A86000BE01665F7F4FBDDD811105C060E070E015
:10A870008EEF92EC4AC0AE014F5F5F4FBE01665F44
:10A880007F4FC80149DF882359F1698148E0649FFF
:10A89000B00111248A81282F30E0322F2227330F74
:10A8A000330F330F262B372B8A858031E1F46885EF
:10A8B00070E08F81AB01481B5109CA019695982F12
:10A8C0008827979587950E948DB760517109207FE1
:10A8D00053E0220F331F5A95E1F7620F731F04C034
:10A8E00060E874EE01C0B901613854EE75070CF4EC
:10A8F000BDCF072E000C880B990B0E94C8B220E038
:10A9000030E040E05CE30E9427B361960FB6F89414
:10A91000DEBF0FBECDBFDF91CF911F910F91089584
:10A92000EF92FF920F931F93CF93DF93CDB7DEB7D4
:10A9300028970FB6F894DEBF0FBECDBF8C01DC01A7
:10A940001696ED91FC911797138615861486DF01F4
:10A950001B9633961E92AE17BF07E1F7F8011482DB
:10A960001582EE24E394BE016F5F7F4FF80186816C
:10A9700097810E946C7E882309F469C067E0CE014C
:10A98000019638DA98858913EECFD8018C91811120
:10A9900021C016968D919C9117971FDEBE016F5FA7
:10A9A0007F4FF80186819781EDDD40E064EBD801AF
:10A9B00016968D919C911797A4DDF8018681978159
:10A9C0004DDDF82ED80116968D919C91179705DED6
:10A9D000FF20B1F1F801F18089818031A1F1BE0140
:10A9E0006F5F7F4FC80101DF8F1520F4D8011196EA
:10A9F0008C910AC08981803111F48CE005C0BE01C0
:10AA00006F5F7F4FC801F1DEF801818384818F5F22
:10AA100084838981883261F030F4803149F0823258
:10AA200009F0A1CF05C08B3319F0823409F09BCF18
:10AA3000D80115968C9115978F5F15968C9393CFAF
:10AA4000D801EC92C7CFBCE0BF1580F2D6CF2896D4
:10AA50000FB6F894DEBF0FBECDBFDF91CF911F912F
:10AA60000F91FF90EF9008950F931F93CF93DF9373
:10AA7000EC01162F60E0812F9DDB612F70E0FB0160
:10AA8000EA5EFF4EE491E883FB01E053F04FE4916E
:10AA9000F0E0EE0FFF1FEA54F04F859194919A83F6
:10AAA00089831B861D861C86FE013B968E010D5FE9
:10AAB0001F4F1292E017F107E1F7DF91CF911F913D
:10AAC0000F9108950F931F93CF93DF931F92CDB7EC
:10AAD000DEB78C01FC01848169830E949665F801D0
:10AAE00083856981862B90E00E9491650F90DF91AC
:10AAF000CF911F910F910C948F650F931F93CF935C
:10AB00008C01C62FDFDF6C2F6460C801DBDF6C2F88
:10AB10006B7FC801D7DF83EC90E00197F1F7CF910D
:10AB20001F910F9108950F931F93CF938C01C62F00
:10AB3000607F6160E2DF80E1C89FB0011124616045
:10AB4000C801DBDF81E090E0CF911F910F91089564
:10AB50000895CF92DF92EF92FF920F931F93CF93BE
:10AB6000DF936C017A018B01C0E0D0E0CE15DF05E8
:10AB700089F0D8016D918D01D601ED91FC91019084
:10AB8000F081E02DC6011995892B11F47E0102C0D8
:10AB90002196ECCFC701DF91CF911F910F91FF90CC
:10ABA000EF90DF90CF900895FC01A089B1898C913E
:10ABB000A689B78982FD0FC09C91818D8F5F8F73AD
:10ABC000228D821749F0218DDF01A20FB11D5D9604
:10ABD0009C93818F08958C910895FC01538D448D31
:10ABE000252F30E0842F90E0821B930B541710F038
:10ABF000CF96089501970895FC01918D828D981745
:10AC000061F0828DDF01A80FB11D5D968C91928D50
:10AC10009F5F9F73928F90E008958FEF9FEF08954D
:10AC2000FC01918D828D981731F0828DE80FF11D16
:10AC3000858D90E008958FEF9FEF0895FC01918D31
:10AC4000228D892F90E0805C9F4F821B91098F732A
:10AC50009927089587EB9DE0F1DF21E0892B09F426
:10AC600020E0822F089584E59EE0E8DF21E0892B33
:10AC700009F420E0822F089581EF9EE0DFDF21E0DC
:10AC8000892B09F420E0822F08958EE89FE0D6DF1B
:10AC900021E0892B09F420E0822F0895FC01848DA6
:10ACA000DF01A80FB11DA35ABF4F2C91848D90E0F6
:10ACB00001968F739927848FA689B7892C93A089D1
:10ACC000B1898C9180648C93938D848D981306C088
:10ACD0000288F389E02D80818F7D80830895EF9233
:10ACE000FF920F931F93CF93DF93EC0181E0888F46
:10ACF0009B8D8C8D981305C0E889F989808185FD2D
:10AD000023C0F62E0B8D10E00F5F1F4F0F7311271E
:10AD1000E02E8C8DE8120BC00FB607FCFACFE88945
:10AD2000F989808185FFF5CFCE01B8DFF2CF8B8D19
:10AD3000FE01E80FF11DE35AFF4FF0820B8FEA8905
:10AD4000FB898081806207C0EE89FF896083E88982
:10AD5000F98980818064808381E090E0DF91CF91E8
:10AD60001F910F91FF90EF900895CF93DF93EC0127
:10AD7000888D8823C1F0EA89FB89808185FD05C023
:10AD8000A889B9898C9186FD0EC00FB607FCF5CF56
:10AD9000808185FFF2CFA889B9898C9185FFEDCF9D
:10ADA000CE017CDFE8CFDF91CF91089580E090E085
:10ADB000892B19F06ADF811116C080E090E0892BA1
:10ADC00019F05ADF811112C080E090E0892B19F050
:10ADD0004ADF81110EC080E090E0892B79F03ADFE4
:10ADE00081110AC008950E940000E7CF0E94000070
:10ADF000EBCF0E940000EFCF0C94000008950E945A
:10AE0000F0B9CF93DF93EC0188819981009711F01D
:10AE10000E9474B8198218821D821C821B821A82B9
:10AE2000DF91CF9108950F931F93CF93DF93EC01A0
:10AE300088819981009729F02A813B81261737075D
:10AE400088F48B016F5F7F4F0E940CB9009761F00F
:10AE5000998388831B830A832C813D81232B11F4E2
:10AE6000FC01108281E001C080E0DF91CF911F9151
:10AE70000F910895EF92FF920F931F93CF93DF935B
:10AE8000FC01248135816115710511F480E018C041
:10AE900041155105A1F07B01EC018A01020F131F3E
:10AEA000B801C1DF882391F3288139818C819D818C
:10AEB000B701820F931F0E941FBA1D830C8381E08C
:10AEC000DF91CF911F910F91FF90EF900895EF9236
:10AED000FF920F931F93CF93DF93EC017B018A01C5
:10AEE000BA01A1DF811103C0CE018BDF07C01D8332
:10AEF0000C83B701888199810E941FBACE01DF912E
:10AF0000CF911F910F91FF90EF900895FC018081E8
:10AF10009181009711F00C94EEAD60E070E0CB01F0
:10AF20000895FC0180819181009711F00C940EAE80
:10AF300060E070E0CB010895AF92BF92CF92DF92B4
:10AF4000EF92FF920F931F93CF93DF93DC01CD908D
:10AF5000DC901197C114D10409F442C01496CD912C
:10AF6000DC9115972097E1F18C0156017501BFEF37
:10AF7000AB1ABB0AF7018081082E000C990B0E94C6
:10AF800092B2892B99F72197CC0DDD1D8881082E6F
:10AF9000000C990B0E9492B2892B91F4AE014F5F85
:10AFA0005F4F4E195F09D80115965C934E93149725
:10AFB000CE14DF0450F4B701C6010E940DBA05C0DB
:10AFC000CE15DF0558F32197E1CFD801ED91FC9123
:10AFD000119714968D919C911597E80FF91F108287
:10AFE000DF91CF911F910F91FF90EF90DF90CF9065
:10AFF000BF90AF900895AF92BF92CF92DF92EF9241
:10B00000FF920F931F93CF93DF93FC01248135812F
:10B01000FB01448155818901041B150B4115510524
:10B0200051F12115310539F12417350720F10217A7
:10B03000130718F08901015011097B01FC01A08060
:10B04000B180C501DFEFCFEF6501C00ED11EC8167C
:10B05000D906A0F0F701608171810E9443BA009780
:10B0600069F09C012A193B090217130710F0D22F2F
:10B07000C32F0196ECCF8FEF9FEF02C08D2F9C2F37
:10B08000DF91CF911F910F91FF90EF90DF90CF90C4
:10B09000BF90AF900895CF93DF93FC012481358159
:10B0A000232B71F0FB01DC01CD91DC91608171817A
:10B0B000CE010E9443BA009719F08C1B9D0B02C071
:10B0C0008FEF9FEFDF91CF910895FC0124813581AF
:10B0D0006217730748F480819181009729F0FC0181
:10B0E000E60FF71F8081089580E00895FB014481F9
:10B0F0005581FC01248135812417350778F0808142
:10B100009181009759F0FB01608171816115710592
:10B1100029F00E9426BA21E0892B09F020E0822F35
:10B120000895CF93DF93EC016115710559F0FB0190
:10B1300001900020E9F73197AF01461B570B9ADECB
:10B14000811102C0CE015DDECE01DF91CF91089565
:10B15000CF93DF93EC01FB014481558160817181C4
:10B1600089DE811102C0CE014CDECE01DF91CF918C
:10B170000895EF92FF920F931F93CF93DF93611582
:10B18000710511F480E01DC08B01EC01CB010E9420
:10B190003BAE0097A9F02C813D817C01E20EF31EAD
:10B1A000B701CE0140DE882369F3288139818C8183
:10B1B0009D81B801820F931F0E9434AEFD82EC8204
:10B1C00081E0DF91CF911F910F91FF90EF90089553
:10B1D000CF93DF931F921F92CDB7DEB769831A8298
:10B1E00041E050E0BE016F5F7F4F44DE0F900F9053
:10B1F000DF91CF9108956115710549F0FB01019030
:10B200000020E9F73197AF01461B570B33CE80E0A2
:10B210000895FB0144815581608171812BCEEF92AD
:10B22000FF920F931F93CF93DF93EC018B01611576
:10B23000710549F0CB010E943BAE7C01BC01CE01FF
:10B24000F2DD811103C0CE01DCDD07C0FD82EC829E
:10B25000B801888199810E9434AECE01DF91CF91EF
:10B260001F910F91FF90EF900895CF93DF93EC0122
:10B270006115710551F0FB0101900020E9F731974C
:10B28000AF01461B570B23DE01C0BBDDCE01DF91B2
:10B29000CF910895CF93DF93EC01FB0186179707B9
:10B2A00051F0608171816115710521F044815581F2
:10B2B0000EDE01C0A6DDCE01DF91CF9108950F9380
:10B2C0001F93CF93DF938C01EB01FC01808191816F
:10B2D0000097B1F0688179816115710579F042813B
:10B2E00053812C813D814217530740F00E941FBAC1
:10B2F0008C819D81F8019583848313C00E9474B86A
:10B3000088819981F801918380838A819B819383CD
:10B3100082838C819D8195838483198218821B820C
:10B320001A821D821C82DF91CF911F910F91089587
:10B33000FC01808191810C9474B8EF92FF920F937D
:10B340001F93CF93DF93CDB7DEB7A1970FB6F894D5
:10B35000DEBF0FBECDBF7C01CB01BA01F701118268
:10B360001082138212821582148242E0420F8E01F3
:10B370000F5F1F4F0E94CFADBC01C70176DFA196C2
:10B380000FB6F894DEBF0FBECDBFDF91CF911F91F6
:10B390000F91FF90EF900895EF92FF920F931F93FC
:10B3A000CF93DF93CDB7DEB7A1970FB6F894DEBF8A
:10B3B0000FBECDBF7C01CB01BA01F7011182108213
:10B3C000138212821582148242E0420F8E010F5FB7
:10B3D0001F4F0E94CFADBC01C70147DFA1960FB63A
:10B3E000F894DEBF0FBECDBFDF91CF911F910F91BB
:10B3F000FF90EF9008950F931F93CF93DF93CDB7F6
:10B40000DEB7A2970FB6F894DEBF0FBECDBF8C019A
:10B41000CB01BA01F80111821082138212821582C7
:10B42000148230E0AE014F5F5F4F0E9458AEBE0104
:10B430006F5F7F4FC80119DFA2960FB6F894DEBF89
:10B440000FBECDBFDF91CF911F910F9108950F9344
:10B450001F93CF93DF93CDB7DEB762970FB6F89403
:10B46000DEBF0FBECDBF8C01CB01F801118210826F
:10B47000138212821582148250E0BE016F5F7F4FEB
:10B480000E9444AEBE016F5F7F4FC801EEDE629640
:10B490000FB6F894DEBF0FBECDBFDF91CF911F91E5
:10B4A0000F910895CF93DF931F921F92CDB7DEB710
:10B4B000FC01118210821382128215821482698328
:10B4C0001A82BE016F5F7F4FD0DE0F900F90DF9129
:10B4D000CF910895FC01118210821382128215828D
:10B4E0001482EDCEFC011182108213821282158229
:10B4F000148295CEFC011182108213821282158271
:10B500001482C8CEFC01118210821382128215822D
:10B5100014826115710549F0FB0101900020E9F7E3
:10B520003197AF01461B570BD2CC0895BF92CF92F3
:10B53000DF92EF92FF920F931F93CF93DF937C01E3
:10B540006B018A01E9012417350720F4812F890155
:10B55000C42FD82F62EC79E0C701D4DFD60114964E
:10B560008D919C91159708171907C8F48C179D07A2
:10B5700008F4EC01D601ED91FC911197EC0FFD1F41
:10B58000B08010824D915C91BA01600F711FC701AC
:10B590006CDED601ED91FC91EC0FFD1FB082C7016E
:10B5A000DF91CF911F910F91FF90EF90DF90CF909F
:10B5B000BF900895DC01ED91FC910190F081E02DA8
:10B5C0001994DC01ED91FC91DB0114964D915C9195
:10B5D00015976D917C910280F381E02D1994EF9283
:10B5E000FF920F931F93CF93DF938C017B01C0E0F9
:10B5F000D0E0F701EC0FFD1F6491662361F0D801E4
:10B60000ED91FC910190F081E02DC8011995892BF5
:10B6100011F02196EECFCE01DF91CF911F910F91C6
:10B62000FF90EF9008956115710579F0FB0101908D
:10B630000020E9F73197AF01461B570BDC01ED9174
:10B64000FC910280F381E02D199480E090E0089550
:10B650004F925F926F927F92EF92FF920F931F93A0
:10B66000CF93DF93CDB7DEB7A1970FB6F894DEBFC7
:10B670000FBECDBF7C01FA01CB0119A2223008F424
:10B680002AE08E010F5D1F4F422E512C612C712C30
:10B69000BF01A30192010E9420B4F901CA01015027
:10B6A00011096A3014F4605D01C0695CD8016C93C3
:10B6B000232B242B252B61F7B801C701B4DFA196FA
:10B6C0000FB6F894DEBF0FBECDBFDF91CF911F91B3
:10B6D0000F91FF90EF907F906F905F904F90089543
:10B6E000CF92DF92EF92FF920F931F93CF93DF934E
:10B6F000EC016A017B012115310579F4E881F981BA
:10B700000190F081E02D642FDF91CF911F910F9177
:10B71000FF90EF90DF90CF9019942A303105D9F443
:10B7200077FF18C06DE246DF8C0144275527BA0128
:10B730004C195D096E097F092AE0CE0189DF800F6F
:10B74000911FDF91CF911F910F91FF90EF90DF90AC
:10B75000CF9008952AE0B701A601CE01DF91CF91E5
:10B760001F910F91FF90EF90DF90CF9071CF9A01D2
:10B77000AB01770F660B770BB3CF60EC79E053CF5B
:10B780000F931F93CF93DF93EC014DDF8C01CE011C
:10B79000F4DF800F911FDF91CF911F910F910895DA
:10B7A0000F931F93CF93DF93EC010BDF8C01CE013E
:10B7B000E4DF800F911FDF91CF911F910F910895CA
:10B7C00032CF1F920F920FB60F9211240BB60F9229
:10B7D0002F933F934F935F936F937F938F939F9399
:10B7E000AF93BF93EF93FF9387EB9DE057DAFF9101
:10B7F000EF91BF91AF919F918F917F916F915F91E9
:10B800004F913F912F910F900BBE0F900FBE0F9055
:10B810001F9018951F920F920FB60F9211240BB61E
:10B820000F922F933F934F935F936F937F938F93D9
:10B830009F93AF93BF93EF93FF9387EB9DE0B4D9B2
:10B84000FF91EF91BF91AF919F918F917F916F91F8
:10B850005F914F913F912F910F900BBE0F900FBEB4
:10B860000F901F9018951F920F920FB60F921124F0
:10B870000BB60F922F933F934F935F936F937F93EA
:10B880008F939F93AF93BF93EF93FF9384E59EE0D5
:10B8900005DAFF91EF91BF91AF919F918F917F91C9
:10B8A0006F915F914F913F912F910F900BBE0F9031
:10B8B0000FBE0F901F9018951F920F920FB60F9208
:10B8C00011240BB60F922F933F934F935F936F9377
:10B8D0007F938F939F93AF93BF93EF93FF9384E5F1
:10B8E0009EE062D9FF91EF91BF91AF919F918F91AF
:10B8F0007F916F915F914F913F912F910F900BBE70
:10B900000F900FBE0F901F9018951F920F920FB6B9
:10B910000F9211240BB60F922F933F934F935F9387
:10B920006F937F938F939F93AF93BF93EF93FF9307
:10B9300081EF9EE0B3D9FF91EF91BF91AF919F91BD
:10B940008F917F916F915F914F913F912F910F90C8
:10B950000BBE0F900FBE0F901F9018951F920F9265
:10B960000FB60F9211240BB60F922F933F934F9364
:10B970005F936F937F938F939F93AF93BF93EF9357
:10B98000FF9381EF9EE010D9FF91EF91BF91AF91AE
:10B990009F918F917F916F915F914F913F912F91E7
:10B9A0000F900BBE0F900FBE0F901F9018951F9217
:10B9B0000F920FB60F9211240BB60F922F933F9355
:10B9C0004F935F936F937F938F939F93AF93BF93A7
:10B9D000EF93FF938EE89FE061D9FF91EF91BF91C4
:10B9E000AF919F918F917F916F915F914F913F9117
:10B9F0002F910F900BBE0F900FBE0F901F901895B8
:10BA00001F920F920FB60F9211240BB60F922F9325
:10BA10003F934F935F936F937F938F939F93AF93D6
:10BA2000BF93EF93FF938EE89FE0BED8FF91EF9115
:10BA3000BF91AF919F918F917F916F915F914F9146
:10BA40003F912F910F900BBE0F900FBE0F901F9044
:10BA50001895CF93DF93EC01E881F9810680F78197
:10BA6000E02D1995EA89FB8980818F7E8083EA89A0
:10BA7000FB898081877F8083EA89FB8980818F773A
:10BA80008083EA89FB8980818F7D80838A8D898F7D
:10BA9000DF91CF910895CF93DF93282F30E0F90104
:10BAA000E45AFF4E8491F901EA5EFF4ED491F90108
:10BAB000E053F04FC491CC2391F081110E94525079
:10BAC000EC2FF0E0EE0FFF1FEA54F04FA591B49178
:10BAD000EC91ED2381E090E021F480E002C080E071
:10BAE00090E0DF91CF910895CF93DF93CDB7DEB78C
:10BAF0002C970FB6F894DEBF0FBECDBF81309105F5
:10BB0000A1F5909381118093801163E572E1CE01DC
:10BB10000196E8DCCE0101960E947238CE010196B2
:10BB200007DC62EF77E0CE010196ECDC6EE873E1B2
:10BB3000CE0101960DDBBC01CE010796DBDC48ECA3
:10BB400050E06FEF7FEFCE0107960E94D133CE0118
:10BB50000796EEDBCE010196EBDB87EB9DE079DF0C
:10BB600040E052EC61E070E066C0009769F5109229
:10BB700081111092801165E472E1CE010196B2DC70
:10BB8000CE0101960E947238CE010196D1DB6EEE95
:10BB900077E0CE010196B6DC6EE873E1CE01019646
:10BBA000D7DABC01CE010796A5DC48EC50E06FEF78
:10BBB0007FEFCE0107960E94D133CE010796B8DB06
:10BBC000CE010196B5DB61C08230910509F05DC000
:10BBD000909381118093801164E372E1CE0101960C
:10BBE00081DCCE0101960E947238CE010196A0DB65
:10BBF00068EF77E0CE01019685DC6EE873E1CE0157
:10BC00000196A6DABC01CE01079674DC48EC50E040
:10BC10006FEF7FEFCE0107960E94D133CE010796DA
:10BC200087DBCE01019684DB87EB9DE012DF40E8E5
:10BC300055E260E070E087EB9DE00E94D43D1092F9
:10BC4000EF0C1092EE0C80E090E00E9421696DEF05
:10BC500077E0CE01019656DC68E873E1CE010196EB
:10BC600077DABC01CE01079645DC40ED57E06FEF77
:10BC70007FEFCE0107960E949832CE01079658DBDF
:10BC8000CE01019655DB81E001C080E02C960FB615
:10BC9000F894DEBF0FBECDBFDF91CF9108950F9313
:10BCA0001F93CF93DF93CDB7DEB72C970FB6F894E1
:10BCB000DEBF0FBECDBF8C0162EC79E087EB92E175
:10BCC000D4DA0830110509F0C4C06AE272E1CE018D
:10BCD000019608DC44E650E06FEF7FEFCE0101965D
:10BCE0000E94D133CE01019623DB6EE172E1CE01D9
:10BCF0000196F8DB44E650E060E070E0CE0101968A
:10BD00000E949832CE01019613DB87EB9DE02DD87F
:10BD10004CE251E061E070E0CE0101960E94D87FD4
:10BD20008091C50C8823A9F063EC79E0CE010796D9
:10BD3000E9DBBE016F5F7F4FCE01079609DA66EC43
:10BD400079E0EFD9BC018EE89FE02ADDCE010796AD
:10BD5000EFDA6DE078E0CE010796D4DBBE01695FD3
:10BD60007F4FCE010196C2D9182FCE010796E0DA97
:10BD7000112309F46BC068EC79E087EB92E175DA86
:10BD800088E090E09093BE0C8093BD0C0E94473EEB
:10BD9000182F61E172E1CE010796A4DB44E650E082
:10BDA00060E070E0CE0107960E949832CE010796BF
:10BDB000BFDA87EB9DE00E94B55648E552E061E0AE
:10BDC00070E0CE0107960E94D87FBE01695F7F4F69
:10BDD000CE01019674DACE010796AADA8091C50CDD
:10BDE0008823A9F063EC79E0CE0107968BDBBE01D6
:10BDF0006F5F7F4FCE010796ABD966EC79E091D9A2
:10BE0000BC018EE89FE0CCDCCE01079691DA68EDAC
:10BE10007BE0CE01079676DBBE01695F7F4FCE01E6
:10BE2000019664D9082FCE01079682DA002371F0BB
:10BE30006DEC79E087EB92E118DA0E94473E8823A7
:10BE400029F0112319F064E072E1E2C06DEF71E1B5
:10BE5000DFC0093F2FEF120709F0EEC063EF71E179
:10BE6000CE0101963FDB44E650E06FEF7FEFCE015D
:10BE700001960E94D133CE0101965ADA65EE71E146
:10BE8000CE0101962FDB44E650E060E070E0CE0189
:10BE900001960E949832CE0101964ADA87EB9DE026
:10BEA0000E94B5564CE251E064E070E0CE0101968C
:10BEB0000E94D87F8091C50C8823A9F063EC79E0BB
:10BEC000CE0107961FDBBE016F5F7F4FCE01079645
:10BED0003FD966EC79E025D9BC018EE89FE060DCB3
:10BEE000CE01079625DA60E070E0CE010196EDD82C
:10BEF000082E000C990BC0970A9708F087C063EDD5
:10BF000079E0CE010796FEDABE016F5F7F4FCE016A
:10BF100007961ED9BC0187EB92E1BCD9CE010796EA
:10BF200007DA89EF9FEF9093BE0C8093BD0C0E94BF
:10BF3000473E182F67ED71E1CE010796D3DA44E64C
:10BF400050E060E070E0CE0107960E949832CE018A
:10BF50000796EED987EB9DE00E94B55648E552E082
:10BF600065E070E0CE0107960E94D87FBE01695F50
:10BF70007F4FCE010196A3D9CE010796D9D98091E2
:10BF8000C50C8823A9F063EC79E0CE010796BADAF4
:10BF9000BE016F5F7F4FCE010796DAD866EC79E07D
:10BFA000C0D8BC018EE89FE0FBDBCE010796C0D96C
:10BFB00060E070E0CE01019688D8282F880F330BFF
:10BFC000205331092A30310508F568ED79E0CE01BA
:10BFD000079698DABE016F5F7F4FCE010796B8D8FB
:10BFE000BC0187EB92E156D9CE010796A1D989EF22
:10BFF0009FEF9093BE0C8093BD0C0E94473E882318
:10C0000029F0112319F06AEC71E102C063EC71E1CF
:10C01000CE01079667DA44E650E060E070E0CE01BA
:10C0200007960E949832CE01079682D962EC79E099
:10C0300087EB92E11AD9FEC069EB71E1CE0101965E
:10C0400051DA44E650E06FEF7FEFCE0101960E9497
:10C05000D133CE0101966CD962EC79E087EB92E1A5
:10C0600004D9053F8FEF180741F467EB78E087EBC1
:10C0700092E1FBD86FEA71E123C0063F2FEF120770
:10C0800041F46BEA78E087EB92E1EFD865EA71E181
:10C0900017C0013F8FEF180741F465EC78E087EB9C
:10C0A00092E1E3D866E971E10BC0023F2FEF12077E
:10C0B000A9F46DED79E087EB92E1D7D866E871E1FC
:10C0C000CE0101960FDA44E650E06FEF7FEFCE012C
:10C0D00001960E949832CE010196B0C0023011053F
:10C0E00009F074C06AE771E1CE010196FBD944E61C
:10C0F00050E06FEF7FEFCE0101960E94D133CE0169
:10C10000019616D96AE671E1CE010196EBD944E6B3
:10C1100050E06FEF7FEFCE0101960E949832CE0182
:10C12000019606D944EF51E066E070E0CE01019639
:10C130000E94D87FBE016F5F7F4F87EB92E1BFD82F
:10C14000CE010196F5D88091BB129091BC12059753
:10C1500008F476C060E070E087EB92E10E946558D9
:10C16000082E000C990BC0970A9708F069C087EB5E
:10C1700092E10E949157613523EC72078105910588
:10C180000CF45EC00E94C8B220E030E048EC52E4FB
:10C190000E9418B5AB01BC0122E0CE010796CDD8B4
:10C1A00065E778E0CE010196ADD9BE01695F7F4FAA
:10C1B000CE0101960E94A858BC0187EB92E16AD893
:10C1C000CE010196B5D8CE01079638C063E571E17E
:10C1D000CE01019687D944E650E06FEF7FEFCE01A4
:10C1E00001960E949832CE010196A2D862EC79E0C5
:10C1F00087EB92E13AD80B3E8FEF180709F457C04E
:10C200008091BB129091BC12892B81F550C068ECD3
:10C2100070E080E090E00E9463516DE371E1CE0137
:10C22000019660D944EF51E06FEF7FEFCE010196A8
:10C230000E949832CE0101967BD839C079D8E0CFE0
:10C240006CE571E1CE0101964DD948EE53E06FEFF8
:10C250007FEFCE0101960E949832CE01019668D8F8
:10C2600062EC79E087EB92E100D8CACF0E94473EAA
:10C27000882369F268EC70E080E090E00E946351EE
:10C2800069E471E1CE0101962DD944EF51E06FEFE1
:10C290007FEFCE0101960E949832CE01019648D8D8
:10C2A0001093BE0C0093BD0CC8010E94D60A2C96B8
:10C2B0000FB6F894DEBF0FBECDBFDF91CF911F91B7
:10C2C0000F910895BF92CF92DF92EF92FF920F935A
:10C2D0001F93CF93DF93CDB7DEB762970FB6F89475
:10C2E000DEBF0FBECDBF8C016B0165EC7BE0CE01E4
:10C2F000019608D96BE371E1C801F4D876012FEFFC
:10C30000E21AF20A4AE0B701CE010796A0D8BE01B0
:10C31000695F7F4FCE010D96EDD86BEF77E0CE01D0
:10C320000D960E949158BC01C8010E940959CE0186
:10C330000D960E949859CE0107960E9498598AE05E
:10C34000B82EBE9CC001BF9C900D1124FC01E75685
:10C35000FE4E7F018081082E000C990B0E9407BAC7
:10C36000892B09F4AFC0B701CE010796CBD8BE0127
:10C37000695F7F4FCE010D96BDD867EF7AE0CE01A1
:10C380000D960E949158BC01C8010E940959CE0126
:10C390000D960E949859CE0107960E949859BC9C10
:10C3A000C001BD9C900D11249C0127563E4E790181
:10C3B000F9016685062E000C770B4AE0CE01079640
:10C3C00046D8BE01695F7F4FCE010D9693D869EEC6
:10C3D00079E0CE010D960E949158BE016F5F7F4FAC
:10C3E0000E94A858BC01C8010E940959CE010D96AF
:10C3F0000E949859CE0107960E94985964E371E112
:10C40000C8010E94B958F7016785062E000C770B0A
:10C410004AE0CE0107961BD8BE01695F7F4FCE016F
:10C420000D9668D8BE016F5F7F4FCE010D960E94BA
:10C43000A858BC01C8010E940959CE010D960E945E
:10C440009859CE0107960E9498596EE271E1C80191
:10C450000E94B958F701608971894AE0CE010796B8
:10C460000E94275ABE01695F7F4FCE010D9642D8C8
:10C47000BE016F5F7F4FCE010D960E94A858BC0190
:10C48000C8010E940959CE010D960E949859CE010B
:10C4900007960E94985969E271E1C8010E94B95853
:10C4A000F701628973894AE0CE0107960E94275AF4
:10C4B000BE01695F7F4FC8010E940959CE010796EE
:10C4C0000E949859CE0101960E949859C80162961F
:10C4D0000FB6F894DEBF0FBECDBFDF91CF911F9195
:10C4E0000F91FF90EF90DF90CF90BF900895EF9263
:10C4F000FF920F931F93CF93DF93CDB7DEB768976B
:10C500000FB6F894DEBF0FBECDBF8C0165EC7BE0AB
:10C51000CE0107960E94825A6BEE79E0CE01019619
:10C520000E94825A65E071E1C8010E94725ABE0100
:10C530006F5F7F4FC8010E9409596CEF70E1C8011D
:10C540000E94B95889E9E82E81E1F82EF70160814F
:10C5500070E04AE0CE010D960E94275ABE01635F4B
:10C560007F4FCE0143960E947A5ABE01695F7F4F8A
:10C57000CE0143960E94A858BC01C8010E940959E7
:10C58000CE0143960E949859CE010D960E9498596B
:10C590006FEE70E1C8010E94B958F7016181062E63
:10C5A000000C770B4AE0CE010D960E94275ABE017F
:10C5B000635F7F4FCE0143960E947A5ABE01695F46
:10C5C0007F4FCE0143960E94A858BC01C8010E942B
:10C5D0000959CE0143960E949859CE010D960E94AA
:10C5E000985965EE70E1C8010E94B958F70162815F
:10C5F000062E000C770B4AE0CE010D960E94275ABA
:10C60000BE01635F7F4FCE0143960E947A5ABE01FE
:10C61000695F7F4FCE0143960E94A858BC01C801B4
:10C620000E940959CE0143960E949859CE010D9659
:10C630000E9498596DED70E1C8010E94B958F70148
:10C64000638174814AE0CE010D960E94275ABE0193
:10C65000635F7F4FCE0143960E947A5ABE016F5F9F
:10C660007F4FCE0143960E94A858BC01C8010E948A
:10C670000959CE0143960E949859CE010D960E9409
:10C68000985966EC70E1C8010E94B958F7016581BC
:10C6900076814AE0CE010D960E94275ABE01635F63
:10C6A0007F4FCE0143960E947A5ABE01695F7F4F49
:10C6B000CE0143960E94A858BC01C8010E940959A6
:10C6C000CE0143960E949859CE010D960E9498592A
:10C6D0006DEB70E1C8010E94B958F7016781062E21
:10C6E000000C770B6F5F7F4F4AE0CE010D960E94E2
:10C6F000275ABE01635F7F4FCE0143960E947A5A4C
:10C70000BE01695F7F4FCE0143960E94A858BC01CD
:10C71000C8010E940959CE0143960E949859CE0142
:10C720000D960E94985962EB70E1C8010E94B958B9
:10C73000F7016085062E000C770B4AE0CE010D96BE
:10C740000E94275ABE01635F7F4FC8010E940959AA
:10C75000CE010D960E949859CE0101960E949859DB
:10C76000CE0107960E949859C80168960FB6F894B2
:10C77000DEBF0FBECDBFDF91CF911F910F91FF9014
:10C78000EF9008958F929F92AF92BF92CF92DF92D7
:10C79000EF92FF920F931F93CF93DF93CDB7DEB746
:10C7A00068970FB6F894DEBF0FBECDBF6C018091C5
:10C7B000801190918111019731F062EC79E0C6010E
:10C7C0000E94825A3BC16EEE79E0CE010D960E9426
:10C7D000825ABE01635F7F4F87EB9DE00E94E15A62
:10C7E0006CE271E080E090E00E946351CE01079618
:10C7F0000E94B08864E670E080E090E00E9463519F
:10C8000000E010E085E0A82EB12C9AE0892E912C52
:10C8100069EF79E0CE0101960E94825ABE016F5FF6
:10C820007F4FCE0107960E944B587C01CE010196A6
:10C830000E949859A7014F5F5F4FBE01695F7F4F0C
:10C84000CE0101960E943B3EBE016F5F7F4FCE013D
:10C850000D960E945F59CE0101960E9498598989D0
:10C860009A89892B69F060E070E0CE010D960E94F4
:10C870006558082E000C990BC0970A9708F4C6C09B
:10C88000F12C62EA70E1CE0101960E94725A44E1F5
:10C8900050E06FEF7FEFCE0101960E941733CE017B
:10C8A00001960E9498590F5F1F4F62E370E080E08D
:10C8B00090E00E946351C801B5010E948DB70197B5
:10C8C00069F5CE0101960E943D878D819E81892B5D
:10C8D00059F0BE016F5F7F4F87EB92E10E944A598A
:10C8E00011D6FF24F39416C0043111059CF0C80141
:10C8F000B4010E948DB7892B69F4BE01635F7F4F3D
:10C9000087EB9DE00E94E15A68EC70E080E090E0E7
:10C910000E946351CE0101960E949859CE01019662
:10C920000E94B088BE016F5F7F4FCE0107960E94C4
:10C930005F59CE0101960E94985962E370E080E051
:10C9400090E00E9463510436110519F0FF2009F4AC
:10C950005FCF8091C50C8823F1F06CEE79E0CE01B9
:10C9600001960E94825ABE01635F7F4FCE010196FD
:10C970000E94A858BC01CE0143960E947A5ACE016B
:10C9800043960E94439ACE0143960E949859CE0145
:10C9900001960E94985989899A89892B71F060E0E3
:10C9A00070E0CE010D960E946558282F880F330B3A
:10C9B000205331092A30310530F06BEF79E0C601A0
:10C9C0000E94825A1AC067E07AE0CE0101960E9466
:10C9D000825ABE016F5F7F4FCE010D960E9476583E
:10C9E000182FCE0101960E9498591111E6CFBE0171
:10C9F000635F7F4FC6010E946A5ACE0107960E946C
:10CA00009859CE010D960E94985918C067E07AE0B7
:10CA1000CE0101960E94825ABE016F5F7F4FCE0108
:10CA20000D960E947658E82ECE0101960E949859E4
:10CA3000FF24F394EE2009F424CF22CFC601689698
:10CA40000FB6F894DEBF0FBECDBFDF91CF911F911F
:10CA50000F91FF90EF90DF90CF90BF90AF909F909D
:10CA60008F900895382F2091B60D9091A613213202
:10CA700008F049C08091930D8111FCCF42E04093B2
:10CA8000930D3093920D3FEF3093910D1092900DD6
:10CA900020938F0DA6E9BDE04FE65DE0FA013E2F41
:10CAA000341B321718F43D913193F9CF10926E0D6B
:10CAB00020916E0D990F922B90936E0D90916D0DAC
:10CAC000913061F410926D0D90916E0D9093BB00BA
:10CAD0009091BC0093FDF8CF95EC01C095EE90933A
:10CAE000BC009091930D9230E1F39091910D9F3F96
:10CAF00079F08091910D803241F08091910D8033D9
:10CB000031F084E005C081E003C082E001C083E031
:10CB10001092950D1092B60D1092940D089581E02B
:10CB2000A1CF682F8BE290E10C94FF8B91E0909362
:10CB3000940D8093A6131092950D1092B60D089542
:10CB4000CF93C82F682F607F8AE993E10E947D55BB
:10CB500080E1C89FB00111248AE993E1CF910C9440
:10CB60007D55CF93DF93CDB7DEB728970FB6F894F6
:10CB7000DEBF0FBECDBF98E0EFE3F5E0DE0111961A
:10CB800001900D929A95E1F79091A313961710F4E6
:10CB90006FEF690FFE013196E60FF11DE60FF11DF3
:10CBA0009081890F806828960FB6F894DEBF0FBE7B
:10CBB000CDBFDF91CF91C4CF4F925F926F927F92A2
:10CBC0008F929F92AF92BF92CF92DF92EF92FF929D
:10CBD0006B017C01B42E9B01AC010E9451B78823EC
:10CBE00019F06FE17AE027C026013701E89477F861
:10CBF0002FEF3FEF4FE75FE7C301B2010E9451B74C
:10CC000081110DC02FEF3FEF4FE75FE7C301B20186
:10CC10000E94C2B218161CF463E27AE00CC02FEF37
:10CC20003FEF4FE75FE4C701B6010E9407B6181651
:10CC300094F467E27AE08EE89FE0FF90EF90DF9057
:10CC4000CF90BF90AF909F908F907F906F905F90AC
:10CC50004F900C94135B2FEF3FEF4FE75FECC70152
:10CC6000B6010E94C2B287FDE4CF20E030E0A90106
:10CC7000C701B6010E94C2B287FF0BC06DE28EE809
:10CC80009FE00E94DA5A4C01F7FAF094F7F8F0941A
:10CC900002C0812C912CA12C60E070E080E09FE329
:10CCA000AB1441F020E030E040E251E40E9418B5BE
:10CCB000A394F6CF9B01AC01C701B6010E9452B408
:10CCC0002B013C010E94B6B56B017C010E94C6B2EB
:10CCD0009B01AC01C301B2010E9451B42B013C0184
:10CCE0002AE0B701A6018EE89FE00E94285B7C0144
:10CCF000E80CF91CBB2039F06EE28EE89FE00E9440
:10CD0000DA5AE80EF91EDB2CDD2031F120E030E0AC
:10CD100040E251E4C301B2010E9427B32B013C0160
:10CD20000E94B6B54B01A12CB12C2AE0B501A4019B
:10CD30008EE89FE00E94285BE80EF91EC501B40151
:10CD40000E94C6B29B01AC01C301B2010E9451B462
:10CD50002B013C01DA94D8CFC701FF90EF90DF9010
:10CD6000CF90BF90AF909F908F907F906F905F908B
:10CD70004F90089510926C0D10926B0D1092950DBE
:10CD80001092B60D1092930D81E08093920D109247
:10CD90006D0D61E084E10E94A85061E085E10E9490
:10CDA000A850E9EBF0E080818E7F808380818D7FC9
:10CDB000808388E48093B80085E48093BC00089564
:10CDC0002F923F924F925F926F927F928F929F929B
:10CDD000AF92BF92CF92DF92EF92FF920F931F9389
:10CDE000CF93DF93CDB7DEB728970FB6F894DEBFA9
:10CDF0000FBECDBF40911B0D50911C0DC0901D0D5D
:10CE0000D0901E0D4C155D052CF03C2D2D2D6A018A
:10CE1000432F522FEFE1FDE060E070E0CB01019184
:10CE200011910417150754F44A01550FAA08BB08BD
:10CE3000680D791D8A1D9B1DA80115C0C016D1065D
:10CE400054F40D2C000CEE08FF086C0D7D1D8E1D9A
:10CE50009F1D680108C0012E000C220B330B600FD0
:10CE6000711F821F931F2DE0EB36F207C1F60E945F
:10CE7000C8B220E030E048E152E40E9418B56B01EE
:10CE80007C010BE11DE0812C912C5401D8016D91A6
:10CE90007D918D01072E000C880B990B0E94C8B262
:10CEA000A70196010E9451B49B01AC010E9427B3D7
:10CEB0009B01AC01C501B4010E9452B44B015C015D
:10CEC000BDE00B361B0711F720E030E04CE152E4E7
:10CED0000E9418B50E9410B74B015C0120E030E0C1
:10CEE00040E85FE30E9407B618160CF06EC00BE135
:10CEF0001DE0212C312C19821A821B821C82F80120
:10CF0000819191918F019C01990F440B550B2D83B9
:10CF10003E834F835887CA01B9010E94C8B2A70156
:10CF200096010E9451B42B013C0120E030E0A901A0
:10CF30000E9407B6181624F077FA709477F8709468
:10CF4000A5019401C301B2010E94C2B287FF13C0C0
:10CF500089819A81AB81BC812D813E814F81588529
:10CF6000820F931FA41FB51F89839A83AB83BC8351
:10CF70003FEF231A330A4DE00B36140709F0BFCFF9
:10CF800020E030E040EC5FE3C501B4010E9427B32C
:10CF90004B015C0155E0251631040CF4A8CF6981E2
:10CFA0007A818B819C810E94C8B26B017C01B101A6
:10CFB000330C880B990B0E94C8B29B01AC01C701CE
:10CFC000B6010E9418B56B017C01C701B601289615
:10CFD0000FB6F894DEBF0FBECDBFDF91CF911F918A
:10CFE0000F91FF90EF90DF90CF90BF90AF909F9008
:10CFF0008F907F906F905F904F903F902F9008950B
:10D000004F925F926F927F928F929F92AF92BF9258
:10D01000CF92DF92EF92FF920F931F93CF93DF9304
:10D0200000D01F92CDB7DEB76B017C0111E0A12EBD
:10D03000B12C4501880C991C880C991CF401E55908
:10D04000FD4F4080518062807380A3019201C7012F
:10D05000B6010E9407B6181614F41F5FE8CFA301AB
:10D060009201C701B6010E94C2B284010D5A1D4F40
:10D07000811106C0D8016D917D918D919C9142C026
:10D08000C5018150904C880F991F880F991FFC0192
:10D09000E559FD4F208131814281538129833A83B3
:10D0A0004B835C83FC01ED5AFD4F80809180A28010
:10D0B000B380C701B6010E9451B46B017C01A50188
:10D0C0009401D8016D917D918D919C910E9451B4F4
:10D0D0009B01AC01C701B6010E9427B36B017C0123
:10D0E00029813A814B815C81C301B2010E9451B414
:10D0F0009B01AC01C701B6010E9418B5A5019401BE
:10D100000E9452B40F900F900F900F90DF91CF912B
:10D110001F910F91FF90EF90DF90CF90BF90AF9055
:10D120009F908F907F906F905F904F9008950F9396
:10D130001F930E949B5160935C0E70935D0E8093D1
:10D140005E0E90935F0EE091540EF091550E0284A6
:10D15000F385E02D84E59EE0199597FF1FC00E949E
:10D160009B5100915C0E10915D0E20915E0E3091EE
:10D170005F0EDC01CB01801B910BA20BB30B009166
:10D18000580E1091590E20915A0E30915B0E801757
:10D190009107A207B307B8F28FEF9FEF1F910F918E
:10D1A00008950F931F93CF93DF931F921F92CDB7D4
:10D1B000DEB709E11DE0F80160818EED93E09A830E
:10D1C0008983CE0101960E94B43DF80161818FED03
:10D1D00093E09A838983CE0101960E94B43DC801F1
:10D1E0000F900F90DF91CF911F910F910895EF92C3
:10D1F000FF920F931F93CF93DF931F921F92CDB790
:10D20000DEB709E911E1895991417C019701200FAD
:10D21000311FF80161918F013A832983CE01019674
:10D220000E94B43DF1E1033A1F0781F789E991E1DA
:10D230000F900F90DF91CF911F910F91FF90EF9082
:10D240000895EF92FF920F931F93CF93DF931F9256
:10D250001F92CDB7DEB70AE011E18A5091417C01FF
:10D260009701200F311FF80161918F013A832983C3
:10D27000CE0101960E94B43DF1E100391F0781F70C
:10D280008AE091E10F900F90DF91CF911F910F9164
:10D29000FF90EF900895EF92FF920F931F93CF931B
:10D2A000DF931F921F92CDB7DEB709E911E18959CB
:10D2B00091417C019701200F311FF80161918F018D
:10D2C0003A832983CE0101960E94B43DF2E10339ED
:10D2D0001F0781F789E991E10F900F90DF91CF91BE
:10D2E0001F910F91FF90EF9008953F924F925F92A0
:10D2F0006F927F928F929F92AF92BF92CF92DF9266
:10D30000EF92FF920F931F93CF93DF9300D01F9262
:10D310001F92CDB7DEB7982E0E949B512B013C0186
:10D3200020ED420E27E0521E611C711C60E08091CE
:10D3300084130E94A85035E0832ECE0101966C0123
:10D34000AA24A394B12C55E0352E380EF601282DD1
:10D3500011922A95E9F7860127E0E22EF12C8091BF
:10D3600085130E944B5D019739F40E949B5164150F
:10D3700075058605970598F3809185130E944B5D8E
:10D38000892B39F40E949B51641575058605970514
:10D3900098F3809186130E944B5D892B51F0F80120
:10D3A0002081C5010E2C01C0880F0A94EAF7822B58
:10D3B0008083F1E0EF1AF10890F60F5F1F4F3012F3
:10D3C000CBCF0E949B51641575058605970550F0DB
:10D3D00061E0809184130E94A85060E070E080ECCE
:10D3E0009FE72CC089818911B1CF9B818A81980FD9
:10D3F000990D8C818913AACF8D818D3009F0A6CF2C
:10D4000061E0809184130E94A8506A818B8170E052
:10D41000762F6627680F711D072E000C880B990B5D
:10D420000E94C8B220E030E040E85DE30E9427B3EC
:10D4300023E333E948E853E40E9451B40F900F907E
:10D440000F900F900F90DF91CF911F910F91FF9050
:10D45000EF90DF90CF90BF90AF909F908F907F9094
:10D460006F905F904F903F9008959091930D911120
:10D47000FCCF91E09093930D9093920D2FEF20931A
:10D48000910D1092900D260F20938F0D90936E0D9D
:10D4900090916E0D880F892B80936E0D80916D0D8C
:10D4A000813061F410926D0D80916E0D8093BB0000
:10D4B0008091BC0083FDF8CF85EC01C085EE8093A0
:10D4C000BC008091930D8130E1F38091900D86171F
:10D4D00010F46091900DAFE6BDE029EF3CE0F9015A
:10D4E0008E2F821B861718F48D918193F9CF862F8A
:10D4F0000895613208F060E2B8DF10926C0D8093FD
:10D500006B0D0895AF92BF92CF92DF92EF92FF9290
:10D510000F931F93CF93DF93CDB7DEB7A4970FB6CA
:10D52000F894DEBF0FBECDBF8091AB13882319F0F6
:10D530001092AB1395C58091BB129091BC120497C9
:10D5400008F041C062EB77E0CE0101960E94825A5A
:10D55000BE016F5F7F4F87EB92E10E947658182FD4
:10D56000CE0101960E949859112369F161E070E0A3
:10D5700087EB92E10E94655880330CF4845E6AE286
:10D5800070E0681B710987FD73954AE0CE01019632
:10D590000E94275ABE016F5F7F4F87EB92E10E9486
:10D5A0005F59CE0101960E94985967EB72E18BEAB0
:10D5B00092E10E944A5987EB92E10E949157CB0178
:10D5C0000E94D60A4DC562EF76E0CE0107960E9412
:10D5D000825ABE01695F7F4F87EB92E10E947658C5
:10D5E000811116C068EF76E0CE0101960E94825A42
:10D5F000BE016F5F7F4F87EB92E10E94765811E08A
:10D60000811101C010E0CE0101960E94985901C01D
:10D6100011E0CE0107960E949859112309F487C39F
:10D620006BE27AE0CE0101960E94825ACE01019609
:10D630000E94439ACE0101960E94985967E37AE0CE
:10D64000CE0107960E94825A6EE873E1CE010796DA
:10D650000E94A858BC01CE0101960E947A5ACE01C0
:10D6600001960E94439ACE0101960E949859CE01DC
:10D6700007960E94985960913D0270913E028091F8
:10D680003F02909140020E94C8B220E030E048EC96
:10D6900052E40E9418B5AB01BC0122E0CE0107960E
:10D6A0000E94CC596DE47AE0CE010D960E94825A18
:10D6B000BE01695F7F4FCE010D960E94A85869E7B1
:10D6C00078E00E949158BC01CE0101960E947A5ADE
:10D6D000CE0101960E94439ACE0101960E9498596C
:10D6E000CE010D960E949859CE0107960E94985936
:10D6F0004091390250913A0260913B0270913C0294
:10D7000024E0CE0107960E94CC5962E67AE0CE0171
:10D710000D960E94825ABE01695F7F4FCE010D9621
:10D720000E94A858BC01CE0101960E947A5ACE01EF
:10D7300001960E94439ACE0101960E949859CE010B
:10D740000D960E949859CE0107960E9498594091D3
:10D750000D0550910E0560910F057091100522E0A6
:10D76000CE0107960E94CC594091190550911A0597
:10D7700060911B0570911C0523E0CE010D960E945F
:10D78000CC5940911105509112056091130570918B
:10D79000140522E0CE0143960E94CC594091150514
:10D7A00050911605609117057091180523E0CE0180
:10D7B00049960E94CC596FE77AE0CE014F960E94BD
:10D7C000825ABE01675E7F4FCE014F960E94A858D5
:10D7D00064E97AE00E949158BE016D5E7F4F0E941D
:10D7E000A85867E97AE00E949158BE01635F7F4FB5
:10D7F0000E94A85864E97AE00E949158BE01695FCE
:10D800007F4F0E94A8586DE97AE00E949158BC01B0
:10D81000CE0101960E947A5ACE0101960E94439A47
:10D82000CE0101960E949859CE014F960E949859B8
:10D83000CE0149960E949859CE0143960E9498596C
:10D84000CE010D960E949859CE0107960E949859D4
:10D8500064E872E1CE0149960E94725AF090391143
:10D860000F2D0F2C000C110B01151105A1F52091A6
:10D870003A1130913B1140913C1150913D1160E0C3
:10D8800070E080EA90E40E9418B5AB01BC0122E090
:10D89000CE0101960E949D5964EE78E0CE01079674
:10D8A0000E94825ABE016F5F7F4FCE0107960E9491
:10D8B000A85864E178E00E949158BC01CE014996D5
:10D8C0000E940959CE0107960E949859CE010196EF
:10D8D0000E94985909C00130110531F466E772E1E0
:10D8E000CE0149960E94B958C8010297029740F5A7
:10D8F0008F2D9AE08902B00111244AE0CE010196F1
:10D900000E94275A62EA7AE0CE0107960E94825A64
:10D91000BE016F5F7F4FCE0107960E94A8586DE051
:10D9200078E00E949158BC01CE0149960E940959A5
:10D93000CE0107960E949859CE0101960E949859EF
:10D940000430110519F464E672E105C005301105D3
:10D9500034F06CE572E1CE0149960E94B958BE01DF
:10D96000675E7F4FCE0101960E947A5ACE010196E2
:10D970000E94439ACE0101960E9498596EEA7AE07D
:10D98000CE0149960E943559809136116091371128
:10D99000709138114AE083300CF050C3CE010196EB
:10D9A0000E94275A69EA7AE0CE0107960E94825ABD
:10D9B000BE016F5F7F4FCE0107960E94A85866EAAE
:10D9C0007BE00E949158BC01CE0149960E94095902
:10D9D000CE0107960E949859CE0101960E9498594F
:10D9E000BE01675E7F4FCE0101960E947A5ACE013A
:10D9F00001960E94439ACE0101960E949859409147
:10DA00003E1150913F11609140117091411122E0FF
:10DA1000CE0107960E94CC596EEB7AE0CE010D96AE
:10DA20000E94825ABE01695F7F4FCE010D960E940F
:10DA3000A85864ED7AE00E949158BC01CE0101968D
:10DA40000E947A5ACE0101960E94439ACE01019615
:10DA50000E949859CE010D960E949859CE010796C2
:10DA60000E9498594091541150915511609156114E
:10DA70007091571122E0CE0107960E94CC596BEDB0
:10DA80007AE0CE010D960E94825ABE01695F7F4FF7
:10DA9000CE010D960E94A85864ED75E00E94915841
:10DAA000BC01CE0101960E947A5ACE0101960E94D5
:10DAB000439ACE0101960E949859CE010D960E947C
:10DAC0009859CE0107960E94985985E2C82E82E0A7
:10DAD000D82E01E010E099E1F92E80912302909177
:10DAE0002402801791070CF44FC0F601A190B19069
:10DAF0006F014AE0B501CE0107960E94275A4AE01D
:10DB0000B801CE010D960E94275A6EEE7AE0CE0142
:10DB100043960E94825ABE01635F7F4FCE014396B7
:10DB20000E94A85866EF7AE00E949158BE01695F92
:10DB30007F4F0E94A85869EF7AE00E949158FA9CA2
:10DB4000B001FB9C700D112465567D4F0E949158C9
:10DB5000BC01CE0101960E947A5ACE0101960E9424
:10DB6000439ACE0101960E949859CE0143960E9495
:10DB70009859CE010D960E949859CE0107960E94A1
:10DB800098590F5F1F4FA9CF8091801190918111FB
:10DB9000892B71F46FEF7AE0CE0101960E94825AD0
:10DBA000CE0101960E94439ACE0101960E94985997
:10DBB0008091801190918111019771F46EE07BE06A
:10DBC000CE0101960E94825ACE0101960E94439A8C
:10DBD000CE0101960E9498598091801190918111F7
:10DBE000029771F468E17BE0CE0101960E94825AAF
:10DBF000CE0101960E94439ACE0101960E94985947
:10DC000060911D0570911E054AE0CE0107960E94A5
:10DC1000275A6AE27BE0CE010D960E94825ABE012D
:10DC2000695F7F4FCE010D960E94A858BC01CE01BE
:10DC300001960E947A5ACE0101960E94439ACE0123
:10DC400001960E949859CE010D960E949859CE01D6
:10DC500007960E94985940910402509105026091E4
:10DC600006027091070222E0CE0107960E94CC596D
:10DC700067E47BE0CE010D960E94825ABE01695F87
:10DC80007F4FCE010D960E94A85862EE75E00E946B
:10DC90009158BC01CE0101960E947A5ACE0101969C
:10DCA0000E94439ACE0101960E949859CE010D968A
:10DCB0000E949859CE0107960E94985940910002FF
:10DCC00050910102609102027091030222E0CE01A4
:10DCD00007960E94CC5967E57BE0CE010D960E9425
:10DCE000825ABE01695F7F4FCE010D960E94A858EF
:10DCF00062EE75E00E949158BC01CE0101960E942F
:10DD00007A5ACE0101960E94439ACE0101960E9452
:10DD10009859CE010D960E949859CE0107960E94FF
:10DD2000985910920902CE0149960E949859209163
:10DD3000BB123091BC122330310508F06CC1213088
:10DD4000310541F460E070E087EB92E10E94655894
:10DD5000E82E59C02230310509F055C062EB77E05A
:10DD6000CE0101960E94825ABE016F5F7F4F87EB02
:10DD700092E10E947658182FCE0101960E94985980
:10DD8000112309F440C061E070E087EB92E10E944A
:10DD90006558682FCE0101960E94525ABE016F5FEE
:10DDA0007F4F8BEA92E10E945F59CE0101960E945B
:10DDB000985960E070E087EB92E10E946558E82E88
:10DDC0008091C50C8823F9F067E67BE0CE010196CF
:10DDD0000E94825A67EB72E1CE0101960E94A85818
:10DDE00065EC7BE00E949158BC018EE89FE00E94A8
:10DDF000E15ACE0101960E9498596BEA72E18EE8D1
:10DE00009FE00E94D05B8E2DEE0C990B0E94F4B91E
:10DE1000892BB1F00E94AA910E94483265EC7BE008
:10DE2000CE0101960E94825A4AE050E060E070E024
:10DE3000CE0101960E941733CE0101960E94985997
:10DE400067EB72E1CE0107960E947A5A60E070E0BB
:10DE5000CE0107960E946558823409F475C0D4F447
:10DE6000803309F491C07CF4833209F484C08A328F
:10DE700009F0AAC060E87BE087EB92E10E94355987
:10DE80008FEF9FEF8FC0813309F48FC0813409F485
:10DE900050C09AC0813609F44CC034F4833409F47C
:10DEA0005EC0843449F090C0833609F458C00CF445
:10DEB0004BC0843609F088C08091AF129091B012A7
:10DEC000892B09F4A1C061E070E0CE0107960E94A1
:10DED0006558182F8091C50C882361F06DE67BE0B2
:10DEE0008EE89FE00E94E05B6BEA72E18EE89FE0C3
:10DEF0000E94D05B10330CF4145E6AE270E0611B88
:10DF0000710917FD73954AE0CE0101960E94275AC8
:10DF1000BE016F5F7F4F8BEA92E10E945F59CE0195
:10DF200001960E9498598BEA92E10E949157CB0189
:10DF300039C064E77BE087EB92E10E94355980911C
:10DF4000BD0C9091BE0C2EC067E77BE087EB92E1A1
:10DF50000E9435591092B0138CEF9FEF23C06AE7EF
:10DF60007BE087EB92E10E94355981E08093B0130A
:10DF70008DEF9FEF17C06DE77BE087EB92E10E948A
:10DF800035598EEF9FEF0EC06DE07AE08BEA92E19B
:10DF90000E9435596DE07AE087EB92E10E94355995
:10DFA00080E090E00E94D60A2FC061E87BE08BEA17
:10DFB00092E10E94355961E87BE087EB92E10E9493
:10DFC000355981E090E0EECFBE01695F7F4F8BEA6B
:10DFD00092E10E944A5960E070E08BEA92E10E946F
:10DFE0006558082E000C990BC0970A9738F48BEAF5
:10DFF00092E10E949157CB010E94D60A64E670E03C
:10E0000080E090E00E946351CE0107960E949859EB
:10E010000E949B5102C00E9456260E949B51609311
:10E02000A7137093A8138093A9139093AA1362EC7B
:10E0300079E087EB92E10E94355912C0CE0101963A
:10E040000E94275A63E87BE0CE0107960E94825A1D
:10E05000BE016F5F7F4FCE0107960E94A858B3CCD8
:10E06000A4960FB6F894DEBF0FBECDBFDF91CF915F
:10E070001F910F91FF90EF90DF90CF90BF90AF90E6
:10E0800008954F925F926F927F92AF92BF92CF921C
:10E09000DF92EF92FF920F931F93CF93DF93CDB751
:10E0A000DEB72C970FB6F894DEBF0FBECDBF81E070
:10E0B00080930902CE0101960E943D87BE016F5FE9
:10E0C0007F4F87EB92E10E945F59CE0101960E943B
:10E0D00098598091BB129091BC12892B89F462E00F
:10E0E00070E0CE0101960E94A88ABE016F5F7F4F4B
:10E0F00087EB92E10E945F59CE0101960E949859E8
:10E100008091BB129091BC12892B89F462E070E07F
:10E11000CE0101960E944389BE016F5F7F4F87EB5E
:10E1200092E10E945F59CE0101960E9498596AE0DF
:10E1300070E080E090E00E9463518091BB1290916A
:10E14000BC12892B09F441C08091C50C8823A9F128
:10E150006CEE79E0CE0101960E94825ABE016F5F9B
:10E160007F4F87EB92E10E947658182FCE010196DF
:10E170000E949859111121C06CE87BE0CE010196F4
:10E180000E94825A67EB72E1CE0101960E94A85864
:10E1900066EC79E00E949158BC01CE0107960E947E
:10E1A0007A5ACE0107960E94439ACE0107960E94A2
:10E1B0009859CE0101960E9498596AE070E080E07B
:10E1C00090E00E9463519ED9EAC180919411882306
:10E1D00009F49CC180919E1190919F1197FF04C0FA
:10E1E00010929F1110929E1180919C1190919D11FF
:10E1F000181619069CF420919E1130919F11281732
:10E20000390764F010929411109299118CE291E008
:10E210000E94F76810929F1110929E11E091A01138
:10E2200080919B11E817D4F18091B013811107C040
:10E2300080919C1190919D111816190634F50E9439
:10E240009B5128EE33E040E050E00E9420B4CA0128
:10E25000B9010E94C6B22091A90C3091AA0C40913C
:10E26000AB0C5091AC0C0E9451B42091040230913F
:10E27000050240910602509107020E9407B6181647
:10E280000CF08DC11092A0118AC1109299111092B8
:10E2900094118CE291E00E94F76881C10E2F0E2E3E
:10E2A000000C110B2AE0E202F0011124E756FE4EA9
:10E2B000E7840E2C000CFF088091A111A82E880F76
:10E2C000BB080E949B51409090115090911160901A
:10E2D000921170909311641975098609970928EEB7
:10E2E00033E040E050E00E9420B4CA01B9010E942E
:10E2F000C6B22B013C016701F7FE04C0CC24DD242B
:10E30000CE18DF08C501B7FE02C080E090E08C1592
:10E310009D050CF09AC08AE0809FF001819FF00D6E
:10E320001124E756FE4E60897189072E000C880B78
:10E33000990B0E94C8B29B01AC01C301B2010E94BB
:10E3400007B618160CF02BC1F7FE09C080919E117C
:10E3500090919F11B6010E948DB7892B71F48AE0CC
:10E36000809FF001819FF00D1124E756FE4E8685B7
:10E37000082E000C990B0E94D60A0E949B516093B4
:10E3800090117093911180939211909393118091B9
:10E39000A1118F5F8093A111082E000C990B8C1591
:10E3A0009D050CF4FCC080919B11082E000C990B6C
:10E3B0000197081719070CF4F2C080919E119091F3
:10E3C0009F11019690939F1180939E118091B0139D
:10E3D000811108C080919C1190919D111816190609
:10E3E0000CF0DDC08CE291E00E94F76863E873E115
:10E3F0008FE992E10E940F5960919E1170919F11D7
:10E400004AE0CE0101960E94275ABE016F5F7F4FFE
:10E410008FE992E10E940959CE0101960E94985914
:10E420006CED75E080E090E00E9463516FE972E16D
:10E43000CE0101960E947A5ACE0101960E94439A1B
:10E44000CE0101960E949859AAC03AE0F32EF09EA0
:10E45000F001F19EF00D1124E756FE4E628973899A
:10E46000072E000C880B990B0E94C8B29B01AC01CF
:10E47000C301B2010E9407B618160CF090C01092AA
:10E48000A1118091A0118F5F8093A011082E000C24
:10E49000990B20919B11022E000C330B82179307CE
:10E4A00004F5F89EF001F99EF00D1124E756FE4E9A
:10E4B000878587FD06C08685082E000C990B0E9473
:10E4C000D60A0E949B516093901170939111809392
:10E4D0009211909393118091A1118F5F8093A1115C
:10E4E0005EC00E949B5128EE33E040E050E00E9465
:10E4F00020B4CA01B9010E94C6B26093A90C7093FE
:10E50000AA0C8093AB0C9093AC0C49C08091B013D3
:10E51000882309F44FC00E949B5128EEC22E23E0AD
:10E52000D22EE12CF12CA70196010E9420B4CA0141
:10E53000B9010E94C6B22091A90C3091AA0C409159
:10E54000AB0C5091AC0C0E9451B42091040230915C
:10E55000050240910602509107020E9407B6181664
:10E560004CF50E949B51A70196010E9420B4CA015C
:10E57000B9010E94C6B26093A90C7093AA0C809353
:10E58000AB0C9093AC0C8091AC139091AD130E94A6
:10E59000D60A64E170E080E090E00E9463518091CF
:10E5A000B013882331F164E670E080E090E00E94CF
:10E5B00063511FC00E949B510091A7131091A81393
:10E5C0002091A9133091AA13DC01CB01801B910B80
:10E5D000A20BB30B88349E4EA105B10500F3109237
:10E5E000A51360E08AE993E10E94625510920C0540
:10E5F000D6CF2C960FB6F894DEBF0FBECDBFDF91FD
:10E60000CF911F910F91FF90EF90DF90CF90BF902F
:10E61000AF907F906F905F904F9008958F929F92F0
:10E62000AF92BF92CF92DF92EF92FF920F931F9320
:10E63000CF93DF93CDB7DEB7E0970FB6F894DEBF88
:10E640000FBECDBF9E012F5F3F4F79018E01015E4E
:10E650001F4F8130910509F091C065E97BE0C90148
:10E660000E94825A68E97BE0CE0107960E94825A96
:10E670006BE97BE0CE010D960E94825A65E773E15B
:10E68000C8010E94725A44E650E06FEF7FEFC80164
:10E690000E94D133C8010E9498596AE673E187EB62
:10E6A00092E10E940F5960911D0570911E054AE08C
:10E6B000CE0185960E94275A67EB72E1C8010E943D
:10E6C0007A5ABE016B5D7F4FC8010E94A858BC01F9
:10E6D000CE018B960E947A5A40ED57E06FEF7FEFA4
:10E6E000CE018B960E949832CE018B960E9498594B
:10E6F000C8010E949859CE0185960E9498596BE5F1
:10E7000073E1C8010E94725A44E650E06FEF7FEF58
:10E71000C8010E94D133C8010E94985963E47BE08C
:10E72000C8010E94825A23E030E0A801B701CE015F
:10E7300085960E94619FBE016B5D7F4F87EB92E1E2
:10E740000E945F59CE0185960E949859C8010E9487
:10E7500098598091BB129091BC12892B09F408C280
:10E7600060E070E087EB92E10E946558082E000C93
:10E77000990BC0970A9708F42EC2FAC18A3F3FEF5F
:10E78000930709F094C06EE97BE0C7010E94825AAA
:10E7900068EA7BE0CE0107960E94825A60EB7BE03C
:10E7A000CE010D960E94825A68EB7BE0CE01439623
:10E7B0000E94825A6CE473E1C8010E94725A44E6D6
:10E7C00050E06FEF7FEFC8010E94D133C8010E9473
:10E7D000985966E473E187EB92E10E940F598091AA
:10E7E0003611670196E08902C00CD11C112467EB39
:10E7F00072E1C8010E947A5AB601C8010E94A85865
:10E80000BC01CE0185960E947A5A40ED57E06FEF29
:10E810007FEFCE0185960E949832CE0185960E94A8
:10E820009859C8010E94985966E373E1C8010E9493
:10E83000725A44E650E06FEF7FEFC8010E94D13377
:10E84000C8010E9498596EEB7BE0C8010E94825A71
:10E8500024E030E0A801B701CE0185960E94619FB7
:10E86000BE016B5D7F4F87EB92E10E945F59CE0145
:10E8700085960E949859C8010E9498598091BB12B0
:10E880009091BC12892B69F060E070E087EB92E117
:10E890000E946558082E000C990BC0970A9708F43F
:10E8A000BEC1D12CCE0143960E94985962C10F96E9
:10E8B00009F0D2C0670162EC79E0C6010E94825A79
:10E8C00036E0C30ED11CC016D106A9F767EC7BE079
:10E8D000C7010E9435598091391181112FC02091B3
:10E8E0003A1130913B1140913C1150913D1160E043
:10E8F00070E080EA90E40E9418B5AB01BC0122E010
:10E90000CE0185960E949D596DEC7BE0C8010E9466
:10E91000825ABE016B5D7F4FC8010E94A8586DE00E
:10E9200078E00E949158BC01C7010E940959C801B2
:10E930000E949859CE0185960E9498596FE173E123
:10E94000CE0107960E940F5963E173E1CE010D9647
:10E950000E940F5967E073E1CE0143960E940F5960
:10E960006BEF72E1CE0149960E940F5965EF72E19B
:10E97000C8010E940F5966EE72E1C8010E94725AE6
:10E9800044E650E06FEF7FEFC8010E94D133C80129
:10E990000E94985962EC79E087EB92E10E94355928
:10E9A00080913911B70196E08902600D711D112423
:10E9B000C8010E947A5A40ED57E06FEF7FEFC8011F
:10E9C0000E949832C8010E94985967ED72E1C8010F
:10E9D0000E94725A44E650E06FEF7FEFC8010E9438
:10E9E000D133C8010E94985967EB72E1C8010E94B7
:10E9F0007A5A25E030E0A801B701CE0185960E9441
:10EA0000619FBE016B5D7F4F87EB92E10E945F5972
:10EA1000CE0185960E949859C8010E94985980910C
:10EA2000BB129091BC12892B69F060E070E087EB1B
:10EA300092E10E946558082E000C990BC0970A9726
:10EA400008F442C1D12C06501109C8010E949859FE
:10EA50000E151F05C1F798C060ED7BE0C7010E944D
:10EA6000825A63E17BE0CE0107960E94825A63EDF1
:10EA70007BE0CE010D960E94825A67EC72E1C801DC
:10EA80000E94725A44E650E06FEF7FEFC8010E9487
:10EA9000D133C8010E94985961EC72E187EB92E191
:10EAA0000E940F59809180119091811126E0289F3A
:10EAB0006001299FD00C1124CE0CDF1C67EB72E1A2
:10EAC000C8010E947A5AB601C8010E94A858BC0128
:10EAD000CE0185960E947A5A40ED57E06FEF7FEFA6
:10EAE000CE0185960E949832CE0185960E94985953
:10EAF000C8010E94985961EB72E1C8010E94725AE4
:10EB000044E650E06FEF7FEFC8010E94D133C801A7
:10EB10000E94985967EB72E1C8010E947A5A23E07B
:10EB200030E0A801B701CE0185960E94619FBE0129
:10EB30006B5D7F4F87EB92E10E945F59CE01859616
:10EB40000E949859C8010E9498598091BB129091D7
:10EB5000BC12892B69F060E070E087EB92E10E94C3
:10EB60006558082E000C990BC0970A9708F4C3C08B
:10EB7000D12CCE010D960E949859CE0107960E9485
:10EB80009859C7010E949859DD2019F064EA72E192
:10EB900002C065E972E1C7010E94725A48EC50E078
:10EBA0006FEF7FEFC7010E949832C7010E9498590A
:10EBB000E0960FB6F894DEBF0FBECDBFDF91CF91C8
:10EBC0001F910F91FF90EF90DF90CF90BF90AF908B
:10EBD0009F908F90089587EB92E10E9491574B018F
:10EBE0005C0162E878E0C8010E94825A26E0289D14
:10EBF000C001299D900D1124B701680F791FC8012C
:10EC00000E94A858BC0187EB92E10E944A59C801B2
:10EC10000E9498590E945626DD24D394AACF87EBF0
:10EC200092E10E9491576230710581059105ACF126
:10EC30006AE273E1C8010E94725A44E650E06FEF45
:10EC40007FEFC8010E949832C8010E94985944EF92
:10EC500051E063E070E0CE0185960E94D87F66EFB8
:10EC600078E0C8010E94825A67EB72E1C8010E94F5
:10EC7000A85864EC7BE00E949158BE016B5D7F4F09
:10EC80000E94A858BC0187EB92E10E944A59C80132
:10EC90000E949859CE01859610C066EF78E0C801B1
:10ECA0000E94825A67EB72E1C8010E94A858BC0119
:10ECB00087EB92E10E944A59C8010E9498590E942C
:10ECC0005626DD24D394EECD6DED78E0C8010E9488
:10ECD000825A67EB72E1C8010E94A858BC0187EB19
:10ECE00092E10E944A59C8010E9498590E945626F2
:10ECF000DD24D394A8CE87EB92E10E949157CB01FB
:10ED00000E94745DD82E35CF2F923F924F925F9222
:10ED10006F927F928F929F92AF92BF92CF92DF922B
:10ED2000EF92FF920F931F93CF93DF93CDB7DEB790
:10ED30002C970FB6F894DEBF0FBECDBF81EF9EE0DB
:10ED40000E94295D40E052EC61E070E081EF9EE0BE
:10ED50000E94D43D8CED95E0A0E0B0E08093F50EEC
:10ED60009093F60EA093F70EB093F80E64E670E061
:10ED700080E090E00E9463518091AE139091AF13B8
:10ED8000019759F483E090E00E949C9481111EC089
:10ED90001092AF131092AE1319C081E090E00E9460
:10EDA0009C94882339F081E090E09093AF13809396
:10EDB000AE130CC083E090E00E949C948111F3CFCD
:10EDC00083E090E00E949C948111EDCF8091AE137E
:10EDD0009091AF130197D9F06BE374E189E992E167
:10EDE0000E940F5969E972E1CE0101960E947A5A98
:10EDF00044E150E06FEF7FEFCE0101960E94983220
:10EE0000CE0101960E9498596FE274E1CEC063E290
:10EE100074E18FE992E10E940F596FE972E1CE012E
:10EE200001960E947A5ACE0101960E947238CE0154
:10EE300001960E94985962E370E080E090E00E94A1
:10EE400063516FE972E1CE0101960E947A5A42E362
:10EE500050E06FEF7FEFCE0101960E94D133CE01DB
:10EE600001960E94985967E174E189E992E10E9454
:10EE70000F5969E972E1CE0101960E947A5A44E184
:10EE800050E06FEF7FEFCE0101960E949832CE01E5
:10EE900001960E9498598BEB8F838AEA888781E0DC
:10EEA0008987412C512C3201E12CF12CC12CD12C21
:10EEB0004AE0242E312CC701B1010E948DB7892B65
:10EEC00049F443E050E0BE01695F7F4F81EF9EE06F
:10EED0000E94A95565E070E080E090E00E946351D7
:10EEE0008FEFE81AF80A00E010E0812C912C540111
:10EEF00081EF9EE00E941E56892B59F484E088160B
:10EF00009104A104B1042CF084E0C816D10434F0BB
:10EF10000AC0063011050CF487C0F6CF80E9E81668
:10EF200081E0F80641F6C301B2010E94C8B220E0B8
:10EF300030E040E251E40E9418B520E030E040E8C3
:10EF40005EE30E9427B36B017C0120E030E040EAE1
:10EF500051E40E9407B6181634F521E0B701A60166
:10EF6000CE0107960E94CC596BE077E0CE01019666
:10EF70000E94825ABE01695F7F4FCE0101960E94B6
:10EF8000A85867ED7BE00E949158BC018FE992E19F
:10EF90000E944A59CE0101960E949859CE010796C7
:10EFA0000E94985906C06BE074E18FE992E10E94DB
:10EFB0000F596FE972E1CE0101960E947A5A4AE038
:10EFC00050E060E070E0CE0101960E94D133CE01A6
:10EFD00001960E9498596FE972E1CE0101960E9454
:10EFE0007A5A65EC7BE0CE0101960E94915869E95E
:10EFF00072E10E94A858BC018FE992E10E944A592F
:10F00000CE0101960E94985981EF9EE00E94295DF1
:10F010008091B013882309F449C060E273E080E076
:10F0200090E00E94635142C081EF9EE00E941E5614
:10F03000892B69F081EF9EE00E94FC55E1E0F0E051
:10F04000EC0FFD1FE00FF11F80830F5F1F4F65E086
:10F0500070E080E090E00E9463510630110501F5F8
:10F0600099818F8198131CC09A818885981318C044
:10F070009B818985981314C02C818D8190E0A0E03C
:10F08000B0E0BA2FA92F982F8827820F911DA11DBC
:10F09000B11D480E591E6A1E7B1E8FEFC81AD80A72
:10F0A0008FEF881A980AA80AB80A22CF2C960FB6B2
:10F0B000F894DEBF0FBECDBFDF91CF911F910F91AE
:10F0C000FF90EF90DF90CF90BF90AF909F908F9088
:10F0D0007F906F905F904F903F902F9008953F9258
:10F0E0004F925F926F927F928F929F92AF92BF9258
:10F0F000CF92DF92EF92FF920F931F93CF93DF9304
:10F10000CDB7DEB7EB970FB6F894DEBF0FBECDBF1D
:10F110002B013C0184E59EE00E94295D64E670E0DD
:10F1200080E090E00E94635140E855E260E070E0CA
:10F1300084E59EE00E94D43D64E670E080E090E0CB
:10F140000E9463516FEF73E189E992E10E940F59C8
:10F1500069E972E1CE0101960E947A5A42E350E0D9
:10F160006FEF7FEFCE0101960E94D133CE01019661
:10F170000E94985964EF73E189E992E10E940F5966
:10F1800069E972E1CE0101960E947A5A42E350E0A9
:10F190006FEF7FEFCE0101960E949832CE0101966B
:10F1A0000E9498598091C30C9091C40C8D7F312C92
:10F1B000C12CD12CE12CF12C00E010E0019709F4D6
:10F1C0006CC0CE01809699AF88AFDE015E96BBAF72
:10F1D000AAAF0E949B51DC01CB0184199509A609B5
:10F1E000B709883B9B40A105B10508F056C084E5EE
:10F1F0009EE00E941E56892B09F448C08CED95E0D4
:10F20000A0E0B0E08093580E9093590EA0935A0E50
:10F21000B0935B0E0E94976897FD06C082349105FB
:10F22000C9F780E090E002C08FEF9FEF892B71F566
:10F23000DE0111964D015D010E94976897FF06C09F
:10F2400089818D3419F520E030E009C0D5018D9316
:10F250005D01E8ADF9ADAE17BF0771F7F1CFD4018D
:10F260008D914D01280F311DEAADFBADAE17BF07E3
:10F27000B1F72E5B3F4F8E8D90E0982F88274F8DF2
:10F28000840F911D2817390709F4FFC062E370E06D
:10F2900080E090E00E9463519CCF0E949B51DC0172
:10F2A000CB0184199509A609B709883B9B40A105A4
:10F2B000B10510F43110C1C00E94483269E972E111
:10F2C000CE0180960E947A5A42E350E066E070E0F8
:10F2D000CE0180960E94D133CE0180960E9498592B
:10F2E000332009F4EAC082E090E09093C40C80934C
:10F2F000C30C4AE0B601CE01C2960E94275A4AE0EA
:10F30000B701CE018C960E94275A4AE0B801CE017F
:10F3100080960E94275ABE01605E7F4FCE0186967E
:10F320000E947A5A6BEF77E0CE0186960E94915840
:10F33000BE01645D7F4F0E94A8586BEF77E00E948A
:10F340009158BE016E5C7F4F0E94A858BC018FE9A6
:10F3500092E10E944A59CE0186960E949859CE01A8
:10F3600080960E949859CE018C960E949859CE01A1
:10F37000C2960E9498596FE972E1CE0180960E9470
:10F380007A5A4AE050E06FEF7FEFCE0180960E94FC
:10F390009832CE0180960E9498596EEE73E18AE908
:10F3A00093E10E94EF5A4AE0B601CE01C2960E9454
:10F3B000275A4AE0B701CE018C960E94275A4AE0AC
:10F3C000B801CE0186960E94275A6AED7BE0CE01F5
:10F3D00080960E94825ABE016A5D7F4FCE01809660
:10F3E0000E94A85865EC7BE00E949158BE01645DC4
:10F3F0007F4F0E94A85865EC7BE00E949158BE01A7
:10F400006E5C7F4F0E94A8586AEE7BE00E94915884
:10F41000BC018FE992E10E944A59CE0180960E9478
:10F420009859CE0186960E949859CE018C960E94DA
:10F430009859CE01C2960E94985962E370E080E02C
:10F4400090E00E94635184E59EE00E94295D62E3A2
:10F4500070E080E090E00E946351EB960FB6F89464
:10F46000DEBF0FBECDBFDF91CF911F910F91FF90F7
:10F47000EF90DF90CF90BF90AF909F908F907F9054
:10F480006F905F904F903F9008950C8110E0102F87
:10F4900000278D81080F111DEE80F12CFE2CEE242B
:10F4A0008F81E80EF11CC884D12CDC2CCC248985FA
:10F4B000C80ED11C33243394E9CE63EE73E18FE997
:10F4C00092E10E940F596FE972E1CE0180960E948D
:10F4D0007A5A4AE050E060E070E0CE0180960E94E7
:10F4E0009832CE0180960E94985960ED73E18FE9C1
:10F4F00092E10E940F598091C30C9091C40C029725
:10F5000009F09BCF1092C40C1092C30C96CFCF92EF
:10F51000DF92EF92FF92CF93DF93CDB7DEB72C97B8
:10F520000FB6F894DEBF0FBECDBF99270E9440945E
:10F53000BC01990F880B990B0E94C8B22DE038E6E8
:10F5400043E55BE30E9427B36B017C0120916B02D2
:10F5500030916C0240916D0250916E020E94C2B2D5
:10F5600018164CF06091530270915402809155022C
:10F57000909156021BC020917F02309180024091F1
:10F58000810250918202C701B6010E9407B687FF2F
:10F5900005C0C701B6010E94006808C060916702FB
:10F5A000709168028091690290916A0220E030E0D7
:10F5B00048EC52E40E9427B320E030E048EA51E4EE
:10F5C0000E9427B320912305309124054091250501
:10F5D000509126050E9418B56B017C0168EC73E11F
:10F5E00089E992E10E940F5969E972E1CE01019621
:10F5F0000E947A5A42E350E060E070E0CE0101964A
:10F600000E94D133CE0101960E94985922E0B701A1
:10F61000A601CE0107960E94CC5968E376E0CE01A0
:10F6200001960E94825ABE01695F7F4FCE0101960A
:10F630000E94A85860EF7BE00E949158BC018FE9BE
:10F6400092E10E944A59CE0101960E949859CE013A
:10F6500007960E9498596FE972E1CE0101960E94C7
:10F660007A5A42E350E06FEF7FEFCE0101960E949D
:10F670009832CE0101960E9498598091B013882348
:10F6800031F060E273E080E090E00E9463512C96DC
:10F690000FB6F894DEBF0FBECDBFDF91CF91FF90C4
:10F6A000EF90DF90CF9008951F93CF93DF93182FA3
:10F6B000CBE1DDE0812F0E941951899399936CE38E
:10F6C00070E080E090E00E9463518DE0CB36D80777
:10F6D00089F70E94E06620E030E040EA50E40E94B2
:10F6E00027B320E030E040E85AE30E9427B3DF91DF
:10F6F000CF911F9108958F929F92AF92BF92EF92F8
:10F70000FF920F931F93CF93DF93D82FC62F1092A2
:10F71000FB121092FC121092FD121092FE12109227
:10F72000FF1261E00E94DA5060E08D2F0E94A85025
:10F730006C2F70E080E090E00E94635160E08D2FBC
:10F740000E94DA508BE990E00197F1F700E911E0AF
:10F750008D2F0E944B5D892B31F401501109C1F7A7
:10F760008EEF9FEF51C000E911E08D2F0E944B5D9D
:10F77000019721F401501109C1F7F2CF18E2C0E856
:10F7800000E020E9E22EFF24F3948D2F0E944B5DD0
:10F79000892B29F481E0E81AF108B9F7E1CF0E943A
:10F7A0003E514B015C0190E9E92EFF24F3948D2F2B
:10F7B0000E944B5D019729F481E0E81AF108B9F73E
:10F7C000CFCF0E943E51DC01CB0188199909AA09CB
:10F7D000BB098997A105B10538F0E02FF0E0ED50A5
:10F7E000FD4E80858C2B80872C2F30E0359527951A
:10F7F0002115310511F0C22F02C00F5FC0E8115072
:10F8000009F0BFCF80E090E0DF91CF911F910F9181
:10F81000FF90EF90BF90AF909F908F900895EF92E0
:10F82000FF920F931F93CF93DF93C82F8B017A0121
:10F8300083E50E9496656C2F8BE290E10E94FF8B1E
:10F840000E948F6583E50E949665B80183E590E08C
:10F850003FD5E701CE018E199F0930916B0D2091A4
:10F860006C0D321731F08BE290E10E94B48B8993DA
:10F87000F1CF8017910729F01092011381E0809356
:10F880000213DF91CF911F910F91FF90EF900C9495
:10F890008F65CF93DF93AC01990F660B770B2AE04E
:10F8A00030E08EE89FE00E94705BEC018EE89FE004
:10F8B0000E94BD5B8C0F9D1FDF91CF9108951F9318
:10F8C000CF93DF931F92CDB7DEB7162FAE014F5FF8
:10F8D0005F4F61E070E0A3DF898190E002C0959501
:10F8E00087951A95E2F781700F90DF91CF911F9164
:10F8F0000895CF93DF93D82FC62F83E50E94966596
:10F900006D2F8BE290E10E94FF8B6C2F8BE290E1D8
:10F910000E94FF8BDF91CF910C948F65FF920F9324
:10F920001F93CF93DF931F92CDB7DEB7182F062F0B
:10F93000F42EAE014F5F5F4F61E070E070DF8981B0
:10F94000FF2049F041E050E001C0440F0A95EAF77A
:10F95000482B498309C021E030E001C0220F0A95FD
:10F96000EAF72095282329836981812FC2DF0F9030
:10F97000DF91CF911F910F91FF900895CF93DF9367
:10F9800042E00E94DC65EC018EE89FE00E94BD5BD6
:10F990008C0F9D1FDF91CF910895AF92BF92CF92B0
:10F9A000DF92EF92FF921F93CF93DF93CDB7DEB735
:10F9B0002A970FB6F894DEBF0FBECDBF182F4FE0C9
:10F9C00053E166E070E082E39F8329DF209110130A
:10F9D00030E0322F222780910F13282B3A8329837E
:10F9E0002091121330E0322F222780911113282BFF
:10F9F0003C832B832091141330E0322F22278091F7
:10FA00001313282B3E832D839E012F5F3F4F5901F7
:10FA100053E0C52E53E1D52EE12E9F81F92EF5013D
:10FA2000619171915F01F601219131914191519163
:10FA30006F01072E000C880B990B2F83388749879D
:10FA40005A870E94C8B22F81388549855A850E94FD
:10FA500027B3F70161937193819391937F01FFE045
:10FA6000CF16F3E1DF06D9F62A960FB6F894DEBF7B
:10FA70000FBECDBFDF91CF911F91FF90EF90DF9030
:10FA8000CF90BF90AF9008954F925F926F927F9208
:10FA90008F929F92AF92BF92CF92DF92EF92FF929E
:10FAA000CF93DF93CDB7DEB764970FB6F894DEBF80
:10FAB0000FBECDBF7C0165EF7BE089E992E10E943A
:10FAC00035590E94483269E972E1CE0101960E94DF
:10FAD0007A5A4AE050E06FEF7FEFCE0101960E9424
:10FAE000D133CE0101960E949859C701DDDD698BA3
:10FAF0007A8B8B8B9C8B8090150590901605A0902F
:10FB00001705B0901805A501940160911905709131
:10FB10001A0580911B0590911C050E9451B42B0180
:10FB20003C0120E030E0A9010E94C2B2882309F420
:10FB300051C0C0901105D0901205E0901305F090CF
:10FB4000140520E030E0A901C701B6010E94C2B24D
:10FB500018160CF03FC080910D0590910E05A091F4
:10FB60000F05B09110058D879E87AF87B88B9C01DC
:10FB7000AD01C701B6010E94C2B2882359F1A701A5
:10FB800096016D857E858F8598890E9418B50E94A3
:10FB90004DB66D877E878F87988BA5019401698903
:10FBA0007A898B899C890E9451B4A30192010E9499
:10FBB00018B52D853E854F8558890E9427B30E9430
:10FBC00085B59B01AC01C701B6010E9427B36B014B
:10FBD0007C0103C0C12CD12C760169E972E1CE0110
:10FBE00001960E947A5A4AE050E060E070E0CE014F
:10FBF00001960E94D133CE0101960E94985920E0CF
:10FC000030E64AEE56E4C701B6010E9407B6181660
:10FC10003CF467E474E18FE992E10E940F5925C03A
:10FC200021E0B701A601CE0101960E94CC596FEFE9
:10FC30007BE0CE0107960E94825ABE016F5F7F4F24
:10FC4000CE0107960E94A85863E07CE00E9491587C
:10FC5000BC018FE992E10E944A59CE0107960E94A9
:10FC60009859CE0101960E9498596FE972E1CE0130
:10FC700001960E947A5A4AE050E06FEF7FEFCE0182
:10FC800001960E949832CE0101960E94985964E62E
:10FC900070E080E090E00E9463518091B01388236F
:10FCA00031F060E273E080E090E00E94635164967E
:10FCB0000FB6F894DEBF0FBECDBFDF91CF91FF909E
:10FCC000EF90DF90CF90BF90AF909F908F907F90FC
:10FCD0006F905F904F900895AF92BF92CF92DF9256
:10FCE000EF92FF920F931F93CF93DF931F92CDB7A5
:10FCF000DEB75C01D62EE72EFC018585811105C09B
:10FD0000C5010E94ED52811106C0F50113861586CA
:10FD1000148680E065C040E060EFC5010E9481521A
:10FD200001E0F12CC12C11E0C5010E942E52682F78
:10FD3000C50169830E942E526981613019F48130B6
:10FD4000B9F433C04F2D50E068131BC0F501838513
:10FD5000181730F4E40FF51F8381802349F402C0A3
:10FD6000181731F060E0193058F4F501148708C015
:10FD7000F501EF0DF11D8381802B838361E009C0C4
:10FD8000C12EF501E40FF51F9381802F8095892303
:10FD90008383C5010E9452521F5F000F11F4F39438
:10FDA00001E0F7E0FF1508F0BFCF113408F4ADCF44
:10FDB000F501C386C11002C081E08587F50183810A
:10FDC000882309F4A2CFD5011396ED2DFE2D9501C0
:10FDD000255F3F4F8D918193A217B307D9F781E03B
:10FDE0000F90DF91CF911F910F91FF90EF90DF90D7
:10FDF000CF90BF90AF9008959F92AF92BF92CF9255
:10FE0000DF92EF92FF920F931F93CF93DF93CDB7C3
:10FE1000DEB761970FB6F894DEBF0FBECDBF8C0181
:10FE20008CE0F8018183C12CD12C2FE5E22E3FE735
:10FE3000B32E4FE1A42E5FE3952EF801848190E06C
:10FE4000C816D9060CF0A2C04C2DBE01665F7F4FCC
:10FE5000C8010E94F151F8018181893038F0F82EF3
:10FE6000FCE0F81728F49CE0F92E02C089E0F82E97
:10FE70008A85803139F0BE01665F7F4FC8010E94DC
:10FE8000F55301C08CE08F1509F47CC0AE014F5FC3
:10FE90005F4FBE01665F7F4FC8010E948C5388236D
:10FEA00009F470C08A85803109F46CC08BE0F816C3
:10FEB00051F0ECE0FE1629F0FAE0FF1206C09D8238
:10FEC00005C0BD8203C0ED8201C0AD82F80186810C
:10FED00097810E94ED52BE01665F7F4FF8018681D7
:10FEE00097810E94C25240E06EE4F80186819781BA
:10FEF0000E94815240E06B81F801868197810E94C7
:10FF0000815240E06C81F801868197810E94815284
:10FF10008A85803139F040E06D81F80186819781D2
:10FF20000E948152F801868197810E94ED52BE01A4
:10FF3000665F7F4FF801868197810E94C252F80167
:10FF4000408168E4868197810E94815264E170E07B
:10FF500080E090E00E946351F8018081882331F0B5
:10FF60006AE070E080E090E00E946351F8018681D1
:10FF700097810E94ED52F8018181F81608F4F82E5D
:10FF8000F801F182FFEFCF1ADF0A57CF61960FB663
:10FF9000F894DEBF0FBECDBFDF91CF911F910F91BF
:10FFA000FF90EF90DF90CF90BF90AF909F9008951B
:10FFB0006F927F928F929F92AF92BF92CF92DF9279
:10FFC000EF92FF920F931F93CF93DF93CDB7DEB7DE
:10FFD0002C970FB6F894DEBF0FBECDBF7C015B013E
:10FFE0004A0162EC79E00E94825A62EC79E0CE012B
:10FFF00007960E94825AC12CD12C35018FEF681AC6
:020000021000EC
:10000000780A8E010F5F1F4FC814D9040CF084C00A
:10001000F701848195818615970508F07DC0B501AB
:10002000C8010E94A88AB801CE0107960E945F59B4
:10003000C8010E94985964E170E080E090E00E945D
:1000400063518B859C85892B61F4B501C8010E94A1
:100050004389B801CE0107960E945F59C8010E94EA
:1000600098598B859C85892B79F062EB77E08F819D
:1000700098850E9416BA892BD9F4F701248135811D
:100080002115310569F514C064E170E080E090E06D
:100090000E946351F701848195818A159B0520F4A4
:1000A000FFEFCF1ADF0AB0CF85E1C80ED11CACCF6D
:1000B000BE01695F7F4FC7010E940959F2E3CF1A61
:1000C000D108B701C8010E947A5A42E350E06FEFAD
:1000D0007FEFC8010E949832C8010E949859DACF78
:1000E0002230310530F462EC79E0C7010E943559C5
:1000F000E5CF2150310940E050E0B701C8010E942E
:10010000965AE016F10621F0B801C7010E945F5926
:10011000C8010E949859D2CFCE0107960E949859E3
:10012000C7012C960FB6F894DEBF0FBECDBFDF918E
:10013000CF911F910F91FF90EF90DF90CF90BF90E4
:10014000AF909F908F907F906F90089596E0899FD9
:10015000D0011124AB5EBC4E90967C936E935F975A
:1001600091E091969C93919790918113E0918213E5
:10017000F0918313992339F0309751F0811108C021
:100180008091311304C0309719F05C968C911994CA
:1001900008950F931F93CF93DF93C82FD62F86E038
:1001A000C89FF0011124EB5EFC4E11A2878D90A137
:1001B00081309105E9F01CF4892B49F041C082306F
:1001C0009105A1F10397E1F560E070E033C066238B
:1001D000B9F161E070E08C2FB9DF0E949B51609310
:1001E0006D1370936E1380936F139093701328C0E8
:1001F0000E949B5100916D1310916E1320916F130B
:1002000030917013AB01BC01401B510B620B730B9F
:1002100080917F1390918013A0E0B0E08417950740
:10022000A607B70718F462E070E004C0D11108C057
:1002300063E070E08C2FDF91CF911F910F9186CFFB
:10024000DF91CF911F910F9108950F931F93CF933B
:10025000DF931F92CDB7DEB7682F80918713698334
:100260000E94966569818BE290E10E94FF8B80E09D
:100270000E94326563E0809187130E94796A8BE265
:1002800090E10E94B48B8C018BE290E10E94B48BD0
:1002900020E030E0382FC901802B912B0F90DF91A7
:1002A000CF911F910F91089586E0CFDFBC0180E0D0
:1002B00090E00E94C6B22AE037ED43EA5CE30E9478
:1002C00027B323E333E948E853E40C9451B4089589
:1002D000613208F060E20E94356A10926C0D8093E2
:1002E0006B0D08951F93CF93DF931F92CDB7DEB7A9
:1002F000682F87E769830E94966569818BE290E1A8
:100300000E94FF8B0E948F6587E70E94966561E0DF
:1003100070E087E790E0DCDF8BE290E10E94B48B35
:10032000182F0E948F65812F0F90DF91CF911F9121
:1003300008950F931F93CF93DF931F92CDB7DEB72E
:10034000682F87E769830E94966569818BE290E157
:100350000E94FF8B0E948F6587E70E94966562E08E
:1003600070E087E790E0B4DF8BE290E10E94B48B0D
:1003700000E010E0182F8BE290E10E94B48B082B74
:10038000192B0E948F65C8010F90DF91CF911F91AB
:100390000F91089587E70E94966564EF8BE290E1E4
:1003A0000E94FF8B6EE28BE290E10E94FF8B0E9425
:1003B0008F6565E070E080E090E00E94635186EF19
:1003C000B8CF3F924F925F926F927F928F929F929F
:1003D000AF92BF92CF92DF92EF92FF920F931F9353
:1003E000CF93DF93CDB7DEB728970FB6F894DEBF73
:1003F0000FBECDBFCFDF6C01E12CF12C1091BD12EF
:100400001295110F110F107C1C5C87E70E949665F6
:1004100064EF8BE290E10E94FF8B612F8BE290E111
:100420000E94FF8B0E948F658091BD12811105C0D3
:1004300065E070E080E090E012C0813029F468E06F
:1004400070E080E090E00BC0823029F46EE070E054
:1004500080E090E004C06AE170E080E090E00E94FB
:10046000635186EF66DF4C01A12CB12CBA2CA92C6C
:10047000982C882488EF36DF882A3090BD1280912E
:10048000D2129091D312A7019601281B390B410972
:100490005109A091D012B091D1120E9410B46B01F9
:1004A0007C01AFE0F594E794D794C794AA95D1F76F
:1004B0006091CA127091CB12CB01770FAA0BBB0BC4
:1004C000BC01CD01BBE0660F771F881F991FBA954D
:1004D000D1F72091CC123091CD128901330F220B2C
:1004E000330BA90198012C0D3D1D4E1D5F1D0E946F
:1004F000F4B3C20ED31EE41EF51E20EAC21A2FE08A
:10050000D20AE108F108A7019601C701B6010E94CD
:100510006AB79B01AC011CE0559547953795279527
:100520001A95D1F729833A834B835C830091BE12DD
:100530001091BF12A091C212B091C312A7019601EF
:100540000E941AB42B013C018DE075946794579476
:1005500047948A95D1F7A091C412B091C512298110
:100560003A814B815C810E941AB4BB2797FDB095FC
:10057000AB2F840D951DA61DB71D0296A11DB11DA3
:1005800032E0B595A795979587953A95D1F79C0157
:10059000AD0130584F4F5F4FA091CE12B091CF12A6
:1005A0000E9410B42B013C014FE07694679457945D
:1005B00047944A95D1F788E090E083199109A50105
:1005C000940104C056954795379527958A95D2F79B
:1005D0002D833E834F8358874801110FAA08BB081B
:1005E00052E0880C991CAA1CBB1C5A95D1F7A0910B
:1005F000C612B091C71229813A814B815C810E9459
:100600001AB49B01AC016BE055954795379527953A
:100610006A95D1F729833A834B835C83A091C012FA
:10062000B091C112A70196010E941AB4DC01CB015E
:100630007BE0B595A795979587957A95D1F7298110
:100640003A814B815C81820F931FA41FB51F880DD7
:10065000991DAA1DBB1D032C04C0880F991FAA1F3A
:10066000BB1F0A94D2F7BC01CD016E5F7F4F8F4F45
:100670009F4F24E030E040E050E00E94F4B38D81D1
:100680009E81AF81B885821B930BA40BB50B9C0197
:10069000AD0180E593ECA0E0B0E0BC01CD0104C069
:1006A00096958795779567953A94D2F70E946AB7A1
:1006B00097FD0BC0660F771F881F991FA30192013A
:1006C0000E9420B469017A010AC0A30192010E942C
:1006D00020B469017A01CC0CDD1CEE1CFF1C9927AB
:1006E000F7FC9A958F2D7E2D6D2D9B01AC010E94FC
:1006F0006AB79B01AC01AEEDBBE00E9410B44C01A7
:10070000BB2497FCB094AB2CA3E4B3EEA7019601F5
:100710000E941CB4BB2797FDB095AB2F880D991D87
:10072000AA1DBB1D8153914FAF4FBF4F44E0B595FC
:10073000A795979587954A95D1F7BC01CD016C0D8A
:100740007D1D8E1D9F1D28960FB6F894DEBF0FBE2F
:10075000CDBFDF91CF911F910F91FF90EF90DF9070
:10076000CF90BF90AF909F908F907F906F905F9051
:100770004F903F900895CF92DF92EF92FF920F93A8
:100780001F9308DEAC0160E070E0EDEBF2E18589DB
:1007900096899A01AB01281B390B41095109A3899C
:1007A000B4890E9410B46B017C018FE0F594E7944A
:1007B000D794C7948A95D1F765857685CB01770F55
:1007C000AA0BBB0BBC01CD012BE0660F771F881F66
:1007D000991F2A95D1F7278530898901330F220B7C
:1007E000330BA90198012C0D3D1D4E1D5F1D0E946C
:1007F000F4B3D701C601820F931FA41FB51F08963B
:10080000A11DB11DBC01CD0134E09595879577956B
:1008100067953A95D1F70E94C8B220E030E040E2F7
:1008200051E40E9418B51F910F91FF90EF90DF9057
:10083000CF9008956F927F928F929F92AF92BF92C6
:10084000CF92DF92EF92FF920F931F93CF93DF939C
:1008500081E0809381130E949B510091711310914C
:1008600072132091731330917413AB01BC01401BC0
:10087000510B620B730B80917D1390917E13A0E05E
:10088000B0E084179507A607B70708F00AC1C0E0D3
:1008900080917B13C81760F4E0917713F09178137F
:1008A000EC0FF11D62E080810E94DA50CF5FF0CF43
:1008B000712C812C912C5401839480917C13781697
:1008C00008F05FC0072D10E0E0917913F0917A13E2
:1008D000E00FF11F61E080810E94DA50E09179130E
:1008E000F0917A13E00FF11F60E080810E94A85020
:1008F000D501C401072C04C0880F991FAA1FBB1F74
:100900000A94D2F76C017C01E094F094612C809100
:100910007B136816F8F4C62DD0E0E0917713F091C0
:100920007813EC0FFD1F80810E944B5D2496CC0F45
:10093000DD1FCB5EDC4E892B29F4888199818C29BF
:100940009D2904C0888199818E219F219983888364
:100950006394DDCFE0917913F0917A13E00FF11FEA
:1009600061E080810E94A8508091791390917A1360
:10097000FC01E00FF11F60E080810E94DA50739467
:100980009CCFE1E3F3E18FEF9FEF23813481232BB1
:1009900021F41082928381831582369623E1ED360D
:1009A000F20799F710E096E0F92E80917B13181763
:1009B00008F051C000E0C12FD0E0CC0FDD1FC35EB6
:1009C000DC4E20917C13021708F043C068817981C6
:1009D000002E02C0769567950A94E2F7617077273A
:1009E000129F90011124200F311DE0917513F09199
:1009F0007613E20FF31F4081E5E1F3E180E0A58D7E
:100A0000B68DA217B30711F461701AC08F5F3696C6
:100A10008A30A9F7672BD9F0E1E3F3E180E090E0B9
:100A2000508151110FC0F89EF001F99EF00D112474
:100A3000EB5EFC4E448F368F258F10A2178E61E03F
:100A4000A8DB05C0019636968A30910549F70F5FFD
:100A5000B8CF1F5FAACF80E090E0C0E0FC01EB5E62
:100A6000FC4E21A12111C1E006968C339105B1F70E
:100A70000E949B5160937113709372138093731350
:100A800090937413CC2369F080913613882349F036
:100A90008091341390913513019719F4809131139B
:100AA00003C01092811380E0DF91CF911F910F91CD
:100AB000FF90EF90DF90CF90BF90AF909F908F907E
:100AC0007F906F9008958F929F92AF92BF92CF9236
:100AD000DF92EF92FF920F931F93CF93DF93DB018F
:100AE000CD91DC91DC011C96ED91FC911D97CE1708
:100AF000DF070CF047C0FE01EE0FFF1F1A968D9125
:100B00009C911B97E80FF91F80809180C170DD27B1
:100B1000B1E0CB27209719F404E610E002C00CE9FD
:100B20001FEF79015A016B01020F131FB801C401B5
:100B300058D7892B89F40E0D1F1DB801C40151D758
:100B4000892B69F4B8016E0D7F1DC4014AD7892B2A
:100B5000E1F023E030E005C021E030E002C022E017
:100B600030E0F5018081918101968217930734F07E
:100B700011821082F6018081918101969183808398
:100B8000CE0105C081E090E002C08FEF9FEFDF91C2
:100B9000CF911F910F91FF90EF90DF90CF90BF907A
:100BA000AF909F908F900895CF93DF93EC014830E2
:100BB00085E058076105710509F441C108F08DC051
:100BC000493481E058076105710509F43BC1E0F53E
:100BD000443481E058076105710509F424C1E8F443
:100BE000413481E058076105710509F413C138F4F7
:100BF000403451406105710509F409C135C14234E1
:100C000081E058076105710509F407C1433451407B
:100C10006105710509F404C127C1463481E0580714
:100C20006105710509F405C108F400C1473481E08C
:100C300058076105710509F4FFC04834514061054A
:100C4000710509F4FCC010C1423085E05807610508
:100C5000710509F4E2C0E8F4443781E05807610502
:100C6000710509F4F5C038F442375140610571054A
:100C700009F4F1C0F9C0411585E058076105710517
:100C800009F4C5C0413055406105710509F4C2C081
:100C9000EBC0453085E058076105710509F4C6C011
:100CA00070F4433085E058076105710509F4B8C058
:100CB000443055406105710509F4B5C0D5C04630D2
:100CC00085E058076105710509F4B3C04730554008
:100CD0006105710509F4B0C0C7C04D3B82E45807F7
:100CE0008FEF6807710509F4BCC008F045C04F3E9E
:100CF00080E158078FEF6807710509F49DC0E8F49B
:100D0000423385E058076105710509F4A4C038F441
:100D1000493055406105710509F494C0A5C04433BC
:100D200085E058076105710509F492C04D3F5240B6
:100D30006F4F710509F48FC097C04D3D82E258078F
:100D40008FEF6807710509F483C038F4473E5841B6
:100D50006F4F710509F46AC087C04F3C80E35807A4
:100D60008FEF6807710509F45EC0473C58436F4F29
:100D7000710509F464C078C0473988E658078FEFD9
:100D80006807710509F446C000F54D3A82E5580739
:100D90008FEF6807710509F461C030F4453B5A4490
:100DA0006F4F7105A1F160C0453A8AE558078FEF92
:100DB0006807710509F446C04D3952466F4F7105F9
:100DC00009F052C06CE976E051C0473588EA58070F
:100DD0008FEF68077105C9F168F445388AE758074D
:100DE0008FEF6807710529F1473658496F4F710534
:100DF000A1F03AC04F3480EB58078FEF68077105B8
:100E000079F04D33524C6F4F710529F12DC06DE0D3
:100E10007AE02CC061E87BE029C06EE77BE026C069
:100E20006BE77BE023C068E77BE020C065E77BE001
:100E30001DC067E07CE01AC069E07CE017C06BE091
:100E40007CE014C06DE17AE011C062EB77E00EC087
:100E500068ED7BE00BC06DE078E008C06CEE79E0F7
:100E600005C06DE07CE002C062EC79E0CE010E943A
:100E7000825ACE01DF91CF910895DF92EF92FF92D7
:100E80000F931F93CF93DF93CDB7DEB762970FB663
:100E9000F894DEBF0FBECDBF8C011092D21362EC6E
:100EA00079E0CE0101960E94825AFF24F3948EE8E5
:100EB0009FE00E941E562091D21318161906ECF5D9
:100EC00021113BC08EE89FE00E94FC55682F809363
:100ED000D1138A3039F06D3029F0CE0101960E948D
:100EE000E85824C08D819E81892B01F1F092D213A4
:100EF0006FE07CE0CE0107960E94825ABE016F5FD0
:100F00007F4FCE0107960E94A858BC01CE010D96D6
:100F10000E947A5ACE010D960E947238CE010D962B
:100F20000E949859CE0107960E9498596AE070E095
:100F300080E090E00E946351BACF222351F02091CB
:100F4000D2138D819E812111A5C0009709F0A2C006
:100F500078C0E12CF12CDD24D39487EB9DE00E9436
:100F60001E561816190624F587EB9DE00E94FC55C5
:100F7000682F8093D1138A3071F08D3061F08091A9
:100F8000D213811108C0CE0101960E94E8588FEF5C
:100F9000E81AF80A06C08D819E81892B11F0D09243
:100FA000D21365E070E080E090E00E946351D5CFFD
:100FB00064E170E080E090E00E946351EF2809F462
:100FC000BECF8D819E81892B09F4B9CF8091C50C4C
:100FD000882361F16CEE79E0CE0107960E94825A77
:100FE000BE01695F7F4FCE0101960E947658F82EB0
:100FF000CE0107960E949859F11018C068E17CE074
:101000008EE89FE00E94E05BBE016F5F7F4FCE01E4
:1010100007960E947A5ABE01695F7F4F8EE89FE073
:101020000E94D05BCE0107960E94985987EB9DE005
:101030000E94B55664E170E080E090E00E94635148
:101040007ECF64E670E080E090E00E9463510E94F1
:101050009B51CB0168EE73E00E948DB7CB0164E633
:1010600070E00E948DB78236910574F08091B013C4
:1010700081110AC08BEA92E10E949157613071059B
:101080008105910509F456C062EC79E0C8010E941F
:10109000825A53C0019709F046C062EE75E0CE0156
:1010A0000D960E94825ABE01635F7F4FCE0101966A
:1010B0000E947658811116C068E077E0CE0107964D
:1010C0000E94825ABE01695F7F4FCE0101960E9445
:1010D0007658FF24F3948111F12CCE0107960E94DB
:1010E000985901C0F12CCE010D960E949859FF200D
:1010F000A1F040E050E0BE016F5F7F4FCE01079648
:101100000E943B3EBE01695F7F4F8BEA92E10E94E5
:101110005F59CE0107960E94985964E170E080E023
:1011200090E00E946351BE016F5F7F4FC8010E9433
:101130006A5A03C00E947097A7CFCE0101960E9401
:101140009859C80162960FB6F894DEBF0FBECDBFA6
:10115000DF91CF911F910F91FF90EF90DF90089555
:10116000DF92EF92FF920F931F93CF93DF93CDB750
:10117000DEB72C970FB6F894DEBF0FBECDBF8C0143
:101180001092D21362EC79E0CE0101960E94825A4D
:10119000E12CF12CDD24D39487EB9DE00E941E56B8
:1011A0001816190624F48091D213882301F162E302
:1011B00070E080E090E00E946351EF2851F087EBEF
:1011C0009DE00E94B55664E670E080E090E00E94E9
:1011D00063518091D21381112AC08D819E81892B08
:1011E00031F562EC79E0C8010E94825A39C087EB80
:1011F0009DE00E94FC55682F8093D1138A3051F0F6
:101200006D3041F0CE0101960E94E8588FEFE81A48
:10121000F80A06C08D819E81892B11F0D092D213DD
:101220006FE070E080E090E00E946351B5CF809164
:10123000C50C882379F0BE016F5F7F4FCE01079602
:101240000E947A5ACE0107960E94439ACE010796D1
:101250000E949859BE016F5F7F4FC8010E946A5A71
:10126000CE0101960E949859C8012C960FB6F894A9
:10127000DEBF0FBECDBFDF91CF911F910F91FF90C9
:10128000EF90DF9008957F928F929F92AF92BF92DE
:10129000CF92DF92EF92FF920F931F93CF93DF9342
:1012A000CDB7DEB762970FB6F894DEBF0FBECDBFE5
:1012B0008C017B0181EC93E10E949E1F892B31F40C
:1012C00062EC79E0C8010E94825A2DC14091C51399
:1012D0005091C6136091C7137091C813CE01079641
:1012E00063DC8091C50C882359F16FE17CE0CE016D
:1012F00001960E94825ABE01695F7F4FCE0101961E
:101300000E94A8586BEF77E00E949158BC018EE8CC
:101310009FE00E94E15ACE0101960E9498594091A7
:10132000C5135091C6136091C7137091C81320E183
:101330008EE89FE00E94285B8EE89FE00E94BD5BE4
:1013400060E070E0CE0107960E946558D82E8AE2D0
:10135000D8121092AB130E949B516093A713709305
:10136000A8138093A9139093AA1362EC79E0CE019D
:1013700001960E94825A2D2DDD0C330B205331092A
:101380002A30310508F069C0CE0107960E949157B6
:1013900063307105810591050CF0ACC0CC24C39479
:1013A000D12C92E0792ECE14DF040CF0A3C06CE2B5
:1013B00071E080E090E00E946351709237101092CB
:1013C0003B10812C912C540181EB93E10E949E1FD4
:1013D000892B91F48EE188169104A104B10441F1A6
:1013E0006EE170E080E090E00E9463518FEF881A18
:1013F000980AA80AB80AE8CF8EE188169104A104D9
:10140000B104B1F04091B5135091B6136091B71388
:101410007091B813CE010D96C7DBBE01635F7F4F9D
:10142000CE0101960E945F59CE010D960E949859F7
:101430008D819E81892B39F0BE016F5F7F4FCE0178
:1014400007960E9409598FEFC81AD80A62EC79E012
:10145000CE0101960E943559A6CF6CE271E080E082
:1014600090E00E94635182E08093371010923B100D
:10147000C12CD12C760181EB93E10E949E1F892B18
:1014800091F48EE1C816D104E104F10441F16EE15A
:1014900070E080E090E00E9463518FEFC81AD80A94
:1014A000E80AF80AE8CF8EE1C816D104E104F10495
:1014B000B1F04091B5135091B6136091B71370918C
:1014C000B813CE010D9670DBBE01635F7F4FCE0176
:1014D00001960E945F59CE010D960E9498598D8108
:1014E0009E81892B39F0BE016F5F7F4FCE01079639
:1014F0000E94095964E670E080E090E00E94635128
:1015000082E08093371010923B10BE01695F7F4FDD
:10151000C8010E946A5ACE0101960E949859CE01D4
:1015200007960E949859C80162960FB6F894DEBFDC
:101530000FBECDBFDF91CF911F910F91FF90EF9024
:10154000DF90CF90BF90AF909F908F907F90089545
:10155000AF92BF92CF92DF92EF92FF920F931F93C1
:10156000CF93DF93CDB7DEB72C970FB6F894DEBFDD
:101570000FBECDBF7C015B015DD9182F811106C064
:1015800062EC79E0C7010E94825A9AC08A3211F057
:101590001092AB130E949B516093A7137093A813F2
:1015A0008093A9139093AA13612FCE0101960E94F4
:1015B000525A812F012E000C990BC0970A9750F5B3
:1015C000CE0101960E949157633071058105910506
:1015D0000CF04BC001E010E00A151B050CF045C0F3
:1015E00062E370E080E090E00E94635123D9C12C57
:1015F000D12C811152C08FEFC81AD80A85E1C816C4
:10160000D10499F16EE170E080E090E00E946351B6
:1016100011D9EFCF612FCE0107960E94525ABE0119
:10162000695F7F4FCE0101960E945F59CE010796F8
:101630000E94985962E370E080E090E00E9463515C
:10164000F9D800E010E08823D9F0682FCE01079682
:101650000E94525ABE01695F7F4FCE0101960E94DF
:101660000959CE0107960E949859BE016F5F7F4FBE
:10167000C7010E946A5ACE0101960E94985920C063
:101680000F5F1F4F0F31110581F36EE170E080E0B5
:1016900090E00E946351CED8D6CF682FCE01079636
:1016A0000E94525ABE01695F7F4FCE0101960E948F
:1016B0000959CE0107960E9498590F5F1F4F8CCF92
:1016C000C7012C960FB6F894DEBF0FBECDBFDF91D9
:1016D000CF911F910F91FF90EF90DF90CF90BF902F
:1016E000AF90089585ED8093BC008091BC0084FD8F
:1016F000FCCF1092930D08954091F513262F30E002
:10170000240F311D21323105DCF42091930D24305A
:10171000C9F4FC0180E090E0861758F43091F5138D
:101720002191DC01AD52BC4EA30FB11D2C9301964B
:10173000F3CF8091F513680F6093F51380E008955F
:1017400081E0089582E008950895E0916C0D809104
:101750006B0DE81730F4F0E0E750F34F808190E034
:1017600008958FEF9FEF089590916C0D80916B0D10
:10177000981750F4E92FF0E0E750F34F208130E064
:101780009F5F90936C0D02C02FEF3FEFC90108954A
:1017900080916B0D90E020916C0D821B9109089552
:1017A000CF92DF92EF92FF920F931F93CF93DF932D
:1017B0007C01262F972F8A018091940D882391F028
:1017C000C62FD72F6E01C40ED51ECC15DD0569F0CE
:1017D0006991D701ED91FC910190F081E02DC70155
:1017E0001995F3CF642F822F87DFC801DF91CF9146
:1017F0001F910F91FF90EF90DF90CF900895CF93BE
:10180000DF931F92CDB7DEB769832091940D222319
:10181000D1F02091B60D203240F021E030E0FC0103
:101820003383228380E090E014C08091950DE82FEF
:10183000F0E0EA56F24F998190838F5F8093950D87
:101840008093B60D04C061E0CE01019655DF81E0C2
:1018500090E00F90DF91CF910895089580E090E09F
:1018600008950C9474B81F920F920FB60F92112422
:101870000BB60F922F933F934F935F936F937F938A
:101880008F939F93AF93BF93EF93FF938091381003
:101890000E944B5D20913C1030913D102F5F3F4FD7
:1018A00030933D1020933C1090913B10953618F0EA
:1018B00096E090933710909137109430C9F128F446
:1018C000923069F09330D1F05EC0953009F451C088
:1018D000963009F058C091E09093081151C08111E1
:1018E00052C020913C1030913D102436310508F44F
:1018F00042C01092081110923B101CC0813009F0B8
:1019000042C0E0913B1091E09E0F90933B10F0E0BD
:1019100020913C1030913D10EE0FFF1FE95CFF4E0F
:101920003087278310923D1010923C1094E029C01C
:10193000811117C0E0913B1091E09E0F90933B10F6
:10194000F0E020913C1030913D10EE0FFF1FE95C5C
:10195000FF4E3087278310923D1010923C1093E089
:1019600010C020913C1030913D102536310558F0C3
:1019700007C0811108C010923D1010923C1003C0A6
:1019800095E09093371090913A109923B9F0811116
:101990000AC080913910882321F08091391061E0CC
:1019A00009C02F9A0BC080913910882331F08091A3
:1019B000391060E00E94A85001C02F98FF91EF916C
:1019C000BF91AF919F918F917F916F915F914F9157
:1019D0003F912F910F900BBE0F900FBE0F901F9055
:1019E0001895CF92DF92EF92FF92CF93DF93EC01A5
:1019F000072E000C880B990B0E94C8B26B017C016A
:101A000020E030E040E45FE30E9427B320E030E0D4
:101A100048E452E40E9418B50E94B1B5C617D70732
:101A2000D4F020E030E040EA5FE3C701B6010E9455
:101A300027B320E030E048E452E40E9418B520E0EB
:101A400030E040E85FE30E9452B40E94B1B521E06B
:101A50006C177D070CF420E0822F90E0DF91CF918E
:101A6000FF90EF90DF90CF9008950F931F93CF9347
:101A7000DF93082F68ED7BE08EE89FE00E94E05B3B
:101A8000C7E0D0E010E0B8010C2E02C07595679554
:101A90000A94E2F76170772742E050E08EE89FE019
:101AA0000E94B75B219778F7DF91CF911F910F913B
:101AB00008951F920F920FB60F9211240BB60F923A
:101AC0002F933F934F935F936F937F938F939F9346
:101AD000AF93BF93EF93FF938091B900887F8036D7
:101AE00009F49CC068F5883209F45BC090F4803139
:101AF00009F454C038F4882309F4F6C0883009F496
:101B00004DC0F5C0883109F44CC0803209F45DC085
:101B1000EEC0803409F468C048F4803309F455C03D
:101B2000883309F0E4C08093910DD8C0803509F462
:101B30004FC0883509F45DC0883409F0D8C0D6C0DC
:101B4000883909F4C7C0A8F4883709F467C038F4A5
:101B5000883609F463C0803709F460C0C8C088388B
:101B600009F4B8C0803909F45FC0803809F0BFC0FB
:101B70005BC0803B09F486C038F4803A09F466C043
:101B8000883A09F47FC0B3C0803C09F4A7C0883C00
:101B900009F4A4C0883B09F48AC0A9C080916E0DE5
:101BA00010C09091900D80918F0D981770F5E09175
:101BB000900D81E08E0F8093900DF0E0E159F24F8F
:101BC00080818093BB0085EC86C08093910D8EC090
:101BD000E091900D81E08E0F8093900D8091BB007D
:101BE000F0E0E159F24F80839091900D80918F0D3C
:101BF0006EC0E091900D81E08E0F8093900D8091EA
:101C0000BB00F0E0E159F24F80838091920D811189
